S0190000636F756E7465725F6573705F626F6172642E73726563FD
S3150802000000000A204D520508312F0408392F04082A
S31508020010412F0408492F0408512F04089D52050848
S315080200200000000000000000000000009D520508C4
S31508020030592F04080000000035030208E1020208ED
S315080200409D5205089D5205089D5205089D520508B0
S315080200509D5205089D5205089D5205089D520508A0
S315080200609D5205089D5205089D520508672F0408EA
S31508020070752F0408832F0408912F04089F2F04085C
S315080200809D5205089D5205089D5205089D52050870
S315080200909D520508AD2F04089D5205089D52050874
S315080200A09D5205089D520508BD2F04089D52050854
S315080200B09D5205089D5205089D5205089D52050840
S315080200C09D5205089D5205089D5205089D52050830
S315080200D0000000009D5205089D520508CD2F040810
S315080200E09D5205089D5205089D5205089D52050810
S315080200F09D5205089D5205089D5205089D52050800
S315080201009D5205089D5205089D5205089D520508EF
S315080201109D5205089D5205089D5205089D520508DF
S315080201209D5205089D520508E12F04089D520508AF
S315080201309D5205089D5205089D5205089D520508BF
S315080201409D5205089D5205089D5205089D520508AF
S315080201509D5205089D5205089D520508F52F04086B
S315080201609D5205089D5205089D5205089D5205088F
S315080201709D5205089D5205089D5205089D5205087F
S315080201809D5205089D5205089D5205089D5205086F
S315080201909D5205089D5205089D5205089D5205085F
S315080201A09D5205089D520508613004089D520508AE
S315080201B09D5205089D5205089D5205089D5205083F
S315080201C09D5205089D5205089D5205089D5205082F
S315080201D09D5205089D5205089D5205089D5205081F
S315080201E09D5205089D5205089D5205089D5205080F
S315080201F09D5205089D5205089D5205089D520508FF
S315080202009D5205089D5205089D52050800000000EA
S31508020210000000009D520508000000009D520508D6
S315080202209D5205089D5205089D5205089D520508CE
S315080202309D5205089D5205089D5205089D520508BE
S315080202409D5205089D5205089D52050800000000AA
S3150802025010B5054C237833B9044B13B10448AFF3F0
S3150802026000800123237010BD400B0020000000000F
S31508020270A021090808B5034B1BB103490348AFF38C
S31508020280008008BD00000000440B0020A0210908D8
S3150802029072B64FF0E0201749C0F8081D16480168E3
S315080202A041F00101016015481249096801604FF0E1
S315080202B0E020134941614FF0070101614FF0000147
S315080202C0C0F8181D4FF07F41C0F81C1D0D49C0F833
S315080202D0201D7047FFF7FEBF01B5BDE80140704714
S315080202E001B500F097F8BDE801407047FFF7FEBF79
S315080202F0FFF7FEBF00000208001000E0AC3B022038
S315080203008FD003000000FF404FF000002D4A106016
S31508020310EFF3148020F0040080F3148862B64FF0DD
S3150802032080504FF0E021C1F8040DBFF34F8FBFF3A1
S315080203306F8FFEE72448254A4FF00003016891B102
S315080203400360EFF3098C2CE9F00F1EF0100F01D1B0
S315080203502CED108A1E4C4CF804EDC1F808C025682D
S315080203600DB18D61236072B61168D1B1016062B6B2
S315080203704F68174C8D6907F101074F602560D1F860
S315080203800CC08CF30B88D1F808C05CF804EB1EF09D
S31508020390100F01D1BCEC108ABCE8F00F8CF3098867
S315080203A0704772B61168016009B962B6F9E74FF08B
S315080203B000674FF0E028C8F8047D62B6D8E700BFA8
S315080203C070470000483C0220B03B0220B43B0220A2
S315080203D0B4410220026922F00702A2F144026FF038
S315080203E0430313604FF0000353609360D3601361B5
S315080203F053619361D361136253629362D362136347
S3150802040053634FF0FF339363D1634FF080731364E2
S31508020410826070472249086800F101000860214B92
S315080204201A683AB1A2F101021A601AB91E4B4FF0C4
S31508020430010018601D490868026822B11C4B4FF07A
S3150802044001021A6008E000F104001A4B1A68904289
S3150802045001D1194B18680860134B1A6812B9144966
S315080204600868C8B101B51249086808B144F010FD18
S315080204700D4B1A6872B144F07DFC1048016849B9FF
S315080204800F4801680F4A13680F484FF08052994285
S3150802049000D00260BDE80140BFF34F8F70470000ED
S315080204A0543C0220B4410220583C0220E43C02207B
S315080204B0E83C0220E03C0220DC3C0220483C0220C8
S315080204C0B03B0220B43B022004ED00E0034613F8D9
S315080204D0012B002AFBD1181A0138704781F0004116
S315080204E002E000BF83F0004330B54FEA41044FEA09
S315080204F0430594EA050F08BF90EA020F1FBF54EAA4
S31508020500000C55EA020C7FEA645C7FEA655C00F03F
S31508020510E2804FEA5454D4EB5555B8BF6D420CDD10
S315080205202C4480EA020281EA030382EA000083EA93
S31508020530010180EA020281EA0303362D88BF30BD33
S3150802054011F0004F4FEA01314FF4801C4CEA113189
S3150802055002D0404261EB410113F0004F4FEA0333E8
S315080205604CEA133302D0524263EB430394EA050F73
S3150802057000F0A780A4F10104D5F1200E0DDB02FAE2
S315080205800EFC22FA05F2801841F1000103FA0EF276
S31508020590801843FA05F359410EE0A5F120050EF13C
S315080205A0200E012A03FA0EFC28BF4CF0020C43FA6D
S315080205B005F3C01851EBE37101F0004507D54FF07A
S315080205C0000EDCF1000C7EEB00006EEB0101B1F5CA
S315080205D0801F1BD3B1F5001F0CD349085FEA300010
S315080205E04FEA3C0C04F101044FEA445212F5800F1B
S315080205F080F09A80BCF1004F08BF5FEA500C50F1B8
S31508020600000041EB045141EA050130BD5FEA4C0C9A
S31508020610404141EB0101013C28BFB1F5801FE9D2F7
S3150802062091F0000F04BF01460020B1FA81F308BF1A
S315080206302033A3F10B03B3F120020CDA0C3208DDE6
S3150802064002F1140CC2F10C0201FA0CF021FA02F1C1
S315080206500CE002F11402D8BFC2F1200C01FA02F131
S3150802066020FA0CFCDCBF41EA0C019040E41AA2BF56
S3150802067001EB0451294330BD6FEA04041F3C1CDA1E
S315080206800C340EDC04F11404C4F1200220FA04F03E
S3150802069001FA02F340EA030021FA04F345EA0301E8
S315080206A030BDC4F10C04C4F1200220FA02F001FAAA
S315080206B004F340EA0300294630BD21FA04F029462C
S315080206C030BD94F0000F83F4801306BF81F48011C5
S315080206D00134013D4EE77FEA645C18BF7FEA655C38
S315080206E029D094EA050F08BF90EA020F05D054EA0A
S315080206F0000C04BF1946104630BD91EA030F1EBF0F
S315080207000021002030BD5FEA545C05D14000494112
S3150802071028BF41F0004130BD14F580043CBF01F505
S31508020720801130BD01F0004545F0FE4141F47001EB
S315080207304FF0000030BD7FEA645C1ABF19461046C6
S315080207407FEA655C1CBF0B46024650EA013406BFC7
S3150802075052EA033591EA030F41F4002130BD00BF86
S3150802076090F0000F04BF0021704730B54FF4806443
S3150802077004F132044FF000054FF0000150E700BFC4
S3150802078090F0000F04BF0021704730B54FF4806423
S3150802079004F1320410F0004548BF40424FF0000110
S315080207A03EE700BF42004FEAE2014FEA31014FEA53
S315080207B002701FBF12F07F4393F07F4F81F06051A2
S315080207C0704732F07F4208BF704793F07F4F04BFED
S315080207D041F40021704730B54FF4607401F00045CA
S315080207E021F000411CE700BF50EA010208BF70472A
S315080207F030B54FF000050AE050EA010208BF70471B
S3150802080030B511F0004502D5404261EB41014FF483
S31508020810806404F132045FEA915C3FF4D8AE4FF08B
S3150802082003025FEADC0C18BF03325FEADC0C18BF6E
S31508020830033202EBDC02C2F1200300FA03FC20FABF
S3150802084002F001FA03FE40EA0E0021FA02F114440C
S31508020850BDE600BF70B54FF0FF0C4CF4E06C1CEA25
S3150802086011541DBF1CEA135594EA0C0F95EA0C0F96
S3150802087000F0DEF82C4481EA030621EA4C5123EA09
S315080208804C5350EA013518BF52EA033541F4801138
S3150802089043F4801338D0A0FB02CE4FF00005E1FBEB
S315080208A002E506F00042E0FB03E54FF00006E1FB35
S315080208B003569CF0000F18BF4EF0010EA4F1FF0478
S315080208C0B6F5007F64F5407404D25FEA4E0E6D41B8
S315080208D046EB060642EAC62141EA55514FEAC520C9
S315080208E040EA5E504FEACE2EB4F1FD0C88BFBCF545
S315080208F0E06F1ED8BEF1004F08BF5FEA500E50F1F6
S31508020900000041EB045170BD06F0004646EA0101BB
S3150802091040EA020081EA0301B4EB5C04C2BFD4EBED
S315080209200C0541EA045170BD41F480114FF0000EE6
S31508020930013C00F3AB8014F1360FDEBF002001F054
S31508020940004170BDC4F10004203C35DA0C341BDCCE
S3150802095004F11404C4F1200500FA05F320FA04F0A0
S3150802096001FA05F240EA020001F0004221F00041D4
S3150802097010EBD37021FA04F642EB06015EEA430E47
S3150802098008BF20EAD37070BDC4F10C04C4F1200577
S3150802099000FA04F320FA05F001FA04F240EA02002A
S315080209A001F0004110EBD37041F100015EEA430EFB
S315080209B008BF20EAD37070BDC4F1200500FA05F21B
S315080209C04EEA020E20FA04F301FA05F243EA02039A
S315080209D021FA04F001F0004121FA04F220EA0200A9
S315080209E000EBD3705EEA430E08BF20EAD37070BDEF
S315080209F094F0000F0FD101F00046400041EB0101CF
S31508020A0011F4801F08BF013CF7D041EA060195F0B0
S31508020A10000F18BF704703F00046520043EB03036A
S31508020A2013F4801F08BF013DF7D043EA0603704757
S31508020A3094EA0C0F0CEA135518BF95EA0C0F0CD062
S31508020A4050EA410618BF52EA4306D1D181EA0301A8
S31508020A5001F000414FF0000070BD50EA410606BFA2
S31508020A601046194652EA430619D094EA0C0F02D1E7
S31508020A7050EA013613D195EA0C0F05D152EA03362C
S31508020A801CBF104619460AD181EA030101F000414A
S31508020A9041F0FE4141F470014FF0000070BD41F093
S31508020AA0FE4141F4780170BD70B54FF0FF0C4CF46D
S31508020AB0E06C1CEA11541DBF1CEA135594EA0C0F8C
S31508020AC095EA0C0F00F0A7F8A4EB050481EA030ED9
S31508020AD052EA03354FEA013100F088804FEA0333C0
S31508020AE04FF0805545EA131343EA12634FEA02228E
S31508020AF045EA111545EA10654FEA00260EF000414F
S31508020B009D4208BF964244F1FD0404F5407402D2A0
S31508020B105B084FEA3202B61A65EB03055B084FEA31
S31508020B2032024FF480104FF4002CB6EB020E75EB2E
S31508020B30030E22BFB61A754640EA0C005B084FEA56
S31508020B403202B6EB020E75EB030E22BFB61A7546D3
S31508020B5040EA5C005B084FEA3202B6EB020E75EB1E
S31508020B60030E22BFB61A754640EA9C005B084FEA96
S31508020B703202B6EB020E75EB030E22BFB61A7546A3
S31508020B8040EADC0055EA060E18D04FEA051545EA92
S31508020B9016754FEA06164FEAC30343EA52734FEA3B
S31508020BA0C2025FEA1C1CC0D111F4801F0BD141EAB4
S31508020BB000014FF000004FF0004CB6E711F4801F19
S31508020BC004BF01430020B4F1FD0C88BFBCF5E06FF9
S31508020BD03FF6AFAEB5EB030C04BFB6EB020C5FEA09
S31508020BE0500C50F1000041EB045170BD0EF0004E5E
S31508020BF04EEA113114EB5C04C2BFD4EB0C0541EA90
S31508020C00045170BD41F480114FF0000E013C90E68C
S31508020C1045EA060E8DE60CEA135594EA0C0F08BF50
S31508020C2095EA0C0F3FF43BAF94EA0C0F0AD150EA4F
S31508020C3001347FF434AF95EA0C0F7FF425AF1046E2
S31508020C4019462CE795EA0C0F06D152EA03353FF40A
S31508020C50FDAE1046194622E750EA410618BF52EA87
S31508020C6043067FF4C5AE50EA41047FF40DAF52EA5B
S31508020C7043057FF4EBAE12E74FF0FF3C06E000BFF8
S31508020C804FF0010C02E000BF4FF0010C4DF804CD05
S31508020C904FEA410C7FEA6C5C4FEA430C18BF7FEAC5
S31508020CA06C5C1BD001B050EA410C0CBF52EA430CF3
S31508020CB091EA030F02BF90EA020F0020704710F173
S31508020CC0000F91EA030F58BF994208BF90422CBF02
S31508020CD0D8176FEAE37040F0010070474FEA410CFB
S31508020CE07FEA6C5C02D150EA013C07D14FEA430C19
S31508020CF07FEA6C5CD6D152EA033CD3D05DF8040B8A
S31508020D00704700BF8446104662468C4619466346BB
S31508020D1000E000BF01B5FFF7B7FF002848BF10F192
S31508020D20000F01BD4DF808EDFFF7F4FF0CBF0120D7
S31508020D3000205DF808FB00BF4DF808EDFFF7EAFF53
S31508020D4034BF012000205DF808FB00BF4DF808ED0E
S31508020D50FFF7E0FF94BF012000205DF808FB00BF03
S31508020D604DF808EDFFF7CEFF94BF012000205DF88D
S31508020D7008FB00BF4DF808EDFFF7C4FF34BF01209A
S31508020D8000205DF808FB00BF4FEA410C7FEA6C5C65
S31508020D9002D150EA013C0AD14FEA430C7FEA6C5C65
S31508020DA002D152EA033C02D14FF0000070474FF0DD
S31508020DB0010070474FEA410212F5001215D211D509
S31508020DC06FF47873B3EB625212D94FEAC12343F038
S31508020DD0004343EA505311F0004F23FA02F018BFBA
S31508020DE0404270474FF00000704750EA013005D183
S31508020DF011F0004008BF6FF0004070474FF0000046
S31508020E00704700BF4A0011D212F5001211D20DD551
S31508020E106FF47873B3EB62520ED44FEAC12343F0F0
S31508020E20004343EA505323FA02F070474FF000009A
S31508020E30704750EA013002D14FF0FF3070474FF049
S31508020E40000070474FEA4102B2F1E04324BFB3F50E
S31508020E50001CDCF1FE5C0DD901F0004C4FEAC00221
S31508020E604CEA5070B2F1004F40EB830008BF20F005
S31508020E700100704711F0804F21D113F13872BCBFBF
S31508020E8001F00040704741F480114FEA5252C2F114
S31508020E901802C2F1200C10FA0CF320FA02F018BF5D
S31508020EA040F001004FEAC1234FEAD32303FA0CFCB0
S31508020EB040EA0C0023FA02F34FEA4303CCE77FEA3F
S31508020EC0625307D150EA01331EBF4FF0FE4040F489
S31508020ED04000704701F0004040F0FE4040F4000038
S31508020EE0704700BF53B94AB9002908BF00281CBF7A
S31508020EF04FF0FF314FF0FF3000F0B4B9ADF1080CF6
S31508020F006DE904CE00F03CF8DDF804E0DDE90223E1
S31508020F1004B0704738B50022002304460D46FFF791
S31508020F200BFF28B920462946BDE8384000F00AB822
S31508020F30204605F1004100F005F8404261EB410107
S31508020F4038BD00BFD0B500220B4B06460F46FFF749
S31508020F5081FCFFF757FF0446FFF702FC0022074B06
S31508020F60FFF778FC02460B4630463946FFF7BAFACF
S31508020F70FFF748FF2146D0BD0000F03D0000F041D2
S31508020F802DE9F04F099D0C46002B4DD18A420F469A
S31508020F9084469646B2FA82F360D94BB102FA03FE48
S31508020FA0C3F120029F4000FA03FC20FA02F217431B
S31508020FB04FEA1E461FFA8EF44FEA1C42B7FBF6F1B9
S31508020FC006FB117701FB04F042EA0742904208D970
S31508020FD01EEB020201F1FF3702D2904200F22D8186
S31508020FE03946121A1FFA8CFCB2FBF6F006FB1022DF
S31508020FF000FB04F44CEA024C644508D91EEB0C0CBF
S3150802100000F1FF3202D2644500F21A81104640EA24
S315080210100140ACEB040C002125B12CFA03F30022A3
S31508021020C5E90032BDE8F08F8B4205D90DB1C5E995
S31508021030000100210846F5E7B3FA83F100294DD1EC
S31508021040A342C0F0F280904280F0EF800646234623
S315080210500846002DE6D0C5E90063E3E7002B40F019
S31508021060A2808A1A4FEA1E471FFA8EF60121B2FBA0
S31508021070F7F407FB14204FEA1C4242EA004206FB39
S3150802108004F090420FD91EEB020204F1FF382CBF7E
S315080210904FF001094FF00009904203D9B9F1000F48
S315080210A000F0C8804446121A1FFA8CFCB2FBF7F00D
S315080210B007FB102200FB06F64CEA024C664508D9E5
S315080210C01EEB0C0C00F1FF3202D2664500F2BB8021
S315080210D01046ACEB060C40EA04409DE7C1F1200637
S315080210E08B4004FA01FE22FA06F720FA06FCF440BF
S315080210F08A401F434EEA0C0300FA01FE4FEA1748DC
S315080211004FEA13491FFA87FCB4FBF8F008FB1044B0
S3150802111049EA044400FB0CF9A1450ED93C1900F131
S31508021120FF3A2CBF4FF0010B4FF0000BA14503D934
S31508021130BBF1000F00F093805046A4EB09041FFA96
S3150802114083F9B4FBF8F308FB134403FB0CFC49EAE6
S315080211500444A44506D93C1903F1FF3801D2A44533
S315080211607AD8434643EA0040A4EB0C04A0FB029853
S315080211704445CC46434602D306D1CE4504D201386D
S31508021180B9EB020C68EB07035DB1BEEB0C0264EB2C
S31508021190030404FA06F622FA01F3CC401E43C5E913
S315080211A0006400213EE702FA03FEC3F1200104FAB5
S315080211B003F200FA03FCCC404FEA1E4720FA01F17B
S315080211C01FFA8EF6B4FBF7F00A4307FB1044110C1C
S315080211D041EA044100FB06F48C420ED91EEB0101DA
S315080211E000F1FF382CBF4FF001094FF000098C427D
S315080211F002D9B9F1000F2CD04046091B92B2B1FBB5
S31508021200F7F407FB141142EA014204FB06F1914284
S3150802121007D91EEB020204F1FF3801D2914215D812
S315080212204446521A44EA004121E7861A64EB03034C
S3150802123001200EE7023C724435E702397244D0E6D1
S31508021240F4440238E3E6F444023842E7023C7244C4
S31508021250E7E702387144D0E7023B3C4482E70238AA
S315080212603C446AE7704700BF80B586B002AF786033
S315080212700023FB60342300934FF230230B4A0C49B8
S315080212800C4844F0AFF80346002B0AD1094BBB6061
S31508021290B86807F04BFFF860FB68002B01D000BF67
S315080212A0FDE700BF1037BD4680BD00BF5C0B0020BE
S315080212B0C02109088CFD002080B500AF074B1B78BA
S315080212C0002B07D0054B01221A7020220021044860
S315080212D06DF0A0FC024B184680BD00BFE0FD002061
S315080212E0C0FD002080B483B000AF786039607B68A7
S315080212F03A681A6000BF0C37BD465DF8047B704732
S3150802130080B582B000AF78607B6818687B68043362
S315080213100522194634F0C6FB00BF0837BD4680BD14
S3150802132080B483B000AF78600B46FB70FB787A68AE
S315080213309B0013445B6818460C37BD465DF8047B70
S315080213407047000080B500AF074B1B78DBB2002B55
S3150802135007D1054B01221A701022002103486DF0AD
S3150802136059FC024B184680BDAEFF0020B0FF002094
S3150802137080B485B000AF78607B681B68FB60FB6849
S315080213800133FB607B68FA681A6000BF1437BD46F2
S315080213905DF8047B704780B485B000AF78607B68DF
S315080213A01B68FB60FB68013BFB607B68FA681A6096
S315080213B000BF1437BD465DF8047B704780B483B01E
S315080213C000AF786039607B683A681A6000BF0C37EC
S315080213D0BD465DF8047B704780B483B000AF786081
S315080213E07B689B6818460C37BD465DF8047B7047D8
S315080213F080B485B000AF78607B689B68FB60FB6849
S315080214000133FB607B68FA689A6000BF1437BD46F1
S315080214105DF8047B704780B485B000AF78607B685E
S315080214209B68FB60FB68013BFB607B68FA689A6015
S3150802143000BF1437BD465DF8047B704780B483B09D
S3150802144000AF786039607B683A689A6000BF0C37EB
S31508021450BD465DF8047B704780B483B000AF786000
S315080214607B681B7918460C37BD465DF8047B7047C6
S3150802147080B483B000AF78600B46FB707B68FA785D
S315080214801A7100BF0C37BD465DF8047B704780B4FD
S3150802149083B000AF78607B685B7918460C37BD4627
S315080214A05DF8047B704780B582B000AF78600B4662
S315080214B0FB7025F069FA0346184626F084FE0346B1
S315080214C0002B03D17B68FA785A7102E07B68FA78B6
S315080214D05A7100BF0837BD4680BD80B483B000AFDD
S315080214E078607B689B7918460C37BD465DF8047BA5
S315080214F0704780B483B000AF78600B46FB707B6898
S31508021500FA789A7100BF0C37BD465DF8047B7047BE
S3150802151080B483B000AF78607B681B7B18460C37B3
S31508021520BD465DF8047B704780B483B000AF78602F
S315080215300B46FB707B68FA781A7300BF0C37BD46F8
S315080215405DF8047B704780B500AF19F011FF19F0FA
S315080215503BFF19F0ADFE19F0DFFE00BF80BD0000AB
S3150802156090B583B000AF0346FB71FB79094918466B
S315080215705DF09FF807485BF050FD044605485BF0AE
S3150802158068FD0346194620461BF014F800BF0C37BF
S31508021590BD4690BDE4FD002080B588B000AF034685
S315080215A0FB710023BB600023FB610023BB610023A0
S315080215B07B6100233B610023FB6025F0E5F90346C6
S315080215C0184626F000FE0346002B03D143F63013D5
S315080215D0FB6002E047F25033FB60FFF7B3FE0346B7
S315080215E01846FFF739FF0346002B00F01D81FFF767
S315080215F0AAFFFFF7A7FE03461846FFF72DFF034685
S31508021600013B042B1CD801A252F823F0211602082A
S31508021610271602082D16020833160208391602087A
S315080216200123FB6119E00223FB6116E00423FB6137
S3150802163013E00823FB6110E04FF4B473FB610CE07E
S31508021640FFF780FE034600211846FFF711FFFFF752
S315080216507AFF0320FFF784FFE6E0FFF773FE0346EF
S315080216601846FFF73AFF03461946FA68FB6992FBE2
S31508021670F3F301FB03F3BB60FFF764FE03460021A5
S315080216801846FFF7DBFEFFF75DFE03461846FFF72F
S31508021690FEFE0346012B29D1FFF754FE03461846E0
S315080216A0FFF736FF0346012B02D119F0EBFD01E0E5
S315080216B019F048FEFFF746FE03461846FFF78CFE6A
S315080216C00246BB685B429A424FDCFFF73BFE034683
S315080216D000211846FFF7CCFEFFF735FF5449554857
S315080216E033F04CFB0120FFF73BFF9DE0FFF72AFE94
S315080216F003461846FFF7CBFE0346022B28D1FFF70F
S3150802170021FE03461846FFF703FF0346012B02D1C3
S3150802171019F0ECFD01E019F041FEFFF713FE03464E
S315080217201846FFF759FE0246BB6893421DDCFFF7CF
S3150802173009FE034600211846FFF79AFEFFF703FF44
S315080217403B493C4833F01AFB0120FFF709FF6BE0DF
S31508021750FFF7F8FD034600211846FFF789FEFFF753
S31508021760F2FE0320FFF7FCFE5EE0FFF7EBFD034601
S315080217701846FFF731FE02463B69934208D0FFF747
S31508021780E1FD03461846FFF727FE386100237B6111
S315080217907B6901337B61BB690133BB617B6940F6B7
S315080217A0B732934217D9FFF7CDFD034600211846F3
S315080217B0FFF75EFEFFF7C7FE1F49204826F03AF8F4
S315080217C068F06EF9012301221B2124F095FC0320FF
S315080217D0FFF7C6FE28E0BB694EF65F2293421BD985
S315080217E0FFF7B0FD034600211846FFF741FEFFF753
S315080217F0AAFE1149124826F01DF868F051F901238C
S3150802180002221B2124F078FC09490E4833F0B6FA65
S315080218100320FFF7A5FE07E0FB79184633F08EFC96
S31508021820012042F0D5FF2EE72037BD4680BD00BF16
S31508021830D4210908E0210908E8210908F82109083C
S315080218400C2209082022090880B582B000AF786008
S31508021850786832F001FE0346002B03D11C4833F0A8
S315080218608DFA02E01B4833F089FA786832F0D4FE22
S315080218700346002B03D1184833F080FA02E01748D2
S3150802188033F07CFA786832F085FD0346002B03D1E3
S31508021890134833F073FA02E0124833F06FFA7868A5
S315080218A02DF09AFE78682AF047FE78682BF070F9D0
S315080218B0786833F099F8786830F06AF878682FF023
S315080218C013FB78682EF00EFC00BF0837BD4680BDB4
S315080218D030220908442209085422090868220908FC
S315080218E0782209089022090880B586B000AF034617
S315080218F0FB710023FB7525F047F80346184625F0C9
S3150802190076FA386125F040F80346184625F061FA5A
S31508021910F860FB685B6A224A934201D10123FB7590
S315080219200822002138696DF075F938220021F86815
S315080219306DF070F93B691B4A1A60FB68194A1A600E
S31508021940FB6840F209125A60FB6840F20912DA6033
S31508021950FB68072283F82C20FB68072283F82D20D0
S31508021960FB68022283F82E20FB68072283F82F20C1
S31508021970FB7D012B03D1FB68094A5A6202E0FB6828
S3150802198000225A62FB68012283F82820FB791A464C
S31508021990F968386900F01AF900BF1837BD4680BDE4
S315080219A01A8057F03330424D80B58AB000AFF860DE
S315080219B0B9607A60FB70002387F8273000233B6101
S315080219C0BB68BB617B687B61BB693B627B69FB6108
S315080219D04FF0FF333B61002387F8273015E097F86D
S315080219E0273003F1016303F57C2318466BF070FE7A
S315080219F003463B613A693B6A1A603B6A04333B62B7
S31508021A0097F82730043387F8273097F82720FB788A
S31508021A109A42E4D34FF0FF333B61002387F827301D
S31508021A2015E097F8273003F1016303F57D2318467D
S31508021A306BF04EFE03463B613A69FB691A60FB6925
S31508021A400433FB6197F82730043387F8273097F871
S31508021A50272097F830309A42E3D3012318462837CD
S31508021A60BD4680BD80B596B002AFF860B960134630
S31508021A70FB7138220021B8686DF0CCF807F118031B
S31508021A803822002118466DF0C5F808220021F868A8
S31508021A906DF0C0F807F110030822002118466DF010
S31508021AA0B9F8FB79002B1AD04FF47A713F4843F004
S31508021AB0CFFD0346002B0DD107F1180207F11001DD
S31508021AC03823009308233A48FFF76EFF374843F056
S31508021AD001FE0EE02421374833F00AF909E007F13E
S31508021AE0180207F110013823009308233048FFF73C
S31508021AF05BFFBB69304A934208D0FB791846FFF769
S31508021B00F3FE15212D4833F0F3F832E007F11803F6
S31508021B1038221946B8686DF034F9B86800F05FFAE9
S31508021B200346002B21D1B86800F076FA0346002B4B
S31508021B301BD1B86800F08DFA0346002B15D1B86898
S31508021B4000F0A4FA0346002B0FD10721B86800F06B
S31508021B5053FA0721B86800F06CFA0221B86800F057
S31508021B6085FA0721B86800F09EFA1421144833F062
S31508021B70BFF83B69104A934208D0FB791846FFF72B
S31508021B80B3FE14210F4833F0B3F80AE007F1100345
S31508021B9008221946F8686DF0F4F813210A4833F05A
S31508021BA0A7F8012318465037BD4680BD301C0120D0
S31508021BB000C01F08A82209083330424DD02209085E
S31508021BC0E8220908002309081823090890B59DB0D8
S31508021BD000AFF860B9601346FB71012387F86F30CE
S31508021BE00023BB66FB687B66BB683B6697F86F306B
S31508021BF0002B39D0FB79002B1AD04FF47A71AA48F8
S31508021C0043F026FD0346002B0DD1FE206BF08FFD17
S31508021C100346002B14BF0123002387F86F30A2481E
S31508021C2043F058FD0EE02421A04833F061F809E09C
S31508021C30FE206BF07CFD0346002B14BF0123002314
S31508021C4087F86F3097F86F3083F00103DBB2002B09
S31508021C500AD0FB79002B03D0954825F0EBFD03E06B
S31508021C602521944833F044F897F86F30002B05D0B5
S31508021C70FB79002B02D1642033F058FB97F86F30BA
S31508021C80002B65D007F150031022FF2118466CF08D
S31508021C90C1FF0023BB6658E07B6E07F15004186843
S31508021CA059689A68DB680FC4FB79002B22D04FF477
S31508021CB07A717D4843F0CCFC0346002B15D1BB6EE6
S31508021CC003F1016303F57C2307F150021146184616
S31508021CD06BF012FD0346002B14BF0123002387F87D
S31508021CE06F30714843F0F6FC16E02421724832F050
S31508021CF0FFFF11E0BB6E03F1016303F57C2307F1D5
S31508021D005002114618466BF0F7FC0346002B14BF27
S31508021D100123002387F86F307B6E10337B6697F8B2
S31508021D206F3083F00103DBB2002B0BD0FB79002B5B
S31508021D3003D0624825F07EFD0AE02921604832F088
S31508021D40D7FF05E0BB6E1033BB66BB6E072BA3D964
S31508021D5097F86F30002B65D007F150031022FF2148
S31508021D6018466CF057FF0023BB6658E03B6E07F136
S31508021D705004186859689A68DB680FC4FB79002B07
S31508021D8022D04FF47A71484843F062FC0346002B8E
S31508021D9015D1BB6E03F1016303F57D2307F15002EA
S31508021DA0114618466BF0A8FC0346002B14BF012304
S31508021DB0002387F86F303C4843F08CFC16E0242158
S31508021DC03D4832F095FF11E0BB6E03F1016303F55E
S31508021DD07D2307F15002114618466BF08DFC034627
S31508021DE0002B14BF0123002387F86F303B6E103394
S31508021DF03B6697F86F3083F00103DBB2002B0BD0FA
S31508021E00FB79002B03D02D4825F014FD0AE0292181
S31508021E102B4832F06DFF05E0BB6E1033BB66BB6E16
S31508021E20372BA3D997F86F30002B37D0FA7907F1F9
S31508021E30100107F148031846FFF714FE07F1480395
S31508021E400822F96818466CF0D5FE0346002B0DD019
S31508021E50FB79002B03D01B4825F0ECFC03E02A2172
S31508021E60194832F045FF002387F86F3007F110034F
S31508021E703822B96818466CF0BDFE0346002B0DD011
S31508021E80FB79002B03D0114825F0D4FC03E02B2163
S31508021E900F4832F02DFF002387F86F3097F86F301E
S31508021EA018467437BD4690BD301C01202C230908FC
S31508021EB05423090878230908A0230908C82309080E
S31508021EC0F02309081C240908482409087424090867
S31508021ED0A024090880B483B000AF78607B681B79B8
S31508021EE018460C37BD465DF8047B704780B483B04C
S31508021EF000AF78600B46FB707B68FA781A7100BFF0
S31508021F000C37BD465DF8047B7047000080B483B089
S31508021F1000AF78607B685B6A054A934201D1012368
S31508021F2000E0002318460C37BD465DF8047B70476F
S31508021F301A8057F080B483B000AF78607B68044A91
S31508021F405A62012318460C37BD465DF8047B704772
S31508021F501A8057F080B483B000AF78607B6800229D
S31508021F605A62012318460C37BD465DF8047B704752
S31508021F7080B483B000AF78607B6893F8293018463E
S31508021F800C37BD465DF8047B704780B483B000AF5A
S31508021F9078607B6893F82A3018460C37BD465DF898
S31508021FA0047B704780B483B000AF78607B6893F88F
S31508021FB02B3018460C37BD465DF8047B704780B453
S31508021FC083B000AF78600B46FB707B68FA7883F8BB
S31508021FD02B2000BF0C37BD465DF8047B704780B4E2
S31508021FE083B000AF78607B6893F82C3018460C37BC
S31508021FF0BD465DF8047B704780B483B000AF786055
S315080220000B46FB707B68FA7883F82C2000BF0C37E6
S31508022010BD465DF8047B704780B483B000AF786034
S315080220207B6893F82D3018460C37BD465DF8047B5D
S31508022030704780B483B000AF78600B46FB707B684C
S31508022040FA7883F82D2000BF0C37BD465DF8047B6D
S31508022050704780B483B000AF78607B6893F82E30FF
S3150802206018460C37BD465DF8047B704780B483B0CA
S3150802207000AF78600B46FB707B68FA7883F82E20EF
S3150802208000BF0C37BD465DF8047B704780B483B049
S3150802209000AF78607B6893F82F3018460C37BD4638
S315080220A05DF8047B704780B483B000AF78600B4656
S315080220B0FB707B68FA7883F82F2000BF0C37BD4681
S315080220C05DF8047B704780B483B000AF78603960EE
S315080220D07B683A681A63012318460C37BD465DF8D1
S315080220E0047B704780B483B000AF78607B681B6B53
S315080220F018460C37BD465DF8047B704780B500AFBD
S3150802210002486BF0E5FA0346184680BD30D01F0830
S3150802211080B582B000AF78607B6893F83430012BC3
S3150802212005D91E21054832F0E3FD002302E07B684B
S3150802213093F8343018460837BD4680BDCC240908C2
S3150802214080B483B000AF78600B46FB707B68FA7880
S3150802215083F8342000BF0C37BD465DF8047B704710
S3150802216080B582B000AF78607B6893F83530022B71
S3150802217005D91D21054832F0BBFD002302E07B6824
S3150802218093F8353018460837BD4680BDEC24090851
S3150802219080B483B000AF78600B46FB707B68FA7830
S315080221A083F8352000BF0C37BD465DF8047B7047BF
S315080221B080B483B000AF0346FB71044AFB791370FF
S315080221C000BF0C37BD465DF8047B704745140120F5
S315080221D080B400AF034B1B781846BD465DF8047BF6
S315080221E0704700BF4514012080B586B000AFF8607D
S315080221F00B467A60FB720023FB752C4832F0BEFD53
S315080222000023FB754AE0FA7D294913461B019B1AEE
S31508022210DB000B441B78012B3DD1FA7D13461B01CB
S315080222209B1ADB00224A134402331946214832F02C
S31508022230A5FD214832F0A2FDFA7D13461B019B1A21
S31508022240DB0018331A4A134419461A4832F096FD27
S315080222501A4832F093FDFA7D154913461B019B1A5B
S31508022260DB000B4448331B782D2B11D0144832F06F
S3150802227085FDFA7D13461B019B1ADB0048330C4A7F
S31508022280134419460B4832F079FD0C4832F076FDB4
S315080222900A4832F073FDFB7D0133FB75FB7D102B7B
S315080222A0B1D900BF00BF1837BD4680BD0C25090845
S315080222B00400002034250908382509083C250908A0
S315080222C04025090880B500AF024832F057FD00BF25
S315080222D080BD00BF4C25090880B584B000AFF86000
S315080222E00B467A60FB7224F04FFB0346184624F02D
S315080222F011FD00BF1037BD4680BD00002DE9F0472D
S3150802230090B006AFF8600B467A60FB72002387F836
S315080223102730002387F8263024F036FB3862C9486E
S3150802232032F02CFD386A25F003FA0346184655F0B2
S31508022330A0FB03461C46386A25F0FAF903461846F6
S3150802234055F0B2FB03461A462146BF4832F016FD3F
S31508022350002387F82630002387F8273035E022F055
S3150802236009FA024697F827301946104623F0A9FEBD
S315080223700346002B2ED022F0FDF9024697F82730A5
S315080223801946104623F09DFE0346184622F0CEFC57
S3150802239003461C4622F0EEF9024697F827301946FC
S315080223A0104623F08EFE0346184623F019F8034614
S315080223B01A462146A54832F0E1FC012387F8263061
S315080223C097F82730013387F8273097F82730172BE5
S315080223D0C5D900E000BF97F82630002B02D19C48E9
S315080223E032F0CCFC9B4832F0C9FC0121386A25F050
S315080223F0B6FD034698460221386A25F0B0FD034623
S3150802240099460421386A25F0AAFD03469A46082108
S31508022410386A25F0A4FD03461C460121386A25F0D0
S31508022420CCFD03461D460221386A25F0C6FD034641
S315080224301E460421386A25F0C0FD03463B60082182
S31508022440386A25F0BAFD034604933B68039302965D
S315080224500195009453464A4641467F4832F08EFC1F
S315080224607C4832F08BFC4DF01FFF034618464DF0B0
S31508022470A2FFF861794832F081FC0121F8695FF020
S315080224803BFB03461D460221F8695FF035FB03460E
S315080224901E460421F8695FF02FFB03469846082179
S315080224A0F8695FF029FB03461C461021F8695FF0BC
S315080224B023FB03460193009443463246294668485D
S315080224C032F05CFCF8695FF033FB0346194665484F
S315080224D032F054FCF8695FF046FB03461C46F8697D
S315080224E05FF05CFB03461D46F8695FF072FB034624
S315080224F01E46F8695FF088FB0346009333462A4670
S315080225002146594832F03AFCC82042F061F951484E
S3150802251032F034FC4DF0C8FE034618464DF057FF1C
S31508022520B861B8695DF0DBFD03461C46B8695DF023
S31508022530E2FD03461D46B8695DF0E9FD03462A46F3
S3150802254021464A4832F01AFC386A25F04FFA10EE4C
S31508022550103A1846FEF726F902460B46444832F068
S315080225600DFC386A25F068FA10EE103A1846FEF79E
S3150802257019F902460B463F4832F000FC386A25F044
S3150802258081FA10EE103A1846FEF70CF902460B4687
S31508022590394832F0F3FB386A25F09AFA10EE103A07
S315080225A01846FEF7FFF802460B46344832F0E6FBB9
S315080225B0C82042F00DF9274832F0E0FB4DF074FED0
S315080225C0034618464DF00FFF7861786962F0A0FB62
S315080225D003461C46786962F0B6FB03461A4621464C
S315080225E0274832F0CBFB0121786962F0D8FB034613
S315080225F01C460221786962F0D2FB03461A46214636
S31508022600204832F0BBFB0421786962F0C8FB034616
S315080226101C460821786962F0C2FB03461A4621461F
S31508022620194832F0ABFB1021786962F0B8FB034611
S315080226301946164832F0A2FB00BF2837BD46BDE848
S31508022640F08700BF6025090878250908902509083A
S315080226509C2509083C250908A4250908CC2509084A
S31508022660EC250908182609082C2609084826090807
S315080226706C2609088026090894260908A826090846
S31508022680BC260908D0260908E826090804270908E5
S31508022690B0B59CB000AFF8600B467A60FB720023B7
S315080226A087F86F307B6803F5C06318466BF071F9DB
S315080226B0034687F86F30FB7A032B09D97B6803F543
S315080226C0C06318466BF065F9034687F86F300BE06E
S315080226D0FB7A032B08D17B6803F5806318466BF0F7
S315080226E058F9034687F86F307B6803F500730422AE
S315080226F0CA4918466CF096FA0346002B40F06C81DC
S315080227007B6803F500731846FDF7E0FE0346042BC3
S3150802271040F062817B6803F580630222C04918464D
S315080227206CF080FA0346002B40F009817B6803F5BA
S3150802273080631846FDF7CAFE0346022B40F0FF8067
S31508022740B84B1B6850221A6497F86F301946B64878
S3150802275032F014FB97F86F30032B2CD101224FF479
S315080227608061B24837F0C0F800224FF40041B04801
S3150802277037F0BAF801224FF48071AC4837F0B4F852
S3150802278001228021A94837F0AFF801224021A74843
S3150802279037F0AAF801224FF48071A64837F0A4F858
S315080227A001228021A34837F09FF801224021A1483F
S315080227B037F09AF80EE197F86F30042B2CD10122E4
S315080227C04FF48071994837F08FF800228021974894
S315080227D037F08AF801224FF48061944837F084F87A
S315080227E001224FF40041924837F07EF80122402137
S315080227F08E4837F079F801224FF480718D4837F008
S3150802280073F8012280218B4837F06EF801224021A5
S31508022810884837F069F8DDE097F86F30052B2CD138
S3150802282001224021814837F05FF800224FF4807177
S31508022830804837F059F801224FF480617B4837F017
S3150802284053F801224FF40041794837F04DF8012236
S315080228504FF48071754837F047F801228021734892
S3150802286037F042F801228021724837F03DF80122FA
S315080228704021704837F038F8ACE097F86F30062BED
S315080228802CD1012280216B4837F02EF800224021F4
S31508022890684837F029F801224FF48061634837F017
S315080228A023F801224FF40041614837F01DF801224E
S315080228B040215E4837F018F801224FF480715D48CE
S315080228C037F012F801224FF48071584837F00CF8A5
S315080228D001228021554837F007F87BE0514B1B68E7
S315080228E000221A6401224FF40041514836F0FCFFD7
S315080228F001224FF480614D4836F0F6FF012280210D
S315080229004A4836F0F1FF01224FF48071474836F003
S31508022910EBFF01224FF48071464836F0E5FF0122AB
S315080229204021424836F0E0FF01224021414836F074
S31508022930DBFF012280213F4836F0D6FF4AE07B685A
S3150802294003F5806303223C4918466CF06BF903468B
S31508022950002B40F0E9857B6803F580631846FDF78E
S31508022960B5FD0346032B40F0DF852E4B1B6800227C
S315080229701A6400224FF400412D4836F0B5FF0022B2
S315080229804FF48061294836F0AFFF0022802127489C
S3150802299036F0AAFF00224FF48071244836F0A4FFCD
S315080229A000224FF48071234836F09EFF0022402110
S315080229B01E4836F099FF002240211E4836F094FF41
S315080229C0002280211B4836F08FFF1C4832F0D6F9C8
S315080229D000F0AABD00F0A8BD7B6803F500730822C3
S315080229E0174918466CF01EF90346002B38D17B6846
S315080229F003F500731846FDF769FD0346082B2FD128
S31508022A0097F86F30022B1DD123F0BEFF0346022131
S31508022A10184626F08EF900F089BD00BF142709086A
S31508022A201C2709086C6D01202027090800080242A4
S31508022A300000024200180242382709083C27090802
S31508022A405427090897F86F30032B40F06F8523F057
S31508022A509BFF03460321184626F06BF900F066BD74
S31508022A607B6803F500730722CC4918466CF0DAF83E
S31508022A700346002B33D17B6803F500731846FDF72E
S31508022A8025FD0346072B2AD17B6803F58063184682
S31508022A906AF07FFF034687F86F3023F075FF034617
S31508022AA042F20F71184626F0B3F823F06DFF02467C
S31508022AB097F86F301946104626F0BDF897F86F302A
S31508022AC01946B74832F05AF9032387F8283007F12E
S31508022AD028030121184616F00DFE00F02BBD7B686F
S31508022AE003F500730522AF4918466CF09BF80346B6
S31508022AF0002B11D17B6803F500731846FDF7E6FC37
S31508022B000346052B08D123F03FFF03460921184641
S31508022B1024F0A8F800F00EBD7B6803F500730822BE
S31508022B20A14918466CF07EF80346002B11D17B6842
S31508022B3003F500731846FDF7C9FC0346082B08D1AE
S31508022B4023F022FF03460121184624F08BF800F0F1
S31508022B50F1BC7B6803F500730922944918466CF0A8
S31508022B6061F80346002B11D17B6803F500731846FA
S31508022B70FDF7ACFC0346092B08D123F005FF0346F3
S31508022B800221184624F06EF800F0D4BC7B6803F5DF
S31508022B9000730722864918466CF044F80346002B50
S31508022BA040F082807B6803F500731846FDF78EFCB9
S31508022BB00346072B78D17B6803F5C06318466AF08B
S31508022BC0E8FE034687F86F307B6803F580630322C5
S31508022BD0784918466CF026F80346002B1CD17B6808
S31508022BE003F580631846FDF771FC0346032B13D1E0
S31508022BF097F86F30012B05D16F4832F0BFF818F0FD
S31508022C0041FB31E097F86F30022B2DD16B4832F039
S31508022C10B5F818F097FB27E07B6803F58063032273
S31508022C20674918466BF0FEFF0346002B1DD17B68E9
S31508022C3003F580631846FDF749FC0346032B14D1B6
S31508022C4097F86F30012B05D15E4832F097F818F0E5
S31508022C504DFB0AE097F86F30022B06D15A4832F03C
S31508022C608DF818F09BFB00E000BF7B6803F58063D4
S31508022C700322564918466BF0D5FF0346002B40F04F
S31508022C8057847B6803F580631846FDF71FFC0346E5
S31508022C90032B40F04D844E4832F070F818F008FBCA
S31508022CA018F066FB00F044BC7B6803F50073062245
S31508022CB0484918466BF0B6FF0346002B11D17B68CC
S31508022CC003F500731846FDF701FC0346062B08D1E7
S31508022CD023F05AFE03460421184623F0C3FF00F0E8
S31508022CE029BC7B6803F5007305223B4918466BF03D
S31508022CF099FF0346002B40F091807B6803F5007329
S31508022D001846FDF7E3FB0346052B40F0878097F844
S31508022D106F301946314832F031F897F86F30013B77
S31508022D200C2B79D801A252F823F000BF612D0208B4
S31508022D306D2D0208792D0208852D0208912D0208AB
S31508022D40E52D0208192E0208192E0208F12D02088D
S31508022D50FF2D0208192E0208192E02080D2E020846
S31508022D60002208211E4836F0BFFD56E00022042143
S31508022D701B4836F0B9FD50E000220221184836F009
S31508022D80B3FD4AE000220121154836F0ADFD44E0C4
S31508022D9000228021124836F0A7FD3EE06027090886
S31508022DA0682709088027090888270908942709082F
S31508022DB0A0270908A8270908AC270908C02709086F
S31508022DC0D4270908D8270908EC2709083827090843
S31508022DD000280908142809081C28090824280908AB
S31508022DE0000C024200224021744836F07DFD14E0B0
S31508022DF000224FF48051724836F076FD0DE000222B
S31508022E004FF400616E4836F06FFD06E0002220217D
S31508022E106C4836F069FD00E000BF8BE37B6803F57A
S31508022E2000730222684918466BF0FCFE0346002B23
S31508022E3039D17B6803F500731846FDF747FB03464D
S31508022E40022B30D197F86F301946604831F096FF59
S31508022E5097F86F30013B032B00F26C8301A252F8FC
S31508022E6023F000BF752E0208812E02088D2E020855
S31508022E70992E020800222021524836F035FD11E02B
S31508022E80002220214F4836F02FFD0BE00022202198
S31508022E904C4836F029FD05E000222021494836F043
S31508022EA023FD00BF46E37B6803F500730222484907
S31508022EB018466BF0B7FE0346002B40F093807B68FA
S31508022EC003F500731846FDF701FB0346022B40F093
S31508022ED0898097F86F3019463E4831F04FFF97F8C8
S31508022EE06F30013B0B2B00F2258301A252F823F027
S31508022EF0212F02082F2F02083D2F02084B2F020806
S31508022F00592F0208652F0208712F02087D2F020821
S31508022F10892F0208952F0208A12F0208AD2F020851
S31508022F2001224FF480412C4836F0DEFC44E00122AF
S31508022F304FF40051284836F0D7FC3DE001224FF401
S31508022F408051254836F0D0FC36E001224FF4006164
S31508022F50214836F0C9FC2FE001220421194836F02F
S31508022F60C3FC29E001220221164836F0BDFC23E003
S31508022F7001220121134836F0B7FC1DE00122202167
S31508022F80164836F0B1FC17E001221021134836F034
S31508022F90ABFC11E001228021114836F0A5FC0BE0BA
S31508022FA0012240210E4836F09FFC05E0012220212D
S31508022FB00B4836F099FC00BFBCE200BF000C024287
S31508022FC0001802420004024234280908382809086F
S31508022FD0482809084C280908001402420008024237
S31508022FE0000002427B6803F500730922C9491846A4
S31508022FF06BF018FE0346002B40F0BB807B6803F596
S3150802300000731846FDF762FA0346092B40F0B180B1
S31508023010C14831F0B3FE01220821C04836F064FCEB
S3150802302001220421BD4836F05FFC01220221BB4879
S3150802303036F05AFC01220121B84836F055FC012225
S315080230408021B64836F050FC01224021B34836F0BA
S315080230504BFC01222021B14836F046FC0122102100
S31508023060AE4836F041FC01224FF48051AC4836F0A6
S315080230703BFC01224FF40061A94836F035FC0122D7
S315080230804FF48061A64836F02FFC01224FF40071F6
S31508023090A34836F029FC01222021A24836F024FC56
S315080230A001224FF400419E4836F01EFC01224FF4DD
S315080230B080419B4836F018FC01224FF4005198488B
S315080230C036F012FC01224FF40071964836F00CFCD9
S315080230D001224FF48071934836F006FC01228021C2
S315080230E0904836F001FC012240218E4836F0FCFB5E
S315080230F000224FF480418C4836F0F6FB00224FF44A
S315080231000051894836F0F0FB00224FF48051864878
S3150802311036F0EAFB00224FF40061834836F0E4FBFE
S31508023120002204217F4836F0DFFB002202217D4877
S3150802313036F0DAFB002201217A4836F0D5FB002266
S3150802314020217A4836F0D0FB00221021774836F043
S31508023150CBFB00228021764836F0C6FB00224021AE
S31508023160734836F0C1FB00222021714836F0BCFBB9
S31508023170E0E17B6803F5007309226E4918466BF095
S3150802318051FD0346002B0BD17B6803F500731846E5
S31508023190FDF79CF90346092B02D117F0B5F9C9E1E7
S315080231A07B6803F500730A22634918466BF03AFDF9
S315080231B00346002B0BD17B6803F500731846FDF70F
S315080231C085F903460A2B02D117F05AF9B2E17B6850
S315080231D003F500730B22594918466BF023FD034683
S315080231E0002B0BD17B6803F500731846FDF76EF9C1
S315080231F003460B2B02D117F06BFA9BE17B6803F5AA
S3150802320000730C224E4918466BF00CFD0346002B40
S315080232100BD17B6803F500731846FDF757F9034689
S315080232200C2B02D117F010FA84E17B6803F50073C0
S315080232300922444918466BF0F5FC0346002B4ED189
S315080232407B6803F500731846FDF740F90346092B18
S3150802325045D17B6803F5806318466AF09AFB0346F4
S3150802326087F86F3097F86F301946374831F086FD80
S3150802327097F86F30022B07D123F086FB034602210B
S31508023280184625F056FD55E197F86F30032B07D1FE
S3150802329023F07AFB03460321184625F04AFD49E145
S315080232A016F0A2FA0346184618F0D4F80346012B7C
S315080232B00AD1264831F062FD23F066FB0346032154
S315080232C0184625F036FD35E1214831F057FD23F041
S315080232D05BFB03460221184625F02BFD2AE17B6893
S315080232E003F5007303221B4918466BF09BFC034641
S315080232F0002B31D17B6803F500731846FDF7E6F813
S315080233000346032B28D101220121054836F0ECFA9F
S3150802331010E100BF5C28090868280908000C024267
S315080233200018024200040242001402420008024245
S31508023330000002427C2809088828090894280908F6
S31508023340A0280908B0280908BC280908D8280908A5
S31508023350F8280908182909087B6803F50073032267
S31508023360764918466BF05EFC0346002B0FD17B6844
S3150802337003F500731846FDF7A9F80346032B06D191
S3150802338001224FF400416E4836F0AEFAD2E07B686D
S3150802339003F5007306226B4918466BF043FC034695
S315080233A0002B0FD17B6803F500731846FDF78EF8DC
S315080233B00346062B06D101224FF40041604836F037
S315080233C093FAB7E07B6803F500730A225E4918464A
S315080233D06BF028FC0346002B19D17B6803F50073B2
S315080233E01846FDF773F803460A2B10D1574B1B688C
S315080233F064229A63554B1B6800225A63002153487C
S315080234003CF02EFE042151483CF0CAFC92E07B684F
S3150802341003F500730A224E4918466BF003FC03466D
S31508023420002B19D17B6803F500731846FDF74EF891
S3150802343003460A2B10D1454B1B6800229A63434B5D
S315080234401B6864225A63042140483CF009FE0021A5
S315080234503E483CF0A5FC6DE07B6803F50073082244
S315080234603C4918466BF0DEFB0346002B08D17B6805
S3150802347003F500731846FDF729F80346082B59D0B9
S315080234807B6803F500730722334918466BF0CAFBBB
S315080234900346002B1AD17B6803F500731846FDF71D
S315080234A015F80346072B11D12C4A07F1140307CA4C
S315080234B083E8070007F1200300221A605A6007F121
S315080234C014030B2118464AF021F933E07B6803F509
S315080234D000730E22224918466BF0A4FB0346002B02
S315080234E028D17B6803F500731846FCF7EFFF0346FD
S315080234F00E2B1FD107F12C0318465FF058FA5DF020
S3150802350057FE044607F12C0318465EF0B6FE05463A
S3150802351007F12C0318465EF0BCFE03461A462946F6
S31508023520204651F039F805E000BF03E000BF01E08C
S3150802353000BFFFE700BF7037BD46B0BD1C290908AA
S31508023540001402422029090828290908D46C0120F6
S3150802355034290908402909084C290908642909084F
S315080235605429090890B589B000AFF8600B467A600D
S31508023570FB720023FB610023BB610023FB7523F06A
S3150802358003FA3861FB7A012B41F2FD867B6803F563
S3150802359000730622B94918466BF044FB0346002B12
S315080235A02DD17B6803F500731846FCF78FFF034697
S315080235B0062B24D1B24831F0E1FB0021386924F008
S315080235C0C2FB0021386924F0E9FB0021386924F09E
S315080235D001FC0021386924F028FC0021386924F00E
S315080235E04FFC0021386924F076FC0021386924F062
S315080235F094FC0121386924F07BFB01F0CCBE7B6880
S3150802360003F5007307229F4918466BF00BFB034626
S31508023610002B10D17B6803F500731846FCF756FF9A
S315080236200346072B07D1984831F0A8FB386923F0DF
S3150802363071FB01F0B0BE7B6803F500730B22934958
S3150802364018466BF0EFFA0346002B3CD17B6803F56C
S3150802365000731846FCF73AFF03460B2B33D17B68F7
S3150802366003F580631A788A4B1B78D31A002B0DD17F
S315080236707B6803F580631846FCF728FF0346012B8F
S3150802368004D10121386924F033FB1AE07B6803F57B
S3150802369080631A787F4B1B78D31A002B0DD17B686F
S315080236A003F580631846FCF711FF0346012B04D184
S315080236B00021386924F01CFB03E0FEF703FE01F043
S315080236C06ABE01F068BE7B6803F50073052272497B
S315080236D018466BF0A7FA0346002B40F09A807B68DF
S315080236E003F500731846FCF7F1FE0346052B40F076
S315080236F090807B6803F5806318466AF04AF9F86198
S31508023700FB69012B1ED17B6803F5C06318466AF074
S3150802371040F9F861FB69012B06D116F077FE5F487E
S3150802372031F02CFB01F032BEFB69002B06D116F0F4
S3150802373079FE5B4831F022FB01F028BEFEF7C2FD96
S3150802374001F029BEFB69022B1ED17B6803F5C06313
S3150802375018466AF01EF9F861FB69012B06D116F0C4
S315080237600DFE504831F00AFB01F010BEFB69002B32
S3150802377006D116F00FFE4C4831F000FB01F006BEEA
S31508023780FEF7A0FD01F007BEFB69032B1ED17B687D
S3150802379003F5C06318466AF0FCF8F861FB69012B69
S315080237A006D116F003FE414831F0E8FA01F0EEBD03
S315080237B0FB69002B06D116F005FE3D4831F0DEFA0C
S315080237C001F0E4BDFEF77EFD01F0E5BDFB69042BC1
S315080237D041F0DC857B6803F5C06318466AF0D9F8C0
S315080237E0F861FB69012B06D116F0F8FD2F4831F076
S315080237F0C5FA01F0CBBDFB69002B06D116F0FAFD1E
S315080238002B4831F0BBFA01F0C1BDFEF75BFD01F0B2
S31508023810C2BD7B6803F500730222264918466BF07F
S3150802382001FA0346002B40F09E827B6803F500737B
S315080238301846FCF74BFE0346022B40F094827B683F
S3150802384003F5806318466AF0A4F8F861FB69012B50
S3150802385047D17B6803F5C06318466AF09AF8F8619F
S31508023860FB69012B2CD101220121134836F03CF8C1
S31508023870124831F083FA01F08EBD00BF7829090893
S31508023880802909089C290908A4290908CC290908B4
S31508023890D8290908DC290908E0290908E8290908B4
S315080238A0FC290908142A0908342A0908542A090885
S315080238B0742A09084828090800180242942A09089D
S315080238C0FB69002B09D100220121B64836F00CF813
S315080238D0B54831F053FA01F05EBDFEF7F3FC01F08C
S315080238E05ABDFB69022B26D17B6803F5C0631846CD
S315080238F06AF04FF8F861FB69012B0AD101224FF4ED
S315080239000041AA4835F0F0FFA94831F037FA01F02C
S3150802391042BDFB69002B0AD100224FF40041A3489D
S3150802392035F0E2FFA34831F029FA01F034BDFEF77B
S31508023930C9FC01F030BDFB69032B26D17B6803F570
S31508023940C06318466AF025F8F861FB69012B0AD1AB
S3150802395001224FF48041954835F0C6FF964831F06A
S315080239600DFA01F018BDFB69002B0AD100224FF4AB
S3150802397080418E4835F0B8FF904831F0FFF901F0E2
S315080239800ABDFEF79FFC01F006BDFB69042B26D192
S315080239907B6803F5C063184669F0FBFFF861FB69AB
S315080239A0012B0AD101224FF40051804835F09CFFC1
S315080239B0834831F0E3F901F0EEBCFB69002B0AD12A
S315080239C000224FF40051794835F08EFF7D4831F0D8
S315080239D0D5F901F0E0BCFEF775FC01F0DCBCFB6929
S315080239E0052B26D17B6803F5C063184669F0D1FF1B
S315080239F0F861FB69012B0AD101224FF480516B4809
S31508023A0035F072FF704831F0B9F901F0C4BCFB69B0
S31508023A10002B0AD100224FF48051644835F064FF26
S31508023A206A4831F0ABF901F0B6BCFEF74BFC01F07F
S31508023A30B2BCFB69062B26D17B6803F5C063184620
S31508023A4069F0A7FFF861FB69012B0AD101224FF43D
S31508023A500061564835F048FF5D4831F08FF901F0AC
S31508023A609ABCFB69002B0AD100224FF400614F4829
S31508023A7035F03AFF574831F081F901F08CBCFEF770
S31508023A8021FC01F088BCFB69072B24D17B6803F56E
S31508023A90C063184669F07DFFF861FB69012B09D1FD
S31508023AA0012204214C4835F01FFF4C4831F066F9D3
S31508023AB001F071BCFB69002B09D10022042146489A
S31508023AC035F012FF464831F059F901F064BCFEF7A9
S31508023AD0F9FB01F060BCFB69082B24D17B6803F56E
S31508023AE0C063184669F055FFF861FB69012B09D1D5
S31508023AF001220221384835F0F7FE3A4831F03EF9FC
S31508023B0001F049BCFB69002B09D100220221324887
S31508023B1035F0EAFE344831F031F901F03CBCFEF7E3
S31508023B20D1FB01F038BCFB69092B24D17B6803F56C
S31508023B30C063184669F02DFFF861FB69012B09D1AC
S31508023B4001220121244835F0CFFE284831F016F922
S31508023B5001F021BCFB69002B09D1002201211E4874
S31508023B6035F0C2FE224831F009F901F014BCFEF71D
S31508023B70A9FB01F010BCFB690A2B50D17B6803F53F
S31508023B80C063184669F005FFF861FB69012B35D158
S31508023B9001222021174835F0A7FE174831F0EEF822
S31508023BA001F0F9BB00180242A82A090800140242C9
S31508023BB0BC2A0908D02A0908E42A0908F82A0908A1
S31508023BC00C2B0908202B0908342B0908482B09084D
S31508023BD05C2B09086C2B0908000402427C2B090895
S31508023BE0A42B0908CC2B0908F02B0908182C09085C
S31508023BF0402C090800080242682C0908FB69002BB8
S31508023C0009D100222021C24835F06EFEC14831F0A2
S31508023C10B5F801F0C0BBFEF755FB01F0BCBBFB696A
S31508023C200B2B24D17B6803F5C063184669F0B1FEF5
S31508023C30F861FB69012B09D101221021B44835F03C
S31508023C4053FEB54831F09AF801F0A5BBFB69002B83
S31508023C5009D100221021AE4835F046FEAF4831F0B0
S31508023C608DF801F098BBFEF72DFB01F094BBFB69BA
S31508023C700C2B24D17B6803F5C063184669F089FECC
S31508023C80F861FB69012B09D101228021A44835F08C
S31508023C902BFEA44831F072F801F07DBBFB69002BBC
S31508023CA009D1002280219E4835F01EFE9E4831F039
S31508023CB065F801F070BBFEF705FB01F06CBBFB690A
S31508023CC00D2B24D17B6803F5C063184669F061FEA3
S31508023CD0F861FB69012B09D101222021904835F0B0
S31508023CE003FE924831F04AF801F055BBFB69002BF6
S31508023CF009D1002220218A4835F0F6FD8C4831F098
S31508023D003DF801F048BBFEF7DDFA01F044BBFB695A
S31508023D100E2B24D17B6803F5C063184669F039FE79
S31508023D20F861FB69012B09D1012240217C4835F053
S31508023D30DBFD804831F022F801F02DBBFB69002B30
S31508023D4009D100224021764835F0CEFD7A4831F075
S31508023D5015F801F020BBFEF7B5FA01F01CBBFEF719
S31508023D60B1FA01F018BB7B6803F5007308227349A0
S31508023D7018466AF057FF0346002B40F067837B68B4
S31508023D8003F500731846FCF7A1FB0346082B40F01F
S31508023D905D837B6803F580630422694918466AF0E5
S31508023DA041FF0346002B40F020837B6803F58063BE
S31508023DB01846FCF78BFB0346042B40F016837B68F8
S31508023DC003F5C06305225F4918466AF02BFF0346CE
S31508023DD0002B28D17B6803F5C0631846FCF776FBEF
S31508023DE00346052B1FD1584830F0C8FF10F082FA57
S31508023DF00446FEF7EDF903461A460121204610F05D
S31508023E00AFFB0346002B0AD010F074FA0446FEF7FD
S31508023E10DFF903461A460321204610F037FC4B48C1
S31508023E2030F0ACFFDEE27B6803F5C0630622484940
S31508023E3018466AF0F7FE0346002B28D17B6803F57D
S31508023E40C0631846FCF742FB0346062B1FD14148BE
S31508023E5030F094FF10F04EFA0446FEF7B9F903461D
S31508023E601A460221204610F07BFB0346002B0AD095
S31508023E7010F040FA0446FEF7ABF903461A46042147
S31508023E80204610F003FC344830F078FFAAE27B683B
S31508023E9003F5C0630922314918466AF0C3FE034690
S31508023EA0002B63D17B6803F5C0631846FCF70EFB4B
S31508023EB00346092B5AD122F067FD0346184624F019
S31508023EC082F90346002B03D1254830F057FF02E05A
S31508023ED0244830F053FF10F00DFA0446FEF778F93D
S31508023EE003461A460321204610F03AFB0346002BE6
S31508023EF00AD010F0FFF90446FEF76AF903461A4695
S31508023F000521204610F0C2FB174830F037FF69E258
S31508023F10000802428C2C0908B42C0908DC2C090872
S31508023F2000000242042D0908282D0908502D090807
S31508023F30682D0908802D0908982D0908B02D090849
S31508023F40BC2D0908C42D0908CC2D0908F42D090829
S31508023F50182E0908202E0908482E09086C2E090869
S31508023F60782E0908A42E0908E82E09087B6803F5A5
S31508023F70C0630522C24918466AF054FE0346002B5E
S31508023F8040F0B9807B6803F5C0631846FCF79EFAD1
S31508023F900346052B40F0AF8022F0F6FC034618468E
S31508023FA024F011F90346002B04D1B64830F0E6FE98
S31508023FB001F0F1B97B6803F500630422B249184699
S31508023FC06AF030FE0346002B28D17B6803F50063AE
S31508023FD01846FCF77BFA0346042B1FD1AB4830F090
S31508023FE0CDFE10F087F90446FEF7F2F803461A46A4
S31508023FF00621204610F0B4FA0346002B0AD010F028
S3150802400079F90446FEF7E4F803461A460A212046D9
S3150802401010F03CFB9E4830F0B1FE6BE07B6803F57E
S31508024020006305229B4918466AF0FCFD0346002BED
S3150802403028D17B6803F500631846FCF747FA03465E
S31508024040052B1FD1944830F099FE10F053F9044617
S31508024050FEF7BEF803461A460821204610F080FAF3
S315080240600346002B0AD010F045F90446FEF7B0F8CD
S3150802407003461A460C21204610F008FB874830F002
S315080240807DFE37E07B6803F50063092284491846FA
S315080240906AF0C8FD0346002B28D17B6803F5006346
S315080240A01846FCF713FA0346092B1FD17D4830F050
S315080240B065FE10F01FF90446FEF78AF803461A460B
S315080240C00721204610F04CFA0346002B0AD010F0BE
S315080240D011F90446FEF77CF803461A460B212046D8
S315080240E010F0D4FA704830F049FE03E0FEF7EAF819
S315080240F001F051B976E17B6803F5C06306226B4984
S3150802410018466AF08FFD0346002B40F0E3807B6871
S3150802411003F5C0631846FCF7D9F90346062B40F0A7
S31508024120D98022F031FC0346184624F04CF803469F
S31508024130002B04D1534830F021FE01F02CB97B68DC
S3150802414003F5006303225A4918466AF06BFD0346D3
S31508024150002B28D17B6803F500631846FCF7B6F9ED
S315080241600346032B1FD1534830F008FE10F0C2F85D
S315080241700446FEF72DF803461A460921204610F092
S31508024180EFF90346002B0AD010F0B4F80446FEF7FE
S315080241901FF803461A460D21204610F077FA4648BC
S315080241A030F0ECFD6BE07B6803F5006306224349B9
S315080241B018466AF037FD0346002B28D17B6803F5BB
S315080241C000631846FCF782F90346062B1FD13C48C2
S315080241D030F0D4FD10F08EF80446FDF7F9FF0346D9
S315080241E01A460A21204610F0BBF90346002B0AD0CC
S315080241F010F080F80446FDF7EBFF03461A460E2137
S31508024200204610F043FA2F4830F0B8FD37E07B68B5
S3150802421003F5006309222C4918466AF003FD034692
S31508024220002B28D17B6803F500631846FCF74EF984
S315080242300346092B1FD1254830F0A0FD10F05AF885
S315080242400446FDF7C5FF03461A460B21204610F021
S3150802425087F90346002B0AD010F04CF80446FDF7FE
S31508024260B7FF03461A460F21204610F00FFA1848E0
S3150802427030F084FD03E0FEF725F801F08CB8B1E0D2
S31508024280102F0908182F0908402F0908482F09086E
S31508024290742F09089C2F0908A42F0908D02F09088A
S315080242A0F82F09080430090834300908603009086B
S315080242B0683009086C30090898300908C0300908BE
S315080242C0C8300908F4300908203109082C310908D0
S315080242D05C3109087B6803F5C0630822BE491846A3
S315080242E06AF0A0FC0346002B36D17B6803F5C0634F
S315080242F01846FCF7EBF80346082B2DD122F044FBAF
S315080243000346184623F05FFF0346002B04D1B34841
S3150802431030F034FD01F03FB8B14830F02FFD0FF010
S31508024320E9FF0446FDF754FF03461A4604212046D0
S3150802433010F016F90346002B0AD00FF0DBFF0446ED
S31508024340FDF746FF03461A460721204610F09EF956
S31508024350A44830F013FD45E07B6803F5C0630822E4
S31508024360A14918466AF05EFC0346002B36D17B68E3
S3150802437003F5C0631846FCF7A9F80346082B2DD1A6
S3150802438022F002FB0346184623F01DFF0346002BC4
S3150802439004D1924830F0F2FC00F0FDBF934830F0A9
S315080243A0EDFC0FF0A7FF0446FDF712FF03461A4677
S315080243B00521204610F0D4F80346002B0AD00FF048
S315080243C099FF0446FDF704FF03461A4608212046CC
S315080243D010F05CF9864830F0D1FC03E0FDF772FF75
S315080243E000F0D9BF00BF00F0D3BF7B6803F5806336
S315080243F00722804918466AF015FC0346002B40F04E
S31508024400C7877B6803F580631846FCF75FF803469F
S31508024410072B40F0BD877B6803F5C063184669F031
S31508024420B8FAF861FB69012B04D1734830F0A6FC8F
S3150802443000F0AEBFFB69002B04D1704830F09EFC39
S3150802444000F0A6BFFDF73EFF00F0A5BF7B6803F5A7
S31508024450007305226A4918466AF0E4FB0346002BF4
S3150802446040F0F9807B6803F500731846FCF72EF8CE
S315080244700346052B40F0EF807B6803F5806306222E
S31508024480604918466AF0CEFB0346002B4FD17B687B
S3150802449003F580631846FCF719F80346062B46D13E
S315080244A07B6803F5C063184669F073FAF861FB691D
S315080244B0012B21D1544830F061FC15F095F90346D9
S315080244C0184616F0C7FF0346012B0AD14F4830F0AB
S315080244D055FC22F059FA03460321184624F029FC12
S315080244E0B7E04B4830F04AFC22F04EFA0346022166
S315080244F0184624F01EFCACE0FB69002B13D1454894
S3150802450030F03CFC444B1B6800229A63424B1B6802
S3150802451000225A63002140483BF0A2FD04213E488E
S315080245203BF09EFD95E0FDF7CDFE00F034BF7B68BB
S3150802453003F580630822394918466AF073FB034675
S31508024540002B25D17B6803F580631846FBF7BEFF6F
S315080245500346082B1CD17B6803F5C063184669F02D
S3150802456018FAF861FB69012B05D116F00DF92C48EA
S3150802457030F004FC6DE0FB69002B05D116F010F94A
S31508024580284830F0FBFB64E0FDF79CFE00F003BF11
S315080245907B6803F580630822234918466AF042FBC2
S315080245A00346002B51D17B6803F580631846FBF757
S315080245B08DFF0346082B48D17B6803F5C06318466E
S315080245C069F0E7F9F861FB69012B31D116F0F4F8C5
S315080245D0164830F0D3FB3CE08C310908182F09083D
S315080245E098310908C8310908F83109080432090856
S315080245F034320908A02709086432090894320908DE
S315080246001C280908B4320908BC320908D03209083C
S31508024610E832090800330908D46C0120B02D0908CC
S31508024620143309082C330908443309085033090896
S31508024630FB69002B05D116F0CBF8B34830F09EFB88
S3150802464007E0FDF73FFE00F0A6BEFDF73BFE00F0D1
S31508024650A2BE00F0A0BE7B6803F500730822AB4930
S3150802466018466AF0DFFA0346002B40F0B9807B68E9
S3150802467003F500731846FBF729FF0346082B40F09B
S31508024680AF807B6803F580630322A14918466AF066
S31508024690C9FA0346002B1FD17B6803F580631846C7
S315080246A0FBF714FF0346032B16D1F969994830F034
S315080246B065FB15F067FB15F091FB15F0CBFB15F0C2
S315080246C003FC15F039FC15F071FC15F013FD15F015
S315080246D0D9FC15F0A3FC81E07B6803F5806302220E
S315080246E08D4918466AF09EFA0346002B72D17B68FA
S315080246F003F580631846FBF7E9FE0346022B69D1E8
S315080247007B6803F5C063184669F043F9F8617B686C
S3150802471003F50063184669F03CF9B8617B6803F54E
S315080247202063184669F035F90346FB75FB69002BC9
S315080247304ADDFB69042B47DCF969784830F01EFB31
S31508024740B969774830F01AFBFB7D184615F008FB65
S31508024750FB69012B0BD1BB69012B02D115F020FB9A
S3150802476036E0BB69022B33D115F056FB30E0FB6904
S31508024770022B0BD1BB69012B02D115F089FB27E06D
S31508024780BB69022B24D115F0BBFB21E0FB69032B85
S315080247900BD1BB69012B02D115F0EAFB18E0BB6904
S315080247A0022B15D115F088FC12E0FB69042B0FD1F8
S315080247B0BB69012B02D115F04BFC09E0BB69022B40
S315080247C006D115F011FC03E0FDF77CFD00F0E3BD10
S315080247D000BF03E0FDF776FD00F0DDBD00F0DBBDAE
S315080247E07B6803F5007305224E4918466AF01AFAE1
S315080247F00346002B40F06E817B6803F5007318466A
S31508024800FBF764FE0346052B40F064817B6803F5DB
S31508024810806303223E4918466AF004FA0346002BCF
S315080248200ED17B6803F580631846FBF74FFE0346F5
S31508024830032B05D13C4830F0A1FA0EF0EDFF47E113
S315080248407B6803F580630222334918466AF0EAF95F
S315080248500346002B40F038817B6803F580631846CF
S31508024860FBF734FE0346022B40F02E817B6803F5E4
S31508024870C063184669F08DF8F8617B6803F5206312
S31508024880184669F086F8B861FB69002B40F39580F3
S31508024890FB69092B00F391807B6803F500631A789C
S315080248A0224B1B78D31A002B40F087807B6803F5CE
S315080248B000631846FBF70AFE0346012B7DD1F96908
S315080248C01B4830F05BFAFB69012B07D1BB69DBB2E7
S315080248D01A46012133200EF081FFF1E0FB69022B13
S315080248E007D1BB69DBB21A46012134200EF076FFE6
S315080248F0E6E0FB69032B1DD1BB69DBB21A4601212F
S3150802490035200EF06BFFDBE06833090880330908AF
S31508024910382709088C3309081C270908A43309080B
S31508024920BC330908D0330908D8330908EC33090817
S31508024930F0330908FB69042B07D1BB69DBB21A46B7
S31508024940012136200EF04AFFBAE0FB69052B07D192
S31508024950BB69DBB21A46012137200EF03FFFAFE0F2
S31508024960FB69062B07D1BB69DBB21A46012138203F
S315080249700EF034FFA4E0FB69072B07D1BB69DBB253
S315080249801A46012139200EF029FF99E0FB69082B06
S3150802499007D1BB69DBB21A4601213A200EF01EFF87
S315080249A08EE0FB69092B40F08B80BB69DBB21A46A5
S315080249B001213B200EF012FF82E0FB69002B7BDD12
S315080249C0FB69092B78DC7B6803F500631A78AC4B24
S315080249D01B78D31A002B6FD17B6803F50063184640
S315080249E0FBF774FD0346012B66D1F969A54830F039
S315080249F0C5F9FB69012B07D1BB69DBB21A4602214D
S31508024A0033200EF0EBFE5DE0FB69022B07D1BB6992
S31508024A10DBB21A46022134200EF0E0FE52E0FB69B0
S31508024A20032B07D1BB69DBB21A46022135200EF0E9
S31508024A30D5FE47E0FB69042B07D1BB69DBB21A46F0
S31508024A40022136200EF0CAFE3CE0FB69052B07D18F
S31508024A50BB69DBB21A46022137200EF0BFFE31E0EF
S31508024A60FB69062B07D1BB69DBB21A46022138203D
S31508024A700EF0B4FE26E0FB69072B07D1BB69DBB251
S31508024A801A46022139200EF0A9FE1BE0FB69082B03
S31508024A9007D1BB69DBB21A4602213A200EF09EFE06
S31508024AA010E0FB69092B0DD1BB69DBB21A4602215C
S31508024AB03B200EF093FE05E0FDF704FC00F06BBC0C
S31508024AC000BF05E000BF03E0FDF7FCFB00F063BC96
S31508024AD000F061BC7B6803F5007306226A49184632
S31508024AE06AF0A0F80346002B40F0A2807B6803F523
S31508024AF000731846FBF7EAFC0346062B40F098803B
S31508024B007B6803F580630322604918466AF08AF8CF
S31508024B100346002B0ED17B6803F580631846FBF724
S31508024B20D5FC0346032B05D1594830F027F90EF078
S31508024B308BFF7CE07B6803F58063022255491846A1
S31508024B406AF070F80346002B6ED17B6803F5806322
S31508024B501846FBF7BBFC0346022B65D17B6803F5B7
S31508024B60C063184668F015FFF8617B6803F5206391
S31508024B70184668F00EFFB861FB69002B26DDFB6953
S31508024B80012B23DC7B6803F500631A78424B1B78FA
S31508024B90D31A002B1AD17B6803F500631846FBF774
S31508024BA095FC0346012B11D1F9693C4830F0E6F829
S31508024BB0FB69012B07D1BB69DBB21A4601217920B1
S31508024BC00EF024FF2FE0FDF77DFBE4E3FB69002BE3
S31508024BD026DDFB69012B23DC7B6803F500631A7863
S31508024BE0274B1B78D31A002B1AD17B6803F500636F
S31508024BF01846FBF76BFC0346012B11D1F9692848C5
S31508024C0030F0BCF8FB69012B07D1BB69DBB21A4647
S31508024C10022179200EF0FAFE05E0FDF753FBBAE30E
S31508024C20FDF750FBB7E302E0FDF74CFBB3E3B2E353
S31508024C307B6803F5007303221A49184669F0F2FFE6
S31508024C400346002B44D17B6803F500731846FBF72D
S31508024C503DFC0346032B3BD17B6803F5806318466C
S31508024C6068F097FEF861FB69012B21D100224FF407
S31508024C7000710D4834F038FE0C4830F07FF88AE3AC
S31508024C8004340908083409081C34090838270908AD
S31508024C90243409081C270908EC330908383409089A
S31508024CA04C340908603409080014024264340908BD
S31508024CB0FB69002B09D101224FF40071B74834F081
S31508024CC013FEB74830F05AF865E3FDF7FBFA62E3DC
S31508024CD07B6803F500730822B249184669F0A2FFF9
S31508024CE00346002B40F08B807B6803F50073184659
S31508024CF0FBF7ECFB0346082B40F081807B6803F543
S31508024D0080631A78A84B1B78D31A002B33D17B6899
S31508024D1003F580631846FBF7D9FB0346012B2AD114
S31508024D207B6803F5C0631A78A04B1B78D31A002B4D
S31508024D300BD17B6803F5C0631846FBF7C7FB03462E
S31508024D40012B02D115F0EAF914E07B6803F5C0637A
S31508024D501A78974B1B78D31A002B08D17B6803F570
S31508024D60C0631846FBF7B2FB0346012B02D0FDF7D8
S31508024D70A9FA10E342E07B6803F580631A788D4B43
S31508024D801B78D31A002B36D17B6803F58063184645
S31508024D90FBF79CFB0346012B2DD17B6803F5C06309
S31508024DA01A78824B1B78D31A002B0BD17B6803F532
S31508024DB0C0631846FBF78AFB0346012B02D115F09E
S31508024DC0C3F917E07B6803F5C0631A78784B1B783A
S31508024DD0D31A002B0BD17B6803F5C0631846FBF781
S31508024DE075FB0346012B02D115F0C4F902E0FDF763
S31508024DF069FAD0E202E0FDF765FACCE2CBE27B681B
S31508024E0003F500730D226C49184669F00BFF034639
S31508024E10002B40F0A8807B6803F500731846FBF761
S31508024E2055FB03460D2B40F09E807B6803F5C06355
S31508024E301A785E4B1B78D31A002B42D17B6803F58E
S31508024E40C0631846FBF742FB0346012B39D17B6840
S31508024E5003F5806306225949184669F0E3FE0346BC
S31508024E60002B11D17B6803F580631846FBF72EFBEE
S31508024E700346062B08D116F005FA4FF4FA703FF0EE
S31508024E80A7FC16F015FA6CE07B6803F58063062228
S31508024E904B49184669F0C6FE0346002B61D17B686A
S31508024EA003F580631846FBF711FB0346062B58D118
S31508024EB016F01CFA4FF4FA703FF08AFC16F02CFA38
S31508024EC04FE07B6803F5C0631A783E4B1B78D31A0A
S31508024ED0002B40F05F827B6803F5C0631846FBF738
S31508024EE0F5FA0346012B40F055827B6803F5806389
S31508024EF006223249184669F095FE0346002B11D15F
S31508024F007B6803F580631846FBF7E0FA0346062B2F
S31508024F1008D116F017FA4FF4FA703FF059FC16F05A
S31508024F2027FA1FE07B6803F58063062224491846A0
S31508024F3069F078FE0346002B40F02C827B6803F565
S31508024F4080631846FBF7C2FA0346062B40F0228214
S31508024F5016F024FA4FF4FA703FF03AFC16F034FAD7
S31508024F6018E200BF16E27B6803F500730E221649A3
S31508024F70184669F057FE0346002B27D17B6803F5CE
S31508024F8000731846FBF7A2FA03460E2B1ED1FDF74D
S31508024F901FF90346184607F09FFBFCE1001402427C
S31508024FA0703409087C340908EC330908D829090839
S31508024FB0DC290908043409088834090898340908D8
S31508024FC0A0340908A8340908AC3409087B6803F533
S31508024FD000730D22C049184669F024FE0346002BC9
S31508024FE00FD17B6803F500731846FBF76FFA034681
S31508024FF00D2B06D1FDF7ECF80346184607F0EEFB33
S31508025000C9E17B6803F500730622B449184669F0BC
S3150802501009FE0346002B24D17B6803F50073184664
S31508025020FBF754FA0346062B1BD17B6803F580630C
S31508025030184668F0AEFCF861FB69012B05D115F03C
S31508025040AFF8A7482FF09AFEA5E1FB69002B05D118
S3150802505015F0B1F8A3482FF091FE9CE1FDF732F95D
S3150802506099E17B6803F5007305229F49184669F0A2
S31508025070D9FD0346002B40F0C2807B6803F5007316
S315080250801846FBF723FA0346052B40F0B8809748E3
S315080250902FF074FE14F0A8FB0346184614F0D4FB4E
S315080250A00346012B03D192482FF068FE02E091488D
S315080250B02FF064FE14F098FB0346184614F0EBFB37
S315080250C00346012B03D18C482FF058FE02E08B4889
S315080250D02FF054FE14F088FB0346184614F002FC1F
S315080250E00346012B03D186482FF048FE02E0854885
S315080250F02FF044FE14F078FB0346184614F019FC08
S315080251000346012B03D180482FF038FE02E07F4880
S315080251102FF034FE14F068FB0346184614F030FCF0
S315080251200346012B03D17A482FF028FE02E079487C
S315080251302FF024FE14F058FB0346184614F047FCD9
S315080251400346012B03D174482FF018FE02E0734878
S315080251502FF014FE14F048FB0346184614F05EFCC2
S315080251600346012B03D16E482FF008FE02E06D4874
S315080251702FF004FE14F038FB0346184614F075FCAB
S315080251800346012B03D168482FF0F8FD02E0674871
S315080251902FF0F4FD21F0F8FB0346184623F013F826
S315080251A00346002B00F0F780FCF786F80346042135
S315080251B01846FCF7B5F8044610F03AF810EE103A1D
S315080251C01846FBF7EFFA02460B46214658482FF0D7
S315080251D0D5FDFCF771F8034600211846FCF7A0F83E
S315080251E0044610F06DF810EE103A1846FBF7DAFA94
S315080251F002460B4621464F482FF0C0FDCBE07B689E
S3150802520003F5007306224C49184669F00BFD03465E
S31508025210002B1ED17B6803F500731846FBF756F977
S315080252200346062B15D17B6803F58063184668F09A
S31508025230B0FB0346DCB27B6803F5C063184668F028
S31508025240A8FB0346D9B20423002220460BF0B4FD7C
S31508025250A1E07B6803F5007304223849184669F011
S31508025260E1FC0346002B15D17B6803F5007318464B
S31508025270FBF72CF90346042B0CD17B6803F58063F4
S31508025280184668F086FB0346DBB2042118460BF083
S31508025290ADFB80E07B6803F50073042228491846B3
S315080252A069F0C0FC0346002B4CD17B6803F50073FA
S315080252B01846FBF70BF90346042B43D17B6803F523
S315080252C08063184668F065FB0346DBB2042118467C
S315080252D00BF076FC5FE000BFBC340908CC34090841
S315080252E0D4340908E8340908FC34090804350908DD
S315080252F0203509083C3509085C3509087835090856
S3150802530094350908B4350908D4350908F435090865
S315080253101836090834360908503609086C36090859
S3150802532088360908A4360908C0360908DC36090889
S31508025330FC360908243709084C370908543709087E
S315080253405C3709087B6803F500730422134918467B
S3150802535069F068FC0346002B1DD17B6803F50073D0
S315080253601846FBF7B3F80346042B14D17B6803F5FA
S315080253708063184668F00DFB0346DBB20321184624
S315080253800EF05EF907E0FCF79DFF04E000BF02E0BD
S3150802539000BF00E000BF2437BD4690BD6437090848
S315080253A080B586B000AFF8600B467A60FB7221F0D2
S315080253B0EBFA0346184621F01AFD786121F0E4FA61
S315080253C00346184621F005FD38617B6803F500732C
S315080253D004225649184669F025FC0346002B08D1D3
S315080253E07B6803F500731846FBF770F80346042B2F
S315080253F011D07B6803F500731A784D4B1B78D31AC4
S31508025400002B0FD17B6803F500731846FBF75EF88D
S315080254100346012B06D147482FF0B0FC002004F0C2
S315080254206DFA7FE07B6803F500730322424918464A
S3150802543069F0F8FB0346002B0FD17B6803F500736E
S315080254401846FBF743F80346032B06D13B482FF0D1
S3150802545095FC002004F0CCFA64E07B6803F500733F
S3150802546004223749184669F0DDFB0346002B11D1A1
S315080254707B6803F500731846FBF728F80346042BE6
S3150802548008D130482FF07AFC012239697869FCF78D
S315080254909DFB47E07B6803F5007305222A491846F7
S315080254A069F0C0FB0346002B19D17B6803F500732C
S315080254B01846FBF70BF80346052B10D123482FF0A5
S315080254C05DFC002004F034FA10EE103A1846FBF799
S315080254D069F902460B461E482FF050FC22E07B680B
S315080254E003F5007307221B49184669F09BFB03461E
S315080254F0002B14D17B6803F500731846FAF7E6FF0A
S315080255000346072B0BD114482FF038FC002004F071
S31508025510B1F90346194611482FF030FC02E0FCF7B0
S31508025520D1FE00BF1837BD4680BD00BF6C370908DB
S31508025530DC290908743709089037090894370908D5
S31508025540B0370908B8370908D0370908D83709081B
S31508025550F437090808380908103809082C380908E0
S3150802556090B589B002AFF8600B467A60FB720023E9
S31508025570BB820023FB75FB7A022B40F2B5847B685B
S3150802558003F500730422C949184669F04BFB034622
S31508025590002B40F001837B6803F500731846FAF77F
S315080255A095FF0346042B40F0F7827B6803F5806378
S315080255B00522BF49184669F035FB0346002B25D15B
S315080255C07B6803F580631846FAF780FF0346052BC6
S315080255D01CD10EF08FFE0446FCF7FAFD03461A4666
S315080255E0012120460EF0BCFF0346002B0AD00EF01E
S315080255F081FE0446FCF7ECFD03461A4603212046C3
S315080256000FF044F8AB482FF0B9FBC4E27B6803F508
S3150802561080630622A849184669F004FB0346002B54
S3150802562028D17B6803F580631846FAF74FFF0346CD
S31508025630062B1FD1A1482FF0A1FB0EF05BFE0446F4
S31508025640FCF7C6FD03461A46022120460EF088FFDD
S315080256500346002B0AD00EF04DFE0446FCF7B8FDB1
S3150802566003461A46042120460FF010F894482FF0F4
S3150802567085FB90E27B6803F5806309229149184607
S3150802568069F0D0FA0346002B28D17B6803F58063BC
S315080256901846FAF71BFF0346092B1FD18A482FF033
S315080256A06DFB0EF027FE0446FCF792FD03461A46EA
S315080256B0032120460EF054FF0346002B0AD00EF0B3
S315080256C019FE0446FCF784FD03461A4605212046C0
S315080256D00EF0DCFF7D482FF051FB5CE27B6803F598
S315080256E0806305227A49184669F09CFA0346002B1C
S315080256F040F0B8807B6803F580631846FAF7E6FE41
S315080257000346052B40F0AE8021F03EF903461846C3
S3150802571022F059FD0346002B04D16E482FF02EFBCA
S3150802572000F03FBC7B6803F5C06304226A49184649
S3150802573069F078FA0346002B28D17B6803F5C06323
S315080257401846FAF7C3FE0346042B1FD163482FF007
S3150802575015FB0EF0CFFD0446FCF73AFD03461A4642
S31508025760062120460EF0FCFE0346002B0AD00EF058
S31508025770C1FD0446FCF72CFD03461A460A212046BB
S315080257800EF084FF56482FF0F9FA6AE07B6803F5B3
S31508025790C06305225349184669F044FA0346002BAA
S315080257A028D17B6803F5C0631846FAF78FFE0346CD
S315080257B0052B1FD14C482FF0E1FA0EF09BFD04464B
S315080257C0FCF706FD03461A46082120460EF0C8FED7
S315080257D00346002B0AD00EF08DFD0446FCF7F8FCB2
S315080257E003461A460C2120460EF050FF3F482FF07A
S315080257F0C5FA36E07B6803F5C06309223C491846B8
S3150802580069F010FA0346002B28D17B6803F5C063BA
S315080258101846FAF75BFE0346092B1FD135482FF0C7
S31508025820ADFA0EF067FD0446FCF7D2FC03461A46AB
S31508025830072120460EF094FE0346002B0AD00EF0EE
S3150802584059FD0446FCF7C4FC03461A460B212046BA
S315080258500EF01CFF28482FF091FA02E0FCF732FD01
S315080258609FE398E17B6803F580630622234918467D
S3150802587069F0D8F90346002B40F0E2807B6803F50D
S3150802588080631846FAF722FE0346062B40F0D880B4
S3150802589021F07AF80346184622F095FC0346002BB7
S315080258A02ED10C482FF06AFA7BE300BFBC2D0908FB
S315080258B0C42D0908F42D0908182E09083C380908C8
S315080258C0482E09086C2E09085C380908E82E0908CA
S315080258D0102F0908182F0908402F090898380908AF
S315080258E0742F09089C2F0908BC380908D02F090803
S315080258F0F82F0908E0380908343009086030090821
S315080259007B6803F5C0630322C049184669F08AF921
S315080259100346002B28D17B6803F5C0631846FAF7BD
S31508025920D5FD0346032B1FD1B9482FF027FA0EF0EF
S31508025930E1FC0446FCF74CFC03461A4609212046BC
S315080259400EF00EFE0346002B0AD00EF0D3FC0446D8
S31508025950FCF73EFC03461A460D2120460EF096FE3B
S31508025960AC482FF00BFA6AE07B6803F5C06306229F
S31508025970A949184669F056F90346002B28D17B68CF
S3150802598003F5C0631846FAF7A1FD0346062B1FD195
S31508025990A2482FF0F3F90EF0ADFC0446FCF718FC0A
S315080259A003461A460A2120460EF0DAFD0346002B64
S315080259B00AD00EF09FFC0446FCF70AFC03461A4678
S315080259C00E2120460EF062FE95482FF0D7F936E0F2
S315080259D07B6803F5C06309229249184669F022F9E1
S315080259E00346002B28D17B6803F5C0631846FAF7ED
S315080259F06DFD0346092B1FD18B482FF0BFF90EF018
S31508025A0079FC0446FCF7E4FB03461A460B212046BA
S31508025A100EF0A6FD0346002B0AD00EF06BFC0446D8
S31508025A20FCF7D6FB03461A460F2120460EF02EFE39
S31508025A307E482FF0A3F902E0FCF744FCB1E2AAE0A3
S31508025A407B6803F5806308227949184669F0EAF803
S31508025A500346002B35D17B6803F580631846FAF7AF
S31508025A6035FD0346082B2CD120F08EFF0346184637
S31508025A7022F0A9FB0346002B03D16E482FF07EF9CC
S31508025A808FE26D482FF07AF90EF034FC0446FCF7E3
S31508025A909FFB03461A46042120460EF061FD034683
S31508025AA0002B0AD00EF026FC0446FCF791FB0346AF
S31508025AB01A46072120460EF0E9FD60482FF05EF9E6
S31508025AC069E07B6803F5806308225D49184669F038
S31508025AD0A9F80346002B35D17B6803F5806318467F
S31508025AE0FAF7F4FC0346082B2CD120F04DFF0346A7
S31508025AF0184622F068FB0346002B03D14D482FF0C7
S31508025B003DF94EE24F482FF039F90EF0F3FB044601
S31508025B10FCF75EFB03461A46052120460EF020FDD9
S31508025B200346002B0AD00EF0E5FB0446FCF750FBB1
S31508025B3003461A46082120460EF0A8FD42482FF0D1
S31508025B401DF928E07B6803F5806308223F49184659
S31508025B5069F068F80346002B1AD17B6803F580635F
S31508025B601846FAF7B3FC0346082B11D17B6803F5EE
S31508025B70C063184667F00DFF0346BB82FCF728FB95
S31508025B8003461A46BB8A0221184609F08FFB02E031
S31508025B90FCF798FB05E204E27B6803F5007304222E
S31508025BA02B49184669F03EF80346002B40F0FE8062
S31508025BB07B6803F500731846FAF788FC0346042B3C
S31508025BC040F0F4807B6803F5C063184667F0E1FE8F
S31508025BD00346BB827B6803F580631A781D4B1B78E4
S31508025BE0D31A002B4ED17B6803F580631846FAF761
S31508025BF06DFC0346012B45D1BB8A194616482FF080
S31508025C00BDF814F0CDF80023FB7533E068300908B7
S31508025C100839090898300908C03009082C390908D2
S31508025C20F430090820310908543909085C31090891
S31508025C308C310908182F09087C390908C83109085E
S31508025C40F8310908A839090834320908D039090887
S31508025C5014270908D8290908DC39090864203EF0FE
S31508025C60B7FDFCF7B5FA034618462FF067FAFB7D2F
S31508025C700133FB75FB7D9BB2BA8A9A42EED814F0C1
S31508025C80ADF892E07B6803F580631A78AE4B1B7811
S31508025C90D31A002B26D17B6803F580631846FAF7D8
S31508025CA015FC0346012B1DD1BB8A1946A7482FF0BE
S31508025CB065F814F0EDF80023FB750BE064203EF05E
S31508025CC087FDFCF785FA034618462FF037FAFB7D5F
S31508025CD00133FB75FB7D9BB2BA8A9A42EED814F061
S31508025CE0F3F862E07B6803F580631A78984B1B78B1
S31508025CF0D31A002B26D17B6803F580631846FAF778
S31508025D00E5FB0346012B1DD1BB8A194691482FF0A4
S31508025D1035F814F02DF90023FB750BE064203EF0EC
S31508025D2057FDFCF755FA034618462FF007FAFB7D8E
S31508025D300133FB75FB7D9BB2BA8A9A42EED814F000
S31508025D4035F932E07B6803F580631A78824B1B7853
S31508025D50D31A002B26D17B6803F580631846FAF717
S31508025D60B5FB0346012B1DD1BB8A19467B482FF08A
S31508025D7005F814F06DF90023FB750BE064203EF07C
S31508025D8027FDFCF725FA034618462FF0D7F9FB7DBF
S31508025D900133FB75FB7D9BB2BA8A9A42EED814F0A0
S31508025DA071F902E0FCF78EFAFBE0FAE07B6803F58C
S31508025DB0007307226A49184668F034FF0346002B27
S31508025DC040F08F807B6803F500731846FAF77EFB6E
S31508025DD00346072B40F085807B6803F580631A78B3
S31508025DE0604B1B78D31A002B35D17B6803F5806389
S31508025DF01846FAF76BFB0346012B2CD15A482EF0AC
S31508025E00BDFF7B6803F5C0631A78564B1B78D31A15
S31508025E10002B0BD17B6803F5C0631846FAF756FBCD
S31508025E200346012B02D114F07FFD56E07B6803F589
S31508025E30C0631A78444B1B78D31A002B4DD17B6862
S31508025E4003F5C0631846FAF741FB0346012B44D112
S31508025E5014F052FD41E07B6803F580631A78434BE0
S31508025E601B78D31A002B35D17B6803F58063184655
S31508025E70FAF72CFB0346012B2CD13D482EF07EFF68
S31508025E807B6803F5C0631A78364B1B78D31A002B46
S31508025E900BD17B6803F5C0631846FAF717FB03466E
S31508025EA0012B02D114F04CFD19E07B6803F5C0639F
S31508025EB01A78254B1B78D31A002B10D17B6803F569
S31508025EC0C0631846FAF702FB0346012B07D114F002
S31508025ED01FFD04E0FCF7F6F963E000BF61E000BFCE
S31508025EE05FE0FCF7EFF95CE0FB7A012B56D97B6899
S31508025EF003F5007303221F49184668F093FE03460A
S31508025F00002B4ED17B6803F500731846FAF7DEFAC2
S31508025F100346032B30D120F037FD034601211846EC
S31508025F2021F07FF902230093002301220B21672027
S31508025F3024F0B4FC022300930023002210216F20D0
S31508025F4024F0ACFC2DE000BFA8340908143A09086D
S31508025F504C3A0908503A0908883A09088C3A090855
S31508025F60A0270908D8290908C43A0908DC29090812
S31508025F70E43A0908043B09087B6803F5007308221A
S31508025F800949184668F04EFE0346002B09D17B687C
S31508025F9003F500731846FAF799FA02E0FCF792F944
S31508025FA000BF1C37BD4690BD083B0908B0B5ADF524
S31508025FB0956D00AF07F59563A3F29C43186007F544
S31508025FC09563A3F2A4431A6007F59563A3F29D436A
S31508025FD00A461A700023C7F8A434D24852F0B4FB12
S31508025FE0C7F8A004D7F8A00453F0D2FCC7F89C045B
S31508025FF007F59563A3F29D431B78012B40F2DD83D7
S3150802600007F59563A3F2A4431B6803F500730922F7
S31508026010C549184668F006FE0346002B6DD107F5FA
S315080260209563A3F2A4431B6803F500731846FAF7AF
S315080260304DFA0346092B60D107F59563A3F29D43F2
S315080260401B78022B59D920F09FFC0346184621F0EB
S3150802605061FB0346184651F010FF03461946B3483A
S315080260602EF08CFE07F59563A3F2A4431B6803F58D
S315080260708063184667F08DFCC7F8A404D7F8A434E1
S31508026080002B03DDD7F8A434032B02DDFCF71AF93B
S3150802609096E307F5856372220021184668F0BAFD71
S315080260A0A3482EF06BFED7F8A434DBB287F829345E
S315080260B0652387F82A341E23A7F82E34172387F870
S315080260C032340E2387F83434002387F8373407F539
S315080260D0177207F585631146184657F01CFB07F534
S315080260E09563A3F513731B88DAB207F517730233A0
S315080260F01146184606F086F962E307F59563A3F298
S31508026100A4431B6803F500730A228A49184668F0F5
S3150802611089FD0346002B6DD107F59563A3F2A443C7
S315080261201B6803F500731846FAF7D0F903460A2BDB
S3150802613060D107F59563A3F29D431B78022B59D9C3
S3150802614020F022FC0346184621F0E4FA03461846D4
S3150802615051F093FE0346194674482EF00FFE07F5D2
S315080261609563A3F2A4431B6803F58063184667F098
S3150802617010FCC7F8A404D7F8A434002B03DDD7F81B
S31508026180A434032B02DDFCF79DF819E307F58563B2
S3150802619072220021184668F03DFD67482EF0EEFD92
S315080261A0D7F8A434DBB287F82934652387F82A346A
S315080261B01E23A7F83034172387F832340E2387F8BC
S315080261C03434002387F8373407F5177207F58563E1
S315080261D01146184657F09FFA07F59563A3F5137308
S315080261E01B88DAB207F5177302331146184606F00A
S315080261F009F9E5E207F59563A3F2A4431B6803F5DB
S3150802620000730A224D49184668F00CFD0346002B16
S315080262104BD107F59563A3F2A4431B6803F50073F4
S315080262201846FAF753F903460A2B3ED144482EF08C
S31508026230A5FD07F59563A3F2A4431B6803F58063DE
S31508026240184667F0A6FBC7F8A404D7F8A434002BAF
S3150802625003DDD7F8A434032B02DDFCF733F8AFE2EB
S3150802626007F1140372220021184668F0D3FCD7F806
S31508026270A434DAB207F59563A3F294435A7007F188
S31508026280880207F114031146184657F044FA07F52F
S315080262909563A3F584631B88DAB207F18803023390
S315080262A01146184606F0AEF88AE207F59563A3F298
S315080262B0A4431B6803F5007308222249184668F0AE
S315080262C0B1FC0346002B40F0BD8007F59563A3F2A7
S315080262D0A4431B6803F500731846FAF7F7F8034652
S315080262E0082B40F0AF8007F5856372220021184615
S315080262F068F090FC07F59563A3F2A4431B6803F5BF
S315080263008063184667F045FBC7F8A404D7F8A43497
S31508026310002B03DDD7F8A434032B17DD0A482EF029
S315080263202DFD4DE2F4170120143B0908203B09080C
S31508026330683B0908AC3B0908B83B0908FC3B090855
S31508026340083C0908203C09082C3C0908D7F8A4345B
S31508026350DBB287F8293407F59563A3F2A4431B68D1
S3150802636003F5C063184667F014FBC7F8A404D7F808
S31508026370A434512B0BD0D7F8A4345B2B07D0D7F80B
S31508026380A4345C2B03D0CA482EF0F8FC18E2D7F8DE
S31508026390A434DBB287F82A3407F59563A3F2A4433B
S315080263A01B6803F50063184667F0F3FAC7F8A404F6
S315080263B0D7F8A434DBB287F8333407F59563A3F22A
S315080263C0A4431B6803F52063184667F0E2FAC7F888
S315080263D0A404D7F8A434012B03D1012387F8373450
S315080263E002E0002387F83734002387F82B3400238A
S315080263F087F82C340023A7F82E340023A7F8303464
S31508026400002387F83234002387F83434002387F8C8
S315080264103534002387F8363407F5177207F585638E
S315080264201146184657F077F907F59563A3F51373DE
S315080264301B88DAB207F5177302331146184605F0B8
S31508026440E1FFBDE107F59563A3F2A4431B6803F5D3
S31508026450007307229749184668F0E4FB0346002BA7
S3150802646040F0E98007F59563A3F2A4431B6803F598
S3150802647000731846FAF72AF80346072B40F0DB8022
S3150802648020F082FA0346184622F0DCF80346002B6F
S3150802649003D189482EF072FC92E188482EF06EFCF0
S315080264A007F59563A3F2A4431B6803F580631846B0
S315080264B067F06FFAC7F8A40420F066FA034618468E
S315080264C022F0C0F803461A46D7F8A43493420DDDE3
S315080264D020F05AFA0346184622F0B4F80346C7F8DB
S315080264E0A434D7F8A41476482EF048FC20F04CFAC7
S315080264F0044620F049FA0346184622F0A3F8034652
S315080265001A46D7F8A434DBB2D31ADBB219462046A8
S3150802651022F0A7F840F2CB1200216A4868F07AFB0B
S315080265204FF4E5720021684868F074FB4FF4E5728F
S315080265300021664868F06EFB654B00221A70654BAF
S315080265401B780133DAB2634B1A70624B1B78194611
S315080265505C4852F0EAF80121D7F8A00453F0EEF9A4
S315080265600121D7F8A00453F004FA07F59563A3F5B9
S31508026570157340F227221A8007F59563A3F515735A
S3150802658064225A8007F59563A3F5157300221A71DA
S3150802659007F59563A3F5157304225A7107F5157362
S315080265A001224949184655F022FB494B1B781A46DF
S315080265B0D7F89C349C18444863F08EFB054642483B
S315080265C063F095FB03461A462946204668F0D9FB2E
S315080265D03D4863F08CFB0346DAB23D4B1B78134405
S315080265E0DAB23B4B1A70394856F017FD044636485C
S315080265F063F072FB0546344863F079FB03461A4694
S315080266002946204668F0BDFB2F4BB3F8C8212F4B0D
S315080266101A802E492B4857F066FF2C4856F0FDFC87
S3150802662004462A4856F015FD0346DBB219462046AB
S3150802663016F090F8C4E007F59563A3F2A4431B6825
S3150802664003F5007305222449184668F0EBFA034657
S31508026650002B40F0AF8007F59563A3F2A4431B68AD
S3150802666003F500731846F9F731FF0346052B40F088
S31508026670A18007F59563A3F2A4431B6803F5C063DB
S31508026680184667F086F90346002B0CDD07F5956375
S31508026690A3F2A4431B6803F5C063184667F079F9A9
S315080266A003460F2B1CDD0D482EF068FB88E000BF61
S315080266B0503C09089C3C0908A43C0908B83C09084E
S315080266C0D03C0908F417012020160120481401209D
S315080266D0BF190120F2170120F43C0908FC3C0908FD
S315080266E007F59563A3F2A4431B6803F5806318466E
S315080266F067F04FF90346012B14D107F59563A3F208
S31508026700A4431B6803F5C063184667F042F90346BB
S31508026710DCB2FBF75DFD03461A462146652007F003
S3150802672033F84DE007F59563A3F2A4431B6803F516
S315080267308063184667F02DF90346022B14D107F534
S315080267409563A3F2A4431B6803F5C063184667F072
S3150802675020F90346DCB2FBF73BFD03461A462146FF
S31508026760662007F011F82BE007F59563A3F2A44318
S315080267701B6803F58063184667F00BF90346032B7B
S3150802678014D107F59563A3F2A4431B6803F5C06306
S31508026790184667F0FEF80346DCB2FBF719FD034616
S315080267A01A462146672006F0EFFF09E006482EF052
S315080267B0E5FA05E0FBF786FD02E0FBF783FD00BF7D
S315080267C007F59567BD46B0BD283D090890B585B061
S315080267D000AFF8600B467A60FB7220F0D5F80446E3
S315080267E07B6803F50073184667F0D3F80346DBB2F5
S315080267F01946204621F013FF00BF1437BD4690BD47
S3150802680090B589B000AFF8600B467A60FB72002338
S31508026810FB610023BB6100237B61FB7A012B41F2FA
S31508026820DA807B6803F500730722B649184668F0D2
S31508026830F9F90346002B60D17B6803F50073184605
S31508026840F9F744FE0346072B57D17B6803F58063A5
S31508026850184667F09EF8B861BB69002B49DDBB692B
S31508026860052B46DC7B6803F5C063184667F091F88A
S3150802687078617B69002B38DD7B69032B35DC7A6905
S31508026880B969A1482EF07AFA062200219F4868F0D3
S31508026890C1F901219D4850F0CCFFBB69DBB219460C
S315080268A09A4850F0E1FF7B69DBB21946974850F0E7
S315080268B0F6FF67F029F90346DBB21946934851F009
S315080268C03FF89349914856F06DFE914856F0A5FB5C
S315080268D004468F4856F0BDFB0346DBB219462046EE
S315080268E015F038FF00BF01F079B8FBF7EBFC01F0B1
S315080268F075B8FBF7E7FC01F071B87B6803F500731E
S3150802690007228449184668F08DF90346002B5ED1A2
S315080269107B6803F500731846F9F7D8FD0346072B7B
S3150802692055D17B6803F58063184667F032F8F8613B
S315080269307B6803F5C063184667F02BF87861FB6934
S31508026940002B40DDFB69112B3DDC7B69002B02DD48
S315080269507B69042B02DD7B69C82B34D17A69F96914
S315080269606D482EF00BFA06220021684868F052F9A3
S315080269700821664850F05DFFFB69DBB21946634899
S3150802698050F072FF7B69DBB21946604850F087FF08
S3150802699067F0BAF80346DBB219465C4850F0D0FFF6
S315080269A05B495A4856F0FEFD594856F036FB0446EE
S315080269B0574856F04EFB0346DBB21946204615F0F9
S315080269C0C9FE01F00BB8FBF77DFC01F007B87B683E
S315080269D003F5007309225149184668F023F903465C
S315080269E0002B40F03F827B6803F500731846F9F7DF
S315080269F06DFD0346092B40F035827B6803F58063FB
S31508026A0008224749184668F00DF90346002B36D185
S31508026A107B6803F580631846F9F758FD0346082B89
S31508026A202DD140482EF0AAF906220021374868F0EF
S31508026A30F1F80421354850F0FCFE0121334850F0A4
S31508026A4013FF0021314850F02AFF67F05DF803462C
S31508026A50DBB219462D4850F073FF2D492B4856F0E4
S31508026A60A1FD2B4856F0D9FA0446294856F0F1FA00
S31508026A700346DBB21946204615F06CFED4E17B6864
S31508026A8003F5806308222849184668F0CBF80346BE
S31508026A90002B4BD17B6803F580631846F9F716FD80
S31508026AA00346082B42D11F482EF068F90622002118
S31508026AB0164868F0AFF80421144850F0BAFE0221CD
S31508026AC0124850F0D1FE0021104850F0E8FE67F057
S31508026AD01BF80346DBB219460C4850F031FF0C4945
S31508026AE00A4856F05FFD0A4856F097FA04460848DF
S31508026AF056F0AFFA0346DBB21946204615F02AFECF
S31508026B0092E100BF5C3D0908643D0908141601209C
S31508026B1048140120903D0908983D0908C83D09080E
S31508026B20D43D0908E03D0908EC3D09087B6803F5F0
S31508026B3080630A22BD49184668F074F80346002B9A
S31508026B4036D17B6803F580631846F9F7BFFC03461E
S31508026B500A2B2DD1B6482EF011F906220021B54886
S31508026B6068F058F80521B34850F063FE0121B14890
S31508026B7050F07AFE0021AF4850F091FE66F0C4FF4D
S31508026B800346DBB21946AB4850F0DAFEAA49A948D1
S31508026B9056F008FDA84856F040FA0446A64856F0AC
S31508026BA058FA0346DBB21946204615F0D3FD3BE1F7
S31508026BB07B6803F580630A22A049184668F032F812
S31508026BC00346002B36D17B6803F580631846F9F72E
S31508026BD07DFC03460A2B2DD199482EF0CFF80622C2
S31508026BE00021944868F016F80521924850F021FED3
S31508026BF00221904850F038FE00218E4850F04FFE90
S31508026C0066F082FF0346DBB219468A4850F098FEC0
S31508026C108949884856F0C6FC874856F0FEF9044664
S31508026C20854856F016FA0346DBB21946204615F091
S31508026C3091FDF9E07B6803F58063052281491846D0
S31508026C4067F0F0FF0346002B36D17B6803F58063B5
S31508026C501846F9F73BFC0346052B2DD17A482EF048
S31508026C608DF806220021734867F0D4FF0221714885
S31508026C7050F0DFFD05216F4850F0F6FD00216D4802
S31508026C8050F00DFE66F040FF0346DBB2194669482E
S31508026C9050F056FE6849674856F084FC664856F036
S31508026CA0BCF90446644856F0D4F90346DBB21946E1
S31508026CB0204615F04FFDB7E07B6803F58063062290
S31508026CC06249184667F0AEFF0346002B36D17B6849
S31508026CD003F580631846F9F7F9FB0346062B2DD10F
S31508026CE05B482EF04BF806220021524867F092FFC5
S31508026CF00621504850F09DFD05214E4850F0B4FD3E
S31508026D0000214C4850F0CBFD66F0FEFE0346DBB28E
S31508026D101946484850F014FE4749464856F042FC80
S31508026D20454856F07AF90446434856F092F903461E
S31508026D30DBB21946204615F00DFD75E07B6803F5B2
S31508026D40806309224349184667F06CFF0346002B05
S31508026D5008D17B6803F580631846F9F7B7FB034643
S31508026D60092B13D07B6803F5806309223A49184632
S31508026D7067F058FF0346002B52D17B6803F5806300
S31508026D801846F9F7A3FB0346092B49D10622002127
S31508026D90284867F03FFF0621264850F04AFD7B68DF
S31508026DA003F5806309222B49184667F03BFF034621
S31508026DB0002B10D17B6803F580631846F9F786FB2A
S31508026DC00346092B07D125482DF0D8FFFF2119487C
S31508026DD050F04AFD06E022482DF0D0FFFE21154864
S31508026DE050F042FD0021134850F059FD66F08CFE22
S31508026DF00346DBB219460F4850F0A2FD0E490D486C
S31508026E0056F0D0FB0C4856F008F904460A4856F0E4
S31508026E1020F90346DBB21946204615F09BFC03E02F
S31508026E20FBF750FA00F0DABD00F0D8BDF83D0908C4
S31508026E30043E09081416012048140120143E0908C4
S31508026E40203E0908303E0908383E0908543E09081A
S31508026E505C3E09087C3E0908883E0908943E0908F2
S31508026E60B43E09087B6803F500730A22BF4918462F
S31508026E7067F0D8FE0346002B47D17B6803F50073FB
S31508026E801846F9F723FB03460A2B3ED17B6803F51E
S31508026E908063184666F07DFDF861FB69002B30DDDC
S31508026EA0FB690B2B2DDCF969B1482DF067FF062229
S31508026EB00021B04867F0AEFE0721AE4850F0B9FC93
S31508026EC0FB69DBB21946AB4850F0CEFC66F01CFEF5
S31508026ED00346DBB21946A74850F032FDA649A54833
S31508026EE056F060FBA44856F098F80446A24856F0B5
S31508026EF0B0F80346DBB21946204615F02BFC00F023
S31508026F006DBDFBF7DFF900F069BD7B6803F5007319
S31508026F1009229A49184667F085FE0346002B40F077
S31508026F203F817B6803F500731846F9F7CFFA0346E3
S31508026F30092B40F035817B6803F58063022290496C
S31508026F40184667F06FFE0346002B32D17B6803F5BD
S31508026F5080631846F9F7BAFA0346022B29D18948FB
S31508026F602DF00CFF06220021824867F053FE66F0D8
S31508026F70CBFD0346DBB219467E4850F0E1FC0F21F1
S31508026F807C4850F056FC01217A4850F06DFC7A494B
S31508026F90784856F007FB784856F03FF80446764894
S31508026FA056F057F80346DBB21946204615F0D2FBCF
S31508026FB0D9E07B6803F5806304227349184667F0B3
S31508026FC031FE0346002B32D17B6803F580631846EF
S31508026FD0F9F77CFA0346042B29D16C482DF0CEFE2C
S31508026FE006220021634867F015FE66F08DFD03460A
S31508026FF0DBB219465F4850F0A3FC0F215D4850F0FA
S3150802700018FC02215B4850F02FFC5B49594856F0A0
S31508027010C9FA594856F001F80446574856F019F87D
S315080270200346DBB21946204615F094FB9BE07B68C3
S3150802703003F5806303225649184667F0F3FD0346B3
S31508027040002B40D17B6803F580631846F9F73EFAB0
S315080270500346032B37D17B6803F5C063184666F0EF
S3150802706098FCF861F9694B482DF088FE0622002142
S31508027070404867F0CFFD66F047FD0346DBB2194686
S315080270803C4850F05DFC0F213A4850F0D2FB0321F0
S31508027090384850F0E9FBFB69DBB21946354850F02F
S315080270A0FEFB3549334856F07DFA334855F0B5FFAD
S315080270B00446314855F0CDFF0346DBB21946204651
S315080270C015F048FB4FE07B6803F5806307223249D7
S315080270D0184667F0A7FD0346002B40D17B6803F5E7
S315080270E080631846F9F7F2F90346072B37D17B680E
S315080270F003F5C063184666F04CFCF861F96927483F
S315080271002DF03CFE062200211A4867F083FD66F040
S31508027110FBFC0346DBB21946164850F011FC0F2158
S31508027120144850F086FB0421124850F09DFBFB6977
S31508027130DBB219460F4850F0B2FB0F490D4856F01C
S3150802714031FA0D4855F069FF04460B4855F081FFA0
S315080271500346DBB21946204615F0FCFA03E0FBF7B4
S31508027160B1F800F03BBC00F039BC00BFD43E0908B8
S31508027170E03E090814160120481401200C3F0908AC
S31508027180183F09081C3F0908383F0908403F090803
S315080271905C3F0908603F0908783F0908803F0908EB
S315080271A07B6803F500730822AF49184667F03AFD73
S315080271B00346002B6CD17B6803F500731846F9F772
S315080271C085F90346082B63D1FB7A042B5DD97B68C4
S315080271D003F58063184666F0DCFB0346DAB2A34B76
S315080271E01A707B6803F5C063184666F0D2FB03463D
S315080271F0DAB29F4B1A707B6803F50063184666F08D
S31508027200C8FB0346DAB29B4B1A707B6803F5206308
S31508027210184666F0BEFB0346DAB2974B1A700B2184
S31508027220964850F006FB914B1B781946934850F046
S315080272301BFB8F4B1B781946904850F030FB8D4B41
S315080272401B7819468D4850F045FB8B4B1B7819461F
S315080272508A4850F05AFB66F057FC0346DBB21946D9
S31508027260864850F06DFB8649844856F09BF9844857
S3150802727055F0D3FE0446824855F0EBFE0346DBB2D0
S315080272801946204615F066FAA8E3FBF71BF8A5E3AC
S315080272907B6803F5007306227A49184667F0C2FC32
S315080272A00346002B34D17B6803F500731846F9F7B9
S315080272B00DF90346062B2BD17B6803F58063184626
S315080272C066F067FB78617B69002B05DC7B69032B1B
S315080272D002DDFAF7F7FF81E379696B482DF04EFD77
S315080272E07B69DBB21946694851F098F964496748DF
S315080272F056F0EDFF624855F090FE0446604855F098
S31508027300A8FE0346DBB21946204615F023FA65E3C2
S315080273107B6803F5007307225D49184667F082FC0D
S315080273200346002B34D17B6803F500731846F9F738
S31508027330CDF80346072B2BD17B6803F580631846E5
S3150802734066F027FB78617B69002B05DC7B69032BDA
S3150802735002DDFAF7B7FF41E379694E482DF00EFDD3
S315080273607B69DBB219464C4851F08EF944494A48C2
S3150802737057F00BF8424855F050FE0446404855F07F
S3150802738068FE0346DBB21946204615F0E3F925E303
S315080273907B6803F5007305224049184667F042FCEC
S315080273A00346002B25D17B6803F500731846F9F7C7
S315080273B08DF80346052B1CD166F0A6FB0346DBB205
S315080273C01946374851F0A7FD2D49354857F0D1FCE3
S315080273D02B4855F022FE0446294855F03AFE034644
S315080273E0DBB21946204615F0B5F92E482DF0C6FC33
S315080273F0F4E27B6803F5007308222B49184667F006
S3150802740011FC0346002B55D17B6803F50073184619
S31508027410F9F75CF80346082B4CD17B6803F58063C1
S31508027420184666F0B6FAF861012200211F4867F08D
S31508027430F1FB1F482DF0A2FCFB69DBB219461B487B
S3150802744050F0F2FE0E49194856F0D9FD0C4855F08F
S31508027450E4FD04460A4855F0FCFD0346DBB219462C
S31508027460204615F077F9B9E2A03F0908D01901209C
S31508027470D1190120D2190120D3190120141601208D
S3150802748048140120AC3F0908B43F0908EC1701204B
S31508027490D43F0908DC3F0908F0170120F83F09081C
S315080274A0C019012000400908144009081C160120C9
S315080274B0204009087B6803F500730722AF4918467E
S315080274C067F0B0FB0346002B40F072817B6803F538
S315080274D000731846F8F7FAFF0346072B40F068814F
S315080274E07B6803F580630422A549184667F09AFB70
S315080274F00346002B36D17B6803F580631846F8F7F6
S31508027500E5FF0346042B2DD19E482DF037FC0622B3
S3150802751000219D4867F07EFB09219B4850F089F9B6
S315080275200121994850F0A0F90021974850F0B7F97F
S3150802753066F0EAFA0346DBB21946934850F000FAB7
S315080275409249914856F02EF8904855F066FD044641
S315080275508E4855F07EFD0346DBB21946204615F0E5
S31508027560F9F80AE17B6803F5806307228849184619
S3150802757067F058FB0346002B36D17B6803F5806318
S315080275801846F8F7A3FF0346072B2DD181482DF09D
S31508027590F5FB062200217C4867F03CFB09217A4864
S315080275A050F047F90221784850F05EF900217648F2
S315080275B050F075F966F0A8FA0346DBB21946724826
S315080275C050F0BEF97149704855F0ECFF6F4855F016
S315080275D024FD04466D4855F03CFD0346DBB21946C8
S315080275E0204615F0B7F8C8E07B6803F580630722E2
S315080275F06949184667F016FB0346002B36D17B68A5
S3150802760003F580631846F8F761FF0346072B2DD169
S3150802761062482DF0B3FB062200215B4867F0FAFAAE
S315080276200921594850F005F90321574850F01CF929
S315080276300021554850F033F966F066FA0346DBB284
S315080276401946514850F07CF950494F4855F0AAFF5F
S315080276504E4855F0E2FC04464C4855F0FAFC0346FF
S31508027660DBB21946204615F075F886E07B6803F505
S31508027670806307224A49184667F0D4FA0346002B64
S3150802768036D17B6803F580631846F8F71FFF034671
S31508027690072B2DD143482DF071FB062200213A48CB
S315080276A067F0B8FA0921384850F0C3F80421364879
S315080276B050F0DAF80021344850F0F1F866F024FA6E
S315080276C00346DBB21946304850F03AF92F492E489C
S315080276D055F068FF2D4855F0A0FC04462B4855F096
S315080276E0B8FC0346DBB21946204615F033F844E0E7
S315080276F07B6803F5806304222B49184667F092FAE1
S315080277000346002B36D17B6803F580631846F8F7E3
S31508027710DDFE0346042B2DD124482DF02FFB06222D
S315080277200021194867F076FA0921174850F081F8BE
S315080277300521154850F098F80A21134850F0AFF879
S3150802774066F0E2F90346DBB219460F4850F0F8F83C
S315080277500E490D4855F026FF0C4855F05EFC0446C6
S315080277600A4855F076FC0346DBB21946204614F061
S31508027770F1FF02E0FAF7A6FD30E12FE13C400908E5
S31508027780444009084C4009081416012048140120EF
S31508027790744009087C400908A8400908B04009084D
S315080277A0DC400908E440090810410908184109089B
S315080277B07B6803F500730A228A49184667F032FA8B
S315080277C00346002B40F0D6807B6803F50073184603
S315080277D0F8F77CFE03460A2B40F0CC807B6803F55B
S315080277E0C063184666F0D5F8F861032200217E4880
S315080277F067F010FA7B6803F5806303227B49184613
S3150802780067F010FA0346002B11D17B6803F58063F3
S315080278101846F8F75BFE0346032B08D1F969744844
S315080278202DF0ACFA0121704851F0F4FC82E07B6835
S3150802783003F5806306226F49184667F0F3F9034693
S31508027840002B11D17B6803F580631846F8F73EFED4
S315080278500346062B08D1F96965482DF08FFA0221ED
S31508027860614851F0D7FC65E07B6803F58063022224
S315080278706149184667F0D6F90346002B11D17B6891
S3150802788003F580631846F8F721FE0346022B08D152
S31508027890F9695A482DF072FA0421534851F0BAFC94
S315080278A048E07B6803F5806303225549184667F06A
S315080278B0B9F90346002B11D17B6803F58063184694
S315080278C0F8F704FE0346032B08D1F9694D482DF053
S315080278D055FA0821444851F09DFC2BE07B6803F5D4
S315080278E0806303224849184667F09CF90346002B31
S315080278F01DD17B6803F580631846F8F7E7FD034652
S31508027900032B14D1F96941482DF038FA012136487A
S3150802791051F080FC0221344851F07CFC04213248A3
S3150802792051F078FC0821304851F074FC02E0FAF76D
S31508027930C9FC53E066F0E8F80346DBB219462A4862
S3150802794051F03CFCFB69DBB21946274851F088FC2A
S315080279502F49254857F04EFB2D4855F05EFB044645
S315080279602B4855F076FB0346DBB21946204614F03F
S31508027970F1FE33E07B6803F50073072225491846B2
S3150802798067F050F90346002B22D17B6803F5007392
S315080279901846F8F79BFD0346072B19D11E482DF00A
S315080279A0EDF94FF4E5720021194867F033F91848E2
S315080279B057F048F9164855F030FB0446144855F076
S315080279C048FB0346DBB21946204614F0C3FE05E01F
S315080279D0FAF778FC02E0FAF775FC00BF2437BD46D1
S315080279E090BD00BF44410908C4190120683009083E
S315080279F050410908C0300908684109086C4109085C
S31508027A00884109088C410908A4410908A8410908BE
S31508027A1048140120C0410908C841090880B586B042
S31508027A2000AFF8600B467A60FB720023FB750023F1
S31508027A30BB757B6803F5007309224F49184667F040
S31508027A40F1F80346002B40F08D807B6803F500733E
S31508027A501846F8F73BFD0346092B40F083807B68FE
S31508027A6003F58063184665F094FF0346BB75BB7D34
S31508027A7018460CF033F90346FB75082200213F48E5
S31508027A8067F0C8F840F2D2413C4822F069FABB7D59
S31508027A90022B14D0BB7D032B11D0BB7D062B0ED037
S31508027AA0BB7D072B0BD0BB7D0A2B08D0BB7D0B2BCE
S31508027AB005D0BB7D0E2B02D0BB7D0F2B04D16421D2
S31508027AC02E4822F068FA03E064212C4822F07EFA56
S31508027AD0BB7D1946294822F094FAFB7D19462748A8
S31508027AE022F0AAFABB7D062B05D0BB7D022B02D05B
S31508027AF0BB7D072B04D12149002022F0ADFA30E0E4
S31508027B00BB7D0A2B08D0BB7D0E2B05D0BB7D0F2B68
S31508027B1002D0BB7D0B2B04D11849012022F09CFA16
S31508027B201FE0BB7D012B04D11449022022F094FAEE
S31508027B301CE0BB7D052B04D11049032022F08CFAE8
S31508027B4014E0BB7D092B04D10C49042022F084FAE7
S31508027B500CE0BB7D0D2B09D10849052022F07CFAE1
S31508027B6004E003E006482DF009F900E000BF00BF73
S31508027B701837BD4680BD00BFDC410908C819012077
S31508027B80E841090880B584B000AFF8600B467A6010
S31508027B90FB72FB7A012B77D97B6803F50073042203
S31508027BA03E49184667F03EF80346002B66D17B68C5
S31508027BB003F500731846F8F789FC0346042B5DD1D2
S31508027BC07B6803F580631A78354B1B78D31A002B2A
S31508027BD013D17B6803F580631846F8F777FC0346EA
S31508027BE0012B0AD12F482DF0C9F811F0D1FC034612
S31508027BF00021184611F0E6FC3FE07B6803F5806336
S31508027C001A78294B1B78D31A002B13D17B6803F5F4
S31508027C1080631846F8F75AFC0346012B0AD1234813
S31508027C202DF0ACF811F0B4FC03460121184611F008
S31508027C30C9FC22E07B6803F580631A781C4B1B7823
S31508027C40D31A002B13D17B6803F580631846F8F71D
S31508027C503DFC0346012B0AD116482DF08FF811F088
S31508027C6097FC03460221184611F0ACFC05E01248BF
S31508027C702DF084F8FAF726FB0CE00BE00E482DF0FF
S31508027C807DF8FAF71FFB05E00B482DF077F8FAF7AF
S31508027C9019FB00BF1037BD4680BD00BFF841090871
S31508027CA0D829090800420908A834090828420908F7
S31508027CB04C3A0908544209088042090880B584B03A
S31508027CC000AFF8600B467A60FB727B6803F50073B7
S31508027CD00A22B649184666F0A5FF0346002B44D188
S31508027CE07B6803F500731846F8F7F0FB03460A2B80
S31508027CF03BD17B6803F580631A78AD4B1B78D31AA0
S31508027D00002B13D17B6803F580631846F8F7DEFB70
S31508027D100346012B0AD11EF037FE034601211846F7
S31508027D2020F011F8A3482DF029F851E27B6803F5F3
S31508027D3080631A78A04B1B78D31A002B40F048822E
S31508027D407B6803F580631846F8F7C0FB0346012BE8
S31508027D5040F03E821EF018FE0346002118461FF028
S31508027D60F2FF96482DF00AF832E27B6803F50073B3
S31508027D7008229349184666F055FF0346002B44D15C
S31508027D807B6803F500731846F8F7A0FB0346082B31
S31508027D903BD17B6803F580631A78854B1B78D31A27
S31508027DA0002B13D17B6803F580631846F8F78EFB20
S31508027DB00346012B0AD11EF0E7FD034601211846A8
S31508027DC01FF0ECFF7B482CF0D9FF03E27B6803F532
S31508027DD080631A78784B1B78D31A002B40F0FA8105
S31508027DE07B6803F580631846F8F770FB0346012B98
S31508027DF040F0F0811EF0C8FD0346002118461FF028
S31508027E00CDFF6E482CF0BAFFE4E17B6803F50073F8
S31508027E1008226C49184666F005FF0346002B44D132
S31508027E207B6803F500731846F8F750FB0346082BE0
S31508027E303BD17B6803F580631A785D4B1B78D31AAE
S31508027E40002B13D17B6803F580631846F8F73EFBCF
S31508027E500346012B0AD11EF097FD03460121184657
S31508027E601FF0B8FF53482CF089FFB5E17B6803F58C
S31508027E7080631A78504B1B78D31A002B40F0AC81DA
S31508027E807B6803F580631846F8F720FB0346012B47
S31508027E9040F0A2811EF078FD0346002118461FF025
S31508027EA099FF46482CF06AFF96E17B6803F5007352
S31508027EB008224549184666F0B5FE0346002B44D10A
S31508027EC07B6803F500731846F8F700FB0346082B90
S31508027ED03BD17B6803F580631A78354B1B78D31A36
S31508027EE0002B13D17B6803F580631846F8F7EEFA80
S31508027EF00346012B0AD11EF047FD03460121184607
S31508027F001FF093FF2B482CF039FF67E17B6803F5D6
S31508027F1080631A78284B1B78D31A002B40F05E81AF
S31508027F207B6803F580631846F8F7D0FA0346012BF7
S31508027F3040F054811EF028FD0346002118461FF022
S31508027F4074FF1E482CF01AFF48E17B6803F500739C
S31508027F500C221E49184666F065FE0346002B56D1CA
S31508027F607B6803F500731846F8F7B0FA03460C2B3C
S31508027F704DD17B6803F580631A780D4B1B78D31AAB
S31508027F80002B25D17B6803F580631846F8F79EFA1D
S31508027F900346012B1CD11EF0F7FC034601211846A5
S31508027FA01FF06EFF03482CF0E9FE19E1D0430908D9
S31508027FB0D8290908DC430908DC290908F443090811
S31508027FC00C440908184409082444090830440908D5
S31508027FD07B6803F580631A78854B1B78D31A002BC6
S31508027FE040F0FE807B6803F580631846F8F76EFA60
S31508027FF00346012B40F0F4801EF0C6FC034600211E
S3150802800018461FF03DFF7B482CF0B8FEE8E07B6877
S3150802801003F500730A227849184666F003FE0346FA
S31508028020002B64D17B6803F500731846F8F74EFAFD
S3150802803003460A2B5BD17B6803F580631A786F4B7C
S315080280401B78D31A002B08D17B6803F58063184680
S31508028050F8F73CFA0346012B13D07B6803F58063D5
S3150802806002226749184666F0DDFD0346002B0FD14A
S315080280707B6803F580631846F8F728FA0346022B4D
S3150802808006D1604B01221A705F482CF077FEA9E0F0
S315080280907B6803F580631A78554B1B78D31A002B35
S315080280A008D17B6803F580631846F8F70FFA03468A
S315080280B0012B15D07B6803F58063032253491846C2
S315080280C066F0B0FD0346002B40F08C807B6803F512
S315080280D080631846F8F7FAF90346032B40F08280C4
S315080280E0484B00221A704A482CF048FE7AE07B6810
S315080280F003F500730A224749184666F093FD0346BC
S31508028100002B62D17B6803F500731846F8F7DEF98F
S3150802811003460A2B59D17B6803F580631A78374BD5
S315080281201B78D31A002B08D17B6803F5806318469F
S31508028130F8F7CCF90346012B13D07B6803F5806365
S3150802814002222F49184666F06DFD0346002B0FD111
S315080281507B6803F580631846F8F7B8F90346022BDD
S3150802816006D12D4B01221A702C482CF007FE3BE053
S315080281707B6803F580631A781D4B1B78D31A002B8C
S3150802818008D17B6803F580631846F8F79FF903461A
S31508028190012B13D07B6803F5806303221B4918461B
S315080281A066F040FD0346002B1ED17B6803F580630B
S315080281B01846F8F78BF90346032B15D1164B0022FE
S315080281C01A7017482CF0DAFD0EE0FAF77BF80CE085
S315080281D000BF0AE000BF08E000BF06E000BF04E0F7
S315080281E000BF02E000BF00E000BF1037BD4680BDF9
S315080281F0DC290908F443090840440908D82909086A
S315080282001C270908C1FF00204C4409083827090819
S31508028210644409087C4409080000002088440908C7
S31508028220A044090880B586B000AFF8600B467A60AC
S31508028230FB7200237B610023FB747B6803F52063D2
S31508028240184665F0A6FB0346FB74FB7C1946A6484E
S315080282502CF094FDF9F776F80246FB7C194610468F
S31508028260F9F762F97B6803F5007304229F491846F9
S3150802827066F0D8FC0346002B40F00E837B6803F5B4
S3150802828000731846F8F722F90346042B40F00483D4
S315080282907B6803F5806303229549184666F0C2FC9B
S315080282A00346002B40F089807B6803F580631846F5
S315080282B0F8F70CF90346032B7FD17B6803F5C063F5
S315080282C01A788C4B1B78D31A002B34D17B6803F5AA
S315080282D0C0631846F8F7FAF80346012B2BD17B68D8
S315080282E003F50063184665F054FB78617B69002B39
S315080282F01EDDF9F727F8034600211846F9F75EF856
S31508028300F9F720F8034601211846F9F7B1F8F9F703
S3150802831019F8034601211846F9F7C5F8F9F712F8CC
S3150802832002467B69DBB219461046F9F7E2F843E0E2
S31508028330F9F7C8FFC9E27B6803F5C0631A786E4B82
S315080283401B78D31A002B34D17B6803F5C063184611
S31508028350F8F7BCF80346012B2BD17B6803F50063BB
S31508028360184665F016FB78617B69002B1EDDF8F767
S31508028370E9FF034600211846F9F720F8F8F7E2FF65
S31508028380034601211846F9F773F8F8F7DBFF0346A7
S3150802839002211846F9F787F8F8F7D4FF02467B69EF
S315080283A0DBB219461046F9F7A4F805E0F9F78AFF91
S315080283B08BE2F9F787FF88E26DE27B6803F5806353
S315080283C003224E49184666F02DFC0346002B40F060
S315080283D097807B6803F580631846F8F777F80346B3
S315080283E0032B40F08D807B6803F5C0631A78414BF6
S315080283F01B78D31A002B34D17B6803F5C063184661
S31508028400F8F764F80346012B2BD17B6803F5006362
S31508028410184665F0BEFA78617B69002B1EDDF8F70F
S3150802842091FF034600211846F8F7C8FFF8F78AFFB6
S31508028430034602211846F9F71BF8F8F783FF0346A5
S3150802844001211846F9F72FF8F8F77CFF02467B69EF
S31508028450DBB219461046F9F74CF843E0F9F732FF52
S3150802846033E27B6803F5C0631A78234B1B78D31A69
S31508028470002B34D17B6803F5C0631846F8F726F853
S315080284800346012B2BD17B6803F50063184665F07A
S3150802849080FA78617B69002B1EDDF8F753FF0346E5
S315080284A000211846F8F78AFFF8F74CFF034602211F
S315080284B01846F8F7DDFFF8F745FF03460221184686
S315080284C0F8F7F1FFF8F73EFF02467B69DBB2194679
S315080284D01046F9F70EF805E0F9F7F4FEF5E1F9F7B3
S315080284E0F1FEF2E1D7E100BFB8440908F8410908EC
S315080284F0D0440908EC33090804340908D4440908A5
S315080285007B6803F580630222BB49184666F08AFB3C
S315080285100346002B40F089807B6803F58063184682
S31508028520F7F7D4FF0346022B7FD17B6803F5C063B6
S315080285301A78B24B1B78D31A002B34D17B6803F511
S31508028540C0631846F7F7C2FF0346012B2BD17B6897
S3150802855003F50063184665F01CFA78617B69002BFF
S315080285601EDDF8F7EFFE034600211846F8F726FF48
S31508028570F8F7E8FE034603211846F8F779FFF8F7F5
S31508028580E1FE034601211846F8F78DFFF8F7DAFEF1
S3150802859002467B69DBB219461046F8F7AAFF43E0A2
S315080285A0F9F790FE91E17B6803F5C0631A78944B5C
S315080285B01B78D31A002B34D17B6803F5C06318469F
S315080285C0F7F784FF0346012B2BD17B6803F500637B
S315080285D0184665F0DEF978617B69002B1EDDF8F72F
S315080285E0B1FE034600211846F8F7E8FEF8F7AAFE98
S315080285F0034603211846F8F73BFFF8F7A3FE03469E
S3150802860002211846F8F74FFFF8F79CFE02467B69E7
S31508028610DBB219461046F8F76CFF05E0F9F752FE89
S3150802862053E1F9F74FFE50E135E17B6803F58063C4
S3150802863002227449184666F0F5FA0346002B40F002
S3150802864089807B6803F580631846F7F73FFF034680
S31508028650022B7FD17B6803F5C0631A78674B1B78B8
S31508028660D31A002B34D17B6803F5C0631846F7F793
S315080286702DFF0346012B2BD17B6803F500631846B1
S3150802868065F087F978617B69002B1EDDF8F75AFEDB
S31508028690034600211846F8F791FEF8F753FE0346FB
S315080286A004211846F8F7E4FEF8F74CFE03460121C2
S315080286B01846F8F7F8FEF8F745FE02467B69DBB27C
S315080286C019461046F8F715FF43E0F9F7FBFDFCE0FB
S315080286D07B6803F5C0631A78494B1B78D31A002BBB
S315080286E034D17B6803F5C0631846F7F7EFFE0346F5
S315080286F0012B2BD17B6803F50063184665F049F90F
S3150802870078617B69002B1EDDF8F71CFE0346002103
S315080287101846F8F753FEF8F715FE034604211846DD
S31508028720F8F7A6FEF8F70EFE034602211846F8F7F2
S31508028730BAFEF8F707FE02467B69DBB2194610460F
S31508028740F8F7D7FE05E0F9F7BDFDBEE0F9F7BAFD81
S31508028750BBE0A0E07B6803F580631A782A4B1B7896
S31508028760D31A002B40F094807B6803F58063184681
S31508028770F7F7ACFE0346012B40F08A807B6803F5C7
S31508028780C0631A781D4B1B78D31A002B3ED17B681F
S3150802879003F5C0631846F7F799FE0346012B35D150
S315080287A07B6803F50063184665F0F3F878617B6920
S315080287B0002B1EDDF8F7C6FD034600211846F8F71A
S315080287C0FDFDF8F7BFFD034605211846F8F750FEEA
S315080287D0F8F7B8FD034601211846F8F764FEF8F7DC
S315080287E0B1FD02467B69DBB219461046F8F781FEEF
S315080287F04DE0F9F767FD68E0D8440908EC33090843
S3150802880004340908DC440908D82909087B6803F5F1
S31508028810C0631A782E4B1B78D31A002B34D17B6887
S3150802882003F5C0631846F7F751FE0346012B2BD111
S315080288307B6803F50063184665F0ABF878617B69D7
S31508028840002B1EDDF8F77EFD034600211846F8F7D1
S31508028850B5FDF8F777FD034605211846F8F708FE31
S31508028860F8F770FD034602211846F8F71CFEF8F7DA
S3150802887069FD02467B69DBB219461046F8F739FEEE
S3150802888005E0F9F71FFD20E0F9F71CFD1DE002E0FF
S31508028890F9F718FD19E018E07B6803F500731A78F2
S315080288A00C4B1B78D31A002B0CD17B6803F500738B
S315080288B01846F7F70BFE0346012B03D106482CF0A0
S315080288C05DFA02E0F9F7FEFC00BF1837BD4680BD27
S315080288D004340908E0440908E444090890B599B043
S315080288E000AFF8600B467A60FB720023FB6558F00E
S315080288F06DFCB86507F11403184659F0BEFC044628
S3150802890007F11403184659F0C4FC03461A462146D1
S31508028910B86D4BF041FE0023FB650BE064203BF08B
S3150802892057FFF9F755FC034618462CF007FCFB6D72
S315080289300133FB65FB6D3B2BF0D907F1140318468F
S3150802894059F09BFC044607F11403184659F0A1FC9A
S3150802895003461A462146B86D4BF01EFE0023FB65F8
S315080289600BE064203BF034FFF9F732FC0346184665
S315080289702CF0E4FBFB6D0133FB65FB6D3B2BF0D959
S3150802898000BF00BF6437BD4690BD000090B585B0F4
S3150802899000AFF8600B467A60FB727B6803F50073DA
S315080289A00522CD49184666F03DF90346002B17D134
S315080289B07B6803F500731846F7F788FD0346052B0F
S315080289C00ED128F0D3FA03460021184628F0E6FA13
S315080289D00346184628F0F0FBC0482CF0CFF977E199
S315080289E07B6803F500730322BD49184666F01AF937
S315080289F00346002B19D17B6803F500731846F7F76F
S31508028A0065FD0346032B10D128F0B0FA0346002170
S31508028A10184628F0C3FA0346184628F0C1FB03464F
S31508028A201946B0482CF0AAF952E17B6803F500739F
S31508028A300422AD49184666F0F5F80346002B40F0C5
S31508028A4043817B6803F500731846F7F73FFD034633
S31508028A50042B40F0398128F089FA0346002118468A
S31508028A6028F09CFA0346184628F09AFB0346002B80
S31508028A7000F0BE8028F07AFA03460021184628F04C
S31508028A808DFA044647F010FC03461946204628F09C
S31508028A90CDFE03461A46954B1A7028F067FA034626
S31508028AA00021184628F07AFA044647F0FDFB0346E9
S31508028AB01946204628F0ECFE03461A468C4B1A70D5
S31508028AC028F054FA03460021184628F067FA0446A5
S31508028AD047F0EAFB03461946204628F00BFF0346F1
S31508028AE01A46844B1A7028F041FA034600211846A2
S31508028AF028F054FA044647F0D7FB0346194620469F
S31508028B0028F02AFF03461A467B4B1A7028F02EFADB
S31508028B1003460021184628F041FA0346184628F06B
S31508028B203FFB0346194675482CF028F96F4B1B780C
S31508028B301C4647F0B9FB0346184647F031FC034684
S31508028B40184658F04CFF0346184628F045FB0346DC
S31508028B501A4621466A482CF081F9654B1B781C4651
S31508028B6047F0A2FB0346184647F09DFC0246604BB7
S31508028B701B78013BDBB2194610465FF049FC0346F7
S31508028B80184628F05BFC03461A4621465D482CF037
S31508028B9065F9584B1B781C4647F086FB0346184670
S31508028BA047F039FC0346184657F023FB0346184696
S31508028BB028F054FD03461A46214653482CF04EF92E
S31508028BC04D4B1B781C4647F06FFB0346184647F089
S31508028BD05EFC034618465EF04DFA0346184628F030
S31508028BE0B1FD03461A46214648482CF0C7F86FE0FD
S31508028BF03E4B00221A703E4B00221A703D4B002251
S31508028C001A703D4B00221A7028F0B0F9034600216B
S31508028C10184628F0C3F90346184628F0C1FA03464F
S31508028C20194636482CF0AAF847F03EFB0346184682
S31508028C3047F0B6FB0346184658F0D1FE03461846D7
S31508028C4028F0CAFA0346194631482CF007F947F0C4
S31508028C502BFB0346184647F026FC0246244B1B7894
S31508028C60194610465FF0D4FB0346184628F0E6FB81
S31508028C700346194627482CF0F1F847F015FB034638
S31508028C80184647F0C8FB0346184657F0B2FA034699
S31508028C90184628F0E3FC034619461F482CF0DEF86E
S31508028CA047F002FB0346184647F0F1FB034618460F
S31508028CB05EF0E0F90346184628F044FD03461946D5
S31508028CC016482CF05BF803E015482CF057F800BF5D
S31508028CD000BF1437BD4690BD184509082045090846
S31508028CE0344509083845090850450908D4190120A8
S31508028CF0D5190120D6190120D71901205845090886
S31508028D00704509088045090890450908A0450908DB
S31508028D10B0450908C0450908D0450908E0450908CB
S31508028D20F045090890B585B000AF78600023BB739B
S31508028D300023FB734FF4A0520021204865F06AFF16
S31508028D4007F10E030A221D49786856F055FE0346B6
S31508028D50012B2ED10023FB7328E0FA7B13461B0155
S31508028D609B1ADB00164A13449C1C1448F7F7AEFB01
S31508028D7003461A461149204665F054FF0346002B5E
S31508028D8011D1FA7B0E4913461B019B1ADB000B44D1
S31508028D9014331B68B97B094A0020984709482BF007
S31508028DA0EDFF012306E0FB7B0133FB73FB7B102BF4
S31508028DB0D3D9002318461437BD4690BDC4FF0020F8
S31508028DC0040000203C25090880B582B000AF03469E
S31508028DD0FB71FB790D2B24D14C4B00221A704C489F
S31508028DE02CF03CF84B4B1B78002B16D04A48FFF761
S31508028DF099FF0346012B08D140220021474865F016
S31508028E0009FF4549454865F0A6FF424B00221A70FC
S31508028E1040220021404865F0FDFE41482CF01EF82C
S31508028E206FE0FB790A2B03D1384B00221A7068E0EF
S31508028E30FB791B2B03D1354B01221A7061E0FB79B2
S31508028E405B2B07D1314B1B78012B03D12F4B022207
S31508028E501A7056E0FB79412B1FD12C4B1B78022B3B
S31508028E601BD12A4B00221A702A4B1B78002B48D199
S31508028E702A492C482BF0F2FF2848F7F727FB034626
S31508028E80DAB2244B1A7040220021234865F0C2FE4A
S31508028E902249214865F05FFF33E0FB79082B02D0AF
S31508028EA0FB797F2B16D1194B00221A70194B1B78A6
S31508028EB0002B26D0174B1B78013BDAB2154B1A70DA
S31508028EC0144B1B781A46144B0021995416482BF05A
S31508028ED0C5FF16E00F4B1B785A1CD1B20D4A11700A
S31508028EE019460D4AFB7953540A4B1B7803F03F0384
S31508028EF0DAB2084B1A70FB7919460C482BF0AEFF0A
S31508028F00FFE700BF0837BD4680BD00BFD81901205C
S31508028F103C2509084414012004140120C413012025
S31508028F2008460908342509080C460908104609089E
S31508028F3080B500AF1C2301224A494B483CF0F2FA9D
S31508028F401C23012249494A483CF0ECFA1C23012217
S31508028F50484949483CF0E6FA1C2301224749484851
S31508028F603CF0E0FA1C230122464947483CF0DAFA6B
S31508028F701C230122454946483CF0D4FA1C23012207
S31508028F80444945483CF0CEFA1C2301224349444849
S31508028F903CF0C8FA1C230122424943483CF0C2FA73
S31508028FA01C230122414942483CF0BCFA1C230122F7
S31508028FB0404941483CF0B6FA1C2301223F49404841
S31508028FC03CF0B0FA1C2301223E493F483CF0AAFA7B
S31508028FD01C2301223D493E483CF0A4FA1C230122E7
S31508028FE03C493D483CF09EFA1C2301223B493C4839
S31508028FF03CF098FA1C2301223A493B483CF092FA83
S315080290001C23012239493A483CF08CFA1C230122D6
S31508029010384939483CF086FA1C2301223749384830
S315080290203CF080FA1C230122364937483CF07AFA8A
S315080290301C230122354936483CF074FA1C230122C6
S31508029040344935483CF06EFA1C2301223349344828
S315080290503CF068FA1C230122324933483CF062FA92
S3150802906000BF80BD1C460908A81A01203046090817
S31508029070C41A012048460908E01A0120644609086C
S31508029080FC1A01207C460908181B01209446090887
S31508029090341B0120B0460908501B0120D046090896
S315080290A06C1B0120F4460908881B01201047090891
S315080290B0A41B012024470908C01B012044470908AC
S315080290C0DC1B012060470908F81B012078470908BC
S315080290D0141C012094470908301C0120A8470908D6
S315080290E04C1C0120C0470908681C0120D8470908FA
S315080290F0841C0120F0470908A01C01200848090819
S31508029100BC1C012028480908D81C01204048090827
S31508029110F41C012060480908101D0120804809082E
S315080291202C1D0120A0480908481D012080B58EB0D3
S3150802913008AF786000237B617B683B6107F10C010D
S3150802914000234FF47A6238693CF0D8F80346002BBC
S3150802915001D0022332E0FB68B02206920122059270
S31508029160002204920A2203920A2202924FF47A6297
S31508029170019200930023134A134914483CF0C8FA93
S315080291800346002B01D00E2318E01C2300221049A7
S3150802919010483CF0C7F90346002B01D00C230DE01A
S315080291A006220F210C482BF01BFF0C482BF0E6FD7C
S315080291B07868F8F749FBFFF7BBFE7B69184618374C
S315080291C0BD4680BDE1910208C4480908DC190120A0
S315080291D0D44809088C1A0120E8480908F8480908F9
S315080291E02DE9F0418AB002AF78607B68FB60002304
S315080291F0FB770023BB8300237B8300237B76002334
S315080292003B760023FB750023BB8200237B82B5488D
S315080292102BF0B4FDB449B5482BF0B0FDB449B548B6
S315080292202BF0ACFDB4482BF0A9FD0021B3482BF076
S31508029230A5FD0121B2482BF0A1FD1DF0A5FB0346B1
S3150802924018461DF0C6FD03461846F8F791FE034672
S315080292501946AC482BF092FD1DF096FB03461846BC
S315080292601DF0B7FD03461846F8F78FFE0346194662
S31508029270A5482BF083FDA5482BF080FDF8F71CF8CE
S3150802928003461846F8F73CF8A14B1B780133DAB2C5
S315080292909F4B1A709E4B1B78092B09D99C4B0022AF
S315080292A01A702BF073FF4FF400519A4830F034FBD2
S315080292B01DF06AFB034618461DF0E7FC0346092B18
S315080292C036D1FB7F022B1AD0022B00F37682002BB3
S315080292D002D0012B05D070E210F036FF0123FB778E
S315080292E078E2BB8B5A1CBA83042B40F268820023AD
S315080292F0BB830223FB7788482BF040FD5FE210F020
S3150802930073FA0346184610F089FB0346012B40F010
S31508029310588210F02FFF81482BF030FD0023FB778F
S315080293201DF032FB0346002118461DF09BFC48E25D
S315080293301DF02AFB034618461DF0A7FC0346012B1F
S3150802934045D14FF48061764830F0B6FA0346012BD0
S315080293500CBF01230023DBB21C460821714830F0FA
S31508029360ABFA0346012B0CBF01230023DBB21D46D1
S3150802937080216D4830F0A0FA0346012B14BF012361
S315080293800023DBB21E460221664830F095FA0346F0
S31508029390012B14BF01230023DBB2009333462A466E
S315080293A0214662482BF0EAFC7B8B5A1C7A83132BE4
S315080293B040F210821DF0E8FA0346002118461DF015
S315080293C051FC00237B835A482BF0D8FC02E21DF09D
S315080293D0DBFA034618461DF058FC0346022B50D109
S315080293E00821544830F068FA0346012B0CBF0123C2
S315080293F00023DBB21D4604214E4830F05DFA0346CF
S31508029400012B0CBF01230023DBB21E460221494869
S3150802941030F052FA0346012B0CBF01230023DBB2BC
S3150802942098460121434830F047FA0346012B0CBF00
S3150802943001230023DBB21C4610213B4830F03CFADC
S315080294400346012B0CBF01230023DBB201930094D0
S3150802945043463246294638482BF090FC7B8B5A1CE9
S315080294607A83132B40F2B6811DF08EFA0346002149
S3150802947018461DF0F7FB00237B832D482BF07EFC54
S31508029480A8E11DF081FA034618461DF0FEFB0346C5
S31508029490032B67D13B7E01333B767B7E012B00F2A1
S315080294A099813B7E322B02D811F0ECFE8BE13B7E92
S315080294B0312B05D93B7E372B02D811F0F9FE50E045
S315080294C03B7E362B05D93B7E692B02D811F00EFF5F
S315080294D047E03B7E682B31D93B7E9B2B2ED811F079
S315080294E01BFF3EE01049090838490908404909089E
S315080294F0504909085C490908744909089C49090838
S31508029500B8490908C8490908E4490908004A09087E
S31508029510641D012000080242284A0908384A090837
S31508029520000C02420018024200100242484A090888
S315080295307C4A0908001402428C4A09083B7E9B2B86
S3150802954040F24181A8482BF019FC00233B76002300
S315080295507B761DF019FA0346002118461DF082FB98
S3150802956031E130E11DF010FA034618461DF08DFB75
S315080295700346042B27D1F7F79FFE03460021184618
S31508029580F7F7CEFE0446F7F797FE03460421184678
S31508029590F7F7C6FE0546F7F78FFE0346012118467A
S315080295A0F7F7BEFE0646F7F787FE03460321184677
S315080295B0F7F7B6FE0346009333462A4621468B48FA
S315080295C02BF0DCFB06E11DF0DFF9034618461DF019
S315080295D05CFB0346052B40F0FD807B8A01337B82C8
S315080295E0FB7D022B4ED0022B00F3EF80002B02D01C
S315080295F0012B38D0E9E080217D4830F05DF9034639
S31508029600012B13D17B4B1B6800229A63794B1B688B
S3150802961064225A630021774836F0C2FB0421754852
S3150802962036F01EFD74481EF005F919E0022173484A
S3150802963030F042F90346012B12D16E4B1B686422A5
S315080296409A636C4B1B6800225A630021694836F0FC
S3150802965007FD0421674836F0A3FB69481EF0EAF8BD
S315080296600123FB75B6E0BB8A0133BB82BB8A132B87
S3150802967040F2AD800023BB820223FB7561481EF0CF
S31508029680D9F8A4E080215A4830F016F90346012B8E
S3150802969029D1584B1B6800229A63564B1B68002235
S315080296A05A630021534836F0DBFC0421514836F050
S315080296B0D7FC0023FB7554481EF0BCF81DF064F96C
S315080296C00346002118461DF0CDFA1DF05DF9034642
S315080296D018461DF09AFB03460221184610F074F844
S315080296E000237B822FE00221444830F0E5F8034646
S315080296F0012B28D13F4B1B6800229A633D4B1B68FE
S3150802970000225A6300213B4836F0AAFC0421394854
S3150802971036F0A6FC0023FB753C481EF08BF81DF0BC
S3150802972033F90346002118461DF09CFA1DF02CF960
S31508029730034618461DF069FB03460321184610F036
S3150802974043F800237B827B8A632B42D900237B82E0
S315080297502F481EF06FF80221284830F0ADF803466C
S31508029760012B0BD11DF010F9034618461DF04DFBCF
S3150802977003460321184610F027F82AE080211C48E0
S3150802978030F09AF80346012B0BD11DF0FDF803467B
S3150802979018461DF03AFB03460221184610F014F843
S315080297A017E01DF0F1F8034618461DF02EFB034696
S315080297B00021184610F008F80BE000BF0AE000BFC7
S315080297C008E000BF06E000BF04E000BF02E000BFF9
S315080297D000E000BFFB68DBB218462BF0AFFC642042
S315080297E03AF0F6FF50E500BFC84A0908DC4A0908FC
S315080297F000100242D46C0120184B090800180242D4
S31508029800304B0908484B0908644B0908744B090888
S31508029810844B090880B500AF3AF07AFC00BF80BDD8
S3150802982080B586B004AF00237B601DF0ADF8034611
S3150802983018461DF0CEFA03461846F8F753FC786028
S31508029840002000F0FFF802467B68029301924FF46B
S3150802985000730093054B4FF48072044904483CF0A8
S315080298607DF800BF0837BD4680BD00BF000C024226
S315080298706C1D012080B582B000AF0346FB71FB79EF
S31508029880002B04D104483CF09DF8034600E000236F
S3150802989018460837BD4680BD6C1D012080B582B0CA
S315080298A000AF03460A46FB711346BB71FB79002BD0
S315080298B006D1BB79194605483CF0D6F8034600E0BE
S315080298C0002318460837BD4680BD00BF6C1D01201F
S315080298D080B582B000AF0346FB71FB79002B07D136
S315080298E0002000F0AFF80346194603483CF0DFF8BB
S315080298F000BF0837BD4680BD6C1D012080B584B007
S3150802990000AF0346FB710023FB60FB79002B0BD1EA
S3150802991005210020FFF7C2FFF860F968002000F071
S31508029920A5F80020FFF7D4FF00BF1037BD4680BD5B
S3150802993080B586B000AF0346FB714FF000037B612A
S315080299404FF000033B614FF00003FB604FF000034A
S31508029950BB60FB79002B29D10020FFF78BFF07EEAE
S31508029960900AF8EEE77AC7ED047A002000F06AF862
S3150802997007EE900AF8EEE77AC7ED037A1DF004F8C7
S31508029980034618461DF025FA03461846F8F7AAFBB9
S3150802999007EE900AF8EEE77AC7ED027AD7ED027A71
S315080299A0F5EE407AF1EE10FA14D002E04FF0000319
S315080299B014E097ED047AD7ED037A77EE676A97EDA6
S315080299C0027AC6EE877A9FED097A67EE877AC7ED3D
S315080299D0057A02E04FF000037B617B6907EE903A55
S315080299E0B0EE670A1837BD4680BD00BF000048437F
S315080299F090B585B000AF0346FB710023FB60FB7987
S31508029A00002B19D11E210020FFF748FF044600202B
S31508029A1000F018F80346E31AFB601CF0B5FF03468C
S31508029A2018461DF0D6F90346F9681846F8F74BFBAF
S31508029A30F96803482BF0A2F900BF1437BD4690BD5A
S31508029A40AC4B090880B483B000AF0346FB71FB79BF
S31508029A50002B02D1044B1B6800E0002318460C3782
S31508029A60BD465DF8047B7047681D012080B483B04B
S31508029A7000AF03463960FB71FB79002B02D1044A19
S31508029A803B68136000BF0C37BD465DF8047B704720
S31508029A90681D0120B0B582B002AF1CF075FF0446FE
S31508029AA0F7F70AFC034601211846F7F739FC03467D
S31508029AB09BB2184601F004FB0346DBB21946204660
S31508029AC01DF06EFA1CF060FF0446F7F7F5FB034635
S31508029AD001211846F7F724FC03469BB2194620468D
S31508029AE01DF080FA1CF050FF0446F7F7E5FB034623
S31508029AF003211846F7F714FC03469BB2184601F0F1
S31508029B00DFFA0346DBB2194620461DF09BF91CF024
S31508029B103BFF0446F7F7D0FB034603211846F7F73F
S31508029B20FFFB03469BB2194620461DF0ADF9634B6F
S31508029B301B8801339AB2614B1A80604B1B88B3F5B6
S31508029B407A7F2FD35D4B00221A80F7F7B5FB0346BF
S31508029B5003211846F7F7E4FB03469BB2184601F0C1
S31508029B6043FA10EE103A1846F6F71CFE04460D465E
S31508029B70F7F7A2FB034601211846F7F7D1FB03467E
S31508029B809BB2184601F030FA10EE103A1846F6F76C
S31508029B9009FE02460B46CDE9002322462B464848D3
S31508029BA01DF048FEF7F788FB034601211846F7F72A
S31508029BB0B7FB03469BB2184601F016FAF0EE407A56
S31508029BC0B1EE087AF4EEC77AF1EE10FA05D83D4BF3
S31508029BD01B8801339AB23B4B1A803B4B1B880133D5
S31508029BE09AB2394B1A80384B1B8840F6B7329342E1
S31508029BF02AD9344B1B8840F6533293420DD95FF06B
S31508029C004FFF0123D3220B211CF076FA2D4B1B881A
S31508029C1019462E481DF00EFE10E02A4B1B88952B7E
S31508029C200CD95FF03DFF01236F220B211CF064FA69
S31508029C30244B1B88194626481DF0FCFD214B0022A1
S31508029C401A80214B00221A80224B1B8801339AB2B2
S31508029C50204B1A801F4B1B8840F6B73293422AD9EB
S31508029C601D4B1B8840F6533293420DD95FF018FFFD
S31508029C700123C9220B211CF03FFA174B1B881946F0
S31508029C8016481DF0D7FD10E0134B1B88952B0CD9EF
S31508029C905FF006FF012365220B211CF02DFA0E4BFD
S31508029CA01B8819460E481DF0C5FD0B4B00221A806B
S31508029CB0084B00221A8000BFBD46B0BD901D012088
S31508029CC0D04B09088C1D0120881D0120004C09086B
S31508029CD0384C09088A1D01208E1D0120704C09087E
S31508029CE0A84C090880B582B000AF78601CF04CFE1B
S31508029CF0034618461DF02AFD034618464EF039FB60
S31508029D000346022B21D11CF03FFE034618461DF0DE
S31508029D10F3FC034618464DF065FD0346012B11D1A7
S31508029D208E482BF02BF88E481DF084FD1CF02CFE75
S31508029D30034618461DF00AFD0346012118464EF051
S31508029D4024FB22E010F07EFA04E11CF01DFE034615
S31508029D5018461DF0D1FC034618464DF043FD03464E
S31508029D60022B12D17F481DF065FD10F053FA10F050
S31508029D7069FA1CF009FE034618461DF0E7FC03467D
S31508029D80022118464EF001FBE4E01AF0F3FC034602
S31508029D90012118461AF01CFD0346002B13D11AF0AE
S31508029DA0E9FC0346252118461AF012FD0346002B44
S31508029DB009D11AF0DFFC0346282118461AF008FDD5
S31508029DC00346002B04D010F025FA10F03BFAC1E046
S31508029DD01CF0DAFD034618461DF0D3F80346782B25
S31508029DE009D95FF05DFE01230B220B211CF084F9D1
S31508029DF010F028FAAEE01CF0C7FD034618461DF01F
S31508029E0012F80346782B09D95FF04AFE012301228C
S31508029E100B211CF071F910F0FDF99BE001F02CF80A
S31508029E20514BD3E900014FF00002504BF6F75CFBA9
S31508029E3002460B464C49C1E900234D4BD3E90001C2
S31508029E404FF00002494BF6F74FFB02460B464849CC
S31508029E50C1E90023444BD3E90001464BD3E9002369
S31508029E60F6F774FF0346002B02D010F0DFF90CE078
S31508029E703D4BD3E900013F4BD3E90023F6F77AFFBE
S31508029E800346002B01D010F0DDF9394BD3E9000166
S31508029E90394BD3E90023F6F759FF0346002B02D0C4
S31508029EA010F0ACF90CE0324BD3E90001324BD3E99E
S31508029EB00023F6F75FFF0346002B01D010F0AAF93C
S31508029EC0294BD3E900014FF000022C4BF6F748FF65
S31508029ED00346002B19D01CF057FD034618461DF001
S31508029EE072F80346184600F04BF803461846F6F78A
S31508029EF037FC02460B461F49C1E900231A494FF0AF
S31508029F0000024FF00003C1E90023194BD3E900010F
S31508029F104FF00002194BF6F723FF0346002B19D020
S31508029F201CF032FD034618461CF09FFF03461846EE
S31508029F3000F0DEFB03461846F6F712FC02460B460D
S31508029F400D49C1E900230A494FF000024FF0000308
S31508029F50C1E900230837BD4680BD00BFE04C0908A9
S31508029F60304D0908404D0908981D01200000F03FB0
S31508029F70A01D0120A81D0120B01D01200000494096
S31508029F80B0B52DED028B84B000AF0346FB800023EB
S31508029F90FB731CF0F9FC034618461DF036F8034617
S31508029FA0002B1CD0FB88184601F08AF803461C468B
S31508029FB01CF0EAFC034618461DF0ACFB034618469D
S31508029FC04DF093FF0346053B9C4205DAC84B002237
S31508029FD01A700123FB735DE00423FB735AE0C44B3A
S31508029FE000221A70FB88184601F06AF803461C46D6
S31508029FF01CF0CAFC034618461DF08CFB034618469D
S3150802A0004DF073FF0346053B9C4202DA0123FB73BC
S3150802A01040E0FB88184601F053F803461C461CF03C
S3150802A020B3FC034618461DF075FB034618464DF069
S3150802A0305CFF0346053B9C4216DBFB88184601F08B
S3150802A0403FF803461C461CF09FFC034618461DF0C3
S3150802A05061FB034618464DF048FF0346013B9C4206
S3150802A06002DA0223FB7315E0FB88184601F028F88A
S3150802A07003461C461CF088FC034618461DF04AFB9C
S3150802A080034618464DF031FF0346013B9C4201DB6D
S3150802A0900323FB73974B1B78FA7B9A420BD0954A9C
S3150802A0A0FB7B1370944B00221A70FB7B022B02D1A6
S3150802A0B0924B0A221A70FB7B013B032B00F2FD82AC
S3150802A0C001A252F823F000BFD9A00208E1A00208B3
S3150802A0D005A2020831A50208884B32221A70F5E257
S3150802A0E0854B1B780133DAB2834B1A70834B1B7884
S3150802A0F0312B22D8FB88184600F076FF10EE103A6C
S3150802A1001846F6F74FFB04460D467D4B1B88184644
S3150802A11000F06AFF10EE103A1846F6F743FB72A3F0
S3150802A120D3E90023F6F7DEF902460B46204629460E
S3150802A130F6F702FE0346002B2CD0FB88184600F0E1
S3150802A14053FF10EE103A1846F6F72CFB04460D4656
S3150802A1506B4B1B88184600F047FF10EE103A18465C
S3150802A160F6F720FB60A3D3E90023F6F7BBF902460C
S3150802A1700B4620462946F6F7DFFD0346002B09D093
S3150802A1805E4B32221A705C4B00221A705C4AFB88BC
S3150802A19013809BE2FB88184600F026FF10EE103A61
S3150802A1A01846F6F7FFFA04460D46554B1B8818461D
S3150802A1B000F01AFF10EE103A1846F6F7F3FA4AA319
S3150802A1C0D3E90023F6F790F902460B4620462946BC
S3150802A1D0F6F7D0FD0346002B05D0484B05221A7028
S3150802A1E0474AFB881380444B1B78022B40F269824C
S3150802A1F0414B00221A70414B1B780533DAB23F4BAA
S3150802A2001A705EE23C4B1B780133DAB23A4B1A708B
S3150802A210FB88184600F054FF03461C461CF0B4FBA4
S3150802A220034618461DF076FA034618464DF05DFEBB
S3150802A23003469C4203D9314B00221A7043E2FB883B
S3150802A240184600F0D1FE10EE103A1846F6F7AAFAAA
S3150802A25004460D461CF098FB034618461DF05AFAAA
S3150802A260034618464DF041FE03461846F6F788FAA5
S3150802A2701DA3D3E90023F6F737F902460B46204613
S3150802A2802946F6F76DFD0346002B6CD0FB88184667
S3150802A29000F0AAFE10EE103A1846F6F783FA0446BC
S3150802A2A00D461CF071FB034618461DF033FA0346A9
S3150802A2B018464DF01AFE03461846F6F761FA4FF0AD
S3150802A2C00002104BF6F710F902460B4620462946BD
S3150802A2D0F6F750FD0346002B16D0084B01221A70DA
S3150802A2E0F1E100BFAFF300809A9999999999C93F0C
S3150802A2F0B81D0120B91D0120BA1D0120BB1D012070
S3150802A300BC1D01200000E03FFB88184600F06CFEE9
S3150802A31010EE103A1846F6F745FA04460D461CF0B2
S3150802A32033FB034618461DF0F5F9034618464DF069
S3150802A330DCFD03461846F6F723FA4FF00002C24B35
S3150802A340F6F7D2F802460B4620462946F6F7F4FCFB
S3150802A3500346002B03D0BD4B02221A70B3E1BB4B56
S3150802A36000221A70AFE1FB88184600F03DFE10EE97
S3150802A370103A1846F6F716FA04460D461CF004FB80
S3150802A380034618461DF0C6F9034618464DF0ADFDBC
S3150802A39003461846F6F7F4F9A7A3D3E90023F6F716
S3150802A3A0A3F802460B4620462946F6F7C5FC03469D
S3150802A3B0002B00D187E1FB88184600F015FEB0EEA7
S3150802A3C0408A1CF0E1FA034618461DF0A3F9034633
S3150802A3D018464DF08AFD034607EE903AF8EEE77AFC
S3150802A3E0B4EEE78AF1EE10FA4ED5FB88184600F06D
S3150802A3F0FBFD10EE103A1846F6F7D4F904460D4658
S3150802A400934B1B88184600F0EFFD10EE103A1846DB
S3150802A410F6F7C8F988A3D3E90023F6F765F80246E2
S3150802A4200B4620462946F6F7A5FC0346002B06D01E
S3150802A430864B00221A70864AFB88138061E0FB88E5
S3150802A440184600F0D1FDF0EE407AB2EE047A67EED5
S3150802A450877AFCEEE77A17EE903A9CB27C4B1B8819
S3150802A460184600F0C1FDF0EE407AB2EE047A67EEC5
S3150802A470877AFCEEE77A17EE903A9BB29C4240D274
S3150802A480734AFB8813803CE0FB88184600F0ACFD53
S3150802A490B0EE408A6E4B1B88184600F0A5FDF0EE1A
S3150802A4A0407AB4EEE78AF1EE10FA06DD674B00222F
S3150802A4B01A70674AFB88138023E0FB88184600F067
S3150802A4C093FDF0EE407AB2EE047A67EE877AFCEEF6
S3150802A4D0E77A17EE903A9CB25D4B1B88184600F055
S3150802A4E083FDF0EE407AB2EE047A67EE877AFCEEE6
S3150802A4F0E77A17EE903A9BB29C4202D2544AFB88FC
S3150802A5001380544B1B78042B40F2DD80514B0022FA
S3150802A5101A704E4B1B780E2B03D94C4B0F221A700E
S3150802A520D1E04A4B1B780533DAB2484B1A70CAE0B7
S3150802A530FB88184600F0C4FD03461C461CF024FAA4
S3150802A540034618461DF0E6F8034618464DF0CDFCBC
S3150802A55003469C420AD33D4B00221A701CF014FA99
S3150802A5600346002118461CF05FFDAFE0FB8818463B
S3150802A57000F03AFD10EE103A1846F6F713F90446BB
S3150802A5800D46334B1B88184600F02EFD10EE103A86
S3150802A5901846F6F707F92AA3D3E90023F5F7A4FF25
S3150802A5A002460B4620462946F6F7E4FB0346002BED
S3150802A5B009D0264B00221A70254AFB881380264B9F
S3150802A5C000221A7029E0FB88184600F00DFDF0EE0D
S3150802A5D0407AB2EE047A67EE877AFCEEE77A17EEED
S3150802A5E0903A9CB21A4B1B88184600F0FDFCF0EE16
S3150802A5F0407AB2EE047A67EE877AFCEEE77A17EECD
S3150802A600903A9BB29C4208D2114AFB881380124B9D
S3150802A6101B780133DAB2104B1A700F4B1B78012BD9
S3150802A6201CD90D4B1B78032B18D8084B0F221A700E
S3150802A6304CE000BFAFF300809A9999999999B93F6E
S3150802A6409A9999999999C93F0000E03FBB1D012043
S3150802A650BC1D0120BA1D0120B81D01201F4B1B7805
S3150802A660032B03D91E4B32221A702FE01D4B1B787F
S3150802A6700133DAB21B4B1A701A4B1B78022B03D121
S3150802A680174B32221A7020E0164B1B78022B1CD964
S3150802A690144B1B78062B18D9124B02221A70104B30
S3150802A6A01B78312B02D90E4B00221A700C4B1B78E1
S3150802A6B00533DAB20A4B1A7007E00B482AF05EFB3A
S3150802A6C004E000BF02E000BF00E000BF044B1B78B5
S3150802A6D018461037BD46BDEC028BB0BDB81D012029
S3150802A6E0BB1D0120BA1D0120504D090800000000BB
S3150802A6F0B0B52DED028B84B000AF0346FB80002374
S3150802A700FB731CF041F9034618461CF0D0FB0346BE
S3150802A710002B1CD0FB88184600F0D2FC03461C46C8
S3150802A7201CF032F9034618461CF0F4FF0346184695
S3150802A7304DF0DBFB0346053B9C4205DAC84B00227B
S3150802A7401A700123FB735DE00423FB735AE0C44BC2
S3150802A75000221A70FB88184600F0B2FC03461C4613
S3150802A7601CF012F9034618461CF0D4FF0346184695
S3150802A7704DF0BBFB0346053B9C4202DA0123FB7301
S3150802A78040E0FB88184600F09BFC03461C461CF07A
S3150802A790FBF8034618461CF0BDFF034618464DF063
S3150802A7A0A4FB0346053B9C4216DBFB88184600F0D1
S3150802A7B087FC03461C461CF0E7F8034618461CF0BD
S3150802A7C0A9FF034618464DF090FB0346013B9C42FF
S3150802A7D002DA0223FB7315E0FB88184600F070FCC8
S3150802A7E003461C461CF0D0F8034618461CF092FF96
S3150802A7F0034618464DF079FB0346013B9C4201DBB2
S3150802A8000323FB73974B1B78FA7B9A420BD0954A24
S3150802A810FB7B1370944B00221A70FB7B022B02D12E
S3150802A820924B0A221A70FB7B013B032B00F2FD8234
S3150802A83001A252F823F000BF49A8020851A802084B
S3150802A84075A90208A1AC0208884B32221A70F5E2F1
S3150802A850854B1B780133DAB2834B1A70834B1B780C
S3150802A860312B22D8FB88184600F0BEFB10EE103AB0
S3150802A8701846F5F797FF04460D467D4B1B88184682
S3150802A88000F0B2FB10EE103A1846F5F78BFF72A3EA
S3150802A890D3E90023F5F726FE02460B46204629464B
S3150802A8A0F6F74AFA0346002B2CD0FB88184600F026
S3150802A8B09BFB10EE103A1846F5F774FF04460D4650
S3150802A8C06B4B1B88184600F08FFB10EE103A1846A1
S3150802A8D0F5F768FF60A3D3E90023F5F703FE0246FE
S3150802A8E00B4620462946F6F727FA0346002B09D0D7
S3150802A8F05E4B32221A705C4B00221A705C4AFB8845
S3150802A90013809BE2FB88184600F06EFB10EE103AA5
S3150802A9101846F5F747FF04460D46554B1B88184659
S3150802A92000F062FB10EE103A1846F5F73BFF4AA311
S3150802A930D3E90023F5F7D8FD02460B4620462946F9
S3150802A940F6F718FA0346002B05D0484B05221A706B
S3150802A950474AFB881380444B1B78022B40F26982D4
S3150802A960414B00221A70414B1B780533DAB23F4B32
S3150802A9701A705EE23C4B1B780133DAB23A4B1A7014
S3150802A980FB88184600F09CFB03461C461BF0FCFF9E
S3150802A990034618461CF0BEFE034618464DF0A5FAB5
S3150802A9A003469C4203D9314B00221A7043E2FB88C4
S3150802A9B0184600F019FB10EE103A1846F5F7F2FEA3
S3150802A9C004460D461BF0E0FF034618461CF0A2FE9D
S3150802A9D0034618464DF089FA03461846F5F7D0FE9F
S3150802A9E01DA3D3E90023F5F77FFD02460B46204651
S3150802A9F02946F6F7B5F90346002B6CD0FB881846AC
S3150802AA0000F0F2FA10EE103A1846F5F7CBFE0446B5
S3150802AA100D461BF0B9FF034618461CF07BFE03469B
S3150802AA2018464DF062FA03461846F5F7A9FE4FF0A6
S3150802AA300002104BF5F758FD02460B4620462946FA
S3150802AA40F6F798F90346002B16D0084B01221A701E
S3150802AA50F1E100BFAFF300809A9999999999C93F94
S3150802AA60BE1D0120BF1D0120C01D0120C11D0120E0
S3150802AA70C21D01200000E03FFB88184600F0B4FA28
S3150802AA8010EE103A1846F5F78DFE04460D461BF0F1
S3150802AA907BFF034618461CF03DFE034618464DF05A
S3150802AAA024FA03461846F5F76BFE4FF00002C24B2E
S3150802AAB0F5F71AFD02460B4620462946F6F73CF9F3
S3150802AAC00346002B03D0BD4B02221A70B3E1BB4BDF
S3150802AAD000221A70AFE1FB88184600F085FA10EEDC
S3150802AAE0103A1846F5F75EFE04460D461BF04CFF73
S3150802AAF0034618461CF00EFE034618464DF0F5F9B5
S3150802AB0003461846F5F73CFEA7A3D3E90023F5F753
S3150802AB10EBFC02460B4620462946F6F70DF9034694
S3150802AB20002B00D187E1FB88184600F05DFAB0EEEB
S3150802AB30408A1BF029FF034618461CF0EBFD034624
S3150802AB4018464DF0D2F9034607EE903AF8EEE77A40
S3150802AB50B4EEE78AF1EE10FA4ED5FB88184600F0F5
S3150802AB6043FA10EE103A1846F5F71CFE04460D464F
S3150802AB70934B1B88184600F037FA10EE103A18461F
S3150802AB80F5F710FE88A3D3E90023F5F7ADFC0246D4
S3150802AB900B4620462946F6F7EDF80346002B06D063
S3150802ABA0864B00221A70864AFB88138061E0FB886E
S3150802ABB0184600F019FAF0EE407AB2EE047A67EE19
S3150802ABC0877AFCEEE77A17EE903A9CB27C4B1B88A2
S3150802ABD0184600F009FAF0EE407AB2EE047A67EE09
S3150802ABE0877AFCEEE77A17EE903A9BB29C4240D2FD
S3150802ABF0734AFB8813803CE0FB88184600F0F4F998
S3150802AC00B0EE408A6E4B1B88184600F0EDF9F0EE5E
S3150802AC10407AB4EEE78AF1EE10FA06DD674B0022B7
S3150802AC201A70674AFB88138023E0FB88184600F0EF
S3150802AC30DBF9F0EE407AB2EE047A67EE877AFCEE3A
S3150802AC40E77A17EE903A9CB25D4B1B88184600F0DD
S3150802AC50CBF9F0EE407AB2EE047A67EE877AFCEE2A
S3150802AC60E77A17EE903A9BB29C4202D2544AFB8884
S3150802AC701380544B1B78042B40F2DD80514B002283
S3150802AC801A704E4B1B780E2B03D94C4B0F221A7097
S3150802AC90D1E04A4B1B780533DAB2484B1A70CAE040
S3150802ACA0FB88184600F00CFA03461C461BF06CFE9D
S3150802ACB0034618461CF02EFD034618464DF015F9B4
S3150802ACC003469C420AD33D4B00221A701BF05CFED7
S3150802ACD00346002118461CF0F9F8AFE0FB8818462F
S3150802ACE000F082F910EE103A1846F5F75BFD0446B5
S3150802ACF00D46334B1B88184600F076F910EE103ACB
S3150802AD001846F5F74FFD2AA3D3E90023F5F7ECFB1E
S3150802AD1002460B4620462946F6F72CF80346002B30
S3150802AD2009D0264B00221A70254AFB881380264B27
S3150802AD3000221A7029E0FB88184600F055F9F0EE51
S3150802AD40407AB2EE047A67EE877AFCEEE77A17EE75
S3150802AD50903A9CB21A4B1B88184600F045F9F0EE59
S3150802AD60407AB2EE047A67EE877AFCEEE77A17EE55
S3150802AD70903A9BB29C4208D2114AFB881380124B26
S3150802AD801B780133DAB2104B1A700F4B1B78012B62
S3150802AD901CD90D4B1B78032B18D8084B0F221A7097
S3150802ADA04CE000BFAFF300809A9999999999B93FF7
S3150802ADB09A9999999999C93F0000E03FC11D0120C6
S3150802ADC0C21D0120C01D0120BE1D01201F4B1B787C
S3150802ADD0032B03D91E4B32221A702FE01D4B1B7808
S3150802ADE00133DAB21B4B1A701A4B1B78022B03D1AA
S3150802ADF0174B32221A7020E0164B1B78022B1CD9ED
S3150802AE00144B1B78062B18D9124B02221A70104BB8
S3150802AE101B78312B02D90E4B00221A700C4B1B7869
S3150802AE200533DAB20A4B1A7007E00B4829F0A6FF77
S3150802AE3004E000BF02E000BF00E000BF044B1B783D
S3150802AE4018461037BD46BDEC028BB0BDBE1D0120AB
S3150802AE50C11D0120C01D0120784D090880B400AF2C
S3150802AE60044B42F228321A8000BFBD465DF8047BC5
S3150802AE70704700BFFC07002080B582B000AF1BF008
S3150802AE8083FD034618461CF07CF80346FB711BF04B
S3150802AE907BFD034618461CF03DFC034618464DF05A
S3150802AEA009F803461A46FB79934216D3FFF7D6FFEB
S3150802AEB019F060FC03462621184619F089FC034658
S3150802AEC0002B4FD029481CF0B5FC19F053FC034659
S3150802AED0262118461BF030F944E0254B1B78FA79EF
S3150802AEE09A420ED2234B1B78002B07D0204B1B7895
S3150802AEF01946FB791A46204829F040FF1C4AFB7975
S3150802AF0013701B4B1B7803F10B02FB799A4210DA7A
S3150802AF10184B1B78002B07D0F979154B1B781A4664
S3150802AF200C23164829F02AFFFFF798FF104AFB79E7
S3150802AF301370134B1B88002B15D0114B1B88013B32
S3150802AF409AB20F4B1A800E4B1B88002B0BD10D4859
S3150802AF5029F014FF5EF0A4FD012302220B211BF047
S3150802AF60CBF800E000BF0837BD4680BDA04D0908F2
S3150802AF70C41D012000000020B84D0908D84D090853
S3150802AF80FC070020FC4D090880B487B000AF87EDA6
S3150802AF90050AC7ED040A87ED031AC7ED021A87EDFB
S3150802AFA0012A97ED057AD7ED047A37EE677AD7ED57
S3150802AFB0016AD7ED027A76EEE77A67EE276A97EDA7
S3150802AFC0037AD7ED047A77EE677A86EEA77AD7ED13
S3150802AFD0027A77EE277AB0EE670A1C37BD465DF825
S3150802AFE0047B70470000000080B52DED048B84B009
S3150802AFF000AF0346FB800023FB730023FB7309E0C3
S3150802B000FB7B2D4A32F81330FA889A4206D3FB7B29
S3150802B0100133FB73FB7B952BF2D900E000BFFB7B68
S3150802B020002B02D1DFED257A38E0FB8807EE903A4D
S3150802B030B8EE678AFB7B013B1F4A32F8133007EEEC
S3150802B040903AF8EE678AFB7B1B4A32F8133007EE12
S3150802B050903AB8EE679AFB7B07EE903AF8EE679A53
S3150802B060FB7B1846F5F78CFB11A3D3E90023F5F70A
S3150802B0703BFA02460B4610461946F5F7E3FE034627
S3150802B08002EE103AF0EE691AB0EE491AF0EE680AC4
S3150802B090B0EE480AFFF778FFF0EE407AB0EE670A9C
S3150802B0A01037BD46BDEC048B80BD00BFAFF30080F0
S3150802B0B0CDCCCCCCCCCCEC3F000800200000000064
S3150802B0C080B485B000AF0346FB800023FB730023E0
S3150802B0D0FB730CE0FB7B0B4A32F81330FA889A4270
S3150802B0E002D2FB7B9BB206E0FB7B0133FB73FB7B45
S3150802B0F0952BEFD9962318461437BD465DF8047B7F
S3150802B100704700BF0008002080B400AF034B1B68DD
S3150802B1101846BD465DF8047B704700BFC81D01206E
S3150802B12080B483B000AF78607B68002B01D100231E
S3150802B13046E07B68012B01D1012341E07B68022BA3
S3150802B14001D102233CE07B68032B01D1032337E0BC
S3150802B1507B68042B01D1042332E07B68052B01D1DD
S3150802B16005232DE07B68062B01D1062328E07B68A0
S3150802B170072B01D1072323E07B68082B01D108237B
S3150802B1801EE07B68092B01D80C2319E07B680A2B81
S3150802B19001D8102314E07B680B2B01D814230FE087
S3150802B1A07B680C2B01D818230AE07B680D2B01D883
S3150802B1B0202305E07B680E2B01D8302300E04023CC
S3150802B1C018460C37BD465DF8047B704780B483B0D9
S3150802B1D000AF0346FB80FB88002B01D1002346E023
S3150802B1E0FB88012B01D1012341E0FB88022B01D107
S3150802B1F002233CE0FB88032B01D1032337E0FB88BB
S3150802B200042B01D1042332E0FB88052B01D1052347
S3150802B2102DE0FB88062B01D1062328E0FB88072BA5
S3150802B22001D1072323E0FB88082B01D108231EE05E
S3150802B230FB880C2B01D8092319E0FB88102B01D8AF
S3150802B2400A2314E0FB88142B01D80B230FE0FB8892
S3150802B250182B01D80C230AE0FB88202B01D80D23D2
S3150802B26005E0FB88302B01D80E2300E00F23184691
S3150802B2700C37BD465DF8047B7047000080B500AF09
S3150802B2804FF400620E490F4854F020FC4FF4006256
S3150802B2900D490E4854F01AFC4FF400720C490D4839
S3150802B2A054F014FC4FF400620B490C4854F00EFC9F
S3150802B2B04FF400620A490B4854F008FC00BF80BDEF
S3150802B2C0DC1D0120CC1D0120EC250120DC250120F6
S3150802B2D0202E0120102E012060300120203001206E
S3150802B2E0A03801206038012084B0B0B400AF07F15D
S3150802B2F00C0484E80F00074B1D4607F10C040FCC1B
S3150802B3000FC50FCC0FC523682B6000BFBD46B0BC66
S3150802B31004B07047EC2D012080B586B000AF786086
S3150802B3200B467B800023FB7500233B610023FB60F1
S3150802B3300023BB6000F042FD0346002B0BD0494BAD
S3150802B340D3F844323B61474BD3F8843AFB607B68B7
S3150802B3501B68BB600AE0434BD3F844323B61414B5E
S3150802B360D3F8843AFB607B681B68BB603A69BB68A2
S3150802B3709A4230D13B4B93F86832002B0AD1394BAB
S3150802B380D3F850227B881344364AC2F85032012336
S3150802B390FB7561E0334BB3F86C321A467B8813446B
S3150802B3A0B3F5006F0BDA2F4BB3F86C227B88134484
S3150802B3B09AB22C4BA3F86C220123FB754CE00023AE
S3150802B3C0FB75284BB3F86C3219467B881A46264811
S3150802B3D029F0D4FC40E0FA68BB689A4227D1214B8F
S3150802B3E093F8A83A002B0AD11E4BD3F850227B8831
S3150802B3F013441C4AC2F850320223FB752CE0194B3F
S3150802B400B3F8AC3A1A467B881344B3F5006F0BDAE5
S3150802B410144BB3F8AC2A7B8813449AB2114BA3F89F
S3150802B420AC2A0223FB7517E00023FB7514E03B697F
S3150802B430002B07D1242279680C4863F0A2FC012369
S3150802B440FB7509E0FB68002B06D1242279680848B7
S3150802B45063F097FC0223FB75FB7D18461837BD4639
S3150802B46080BD00BFEC2D01203C4E0908303001207A
S3150802B4707038012080B584B000AF03463960FB718D
S3150802B4801346BB800023FB73FB79012B19D10023DA
S3150802B490FB7310E0FB7B3A681344012219461948EC
S3150802B4A054F0D4FB0346002B02D1174829F066FC58
S3150802B4B0FB7B0133FB73FB7B9BB2BA889A42E9D8C2
S3150802B4C01BE0FB79022B18D10023FB7310E0FB7BF0
S3150802B4D03A681344012219460C4854F0B7FB03464E
S3150802B4E0002B02D10A4829F049FCFB7B0133FB7386
S3150802B4F0FB7B9BB2BA889A42E9D800BF1037BD4691
S3150802B50080BD00BF20300120604E09086038012046
S3150802B510844E090880B582B000AF0346FB71FB1D55
S3150802B52001221946074854F091FB0346002B04D121
S3150802B530FB791946044829F021FC00BF0837BD46A5
S3150802B54080BD00BF102E0120A84E0908F0B5ABB089
S3150802B55008AFF861B9617A613B610023C7F88430A4
S3150802B560F8692CF0E4FFC7F880000023C7F8843096
S3150802B57044E0D7F884305A1CC7F88420B3F5FA7F1A
S3150802B5803CD907F150031946F8692DF003F93B6DCA
S3150802B590FB607A6DBA60B86D7860FB6D3A6E796E4B
S3150802B5A0B86EFC6E3C603D6F7E6FBC6F0794069664
S3150802B5B005953C68049403900291019200937B6876
S3150802B5C0BA68F968354829F0D9FB7B6E002B07D093
S3150802B5D0FB691B689A69FB691B6822F001029A617A
S3150802B5E0F8692CF0A4FFC7F88000D7F88010F8692C
S3150802B5F02CF0A9FF0023C7F8843006E00721F86972
S3150802B6002DF018F90346002BB3D17A69B969F8699E
S3150802B6102CF049FFF86900F02BFB0346FB67FB6F2A
S3150802B620002B37D007F1200330220021184663F099
S3150802B630F1FAF86900F0E2FA0346194A1360F86962
S3150802B64000F0F7FA0346164A5360154B1A68144B6C
S3150802B6505B6807F12000134963F048FA07F12003F3
S3150802B66018461CF0E7F8F86F00F056FB1BF08CF949
S3150802B67002460B4B1B68DBB2194610461CF0F4FA5D
S3150802B6801BF082F90246064B5B68DBB21946104686
S3150802B6901CF00CFB00BF8C37BD46F0BDD04E090826
S3150802B6A0A4400120144E090880B592B000AF3B466B
S3150802B6B040220021184663F0ADFA0023A7F842306B
S3150802B6C000237B64A04854F0A5FA034683F00103DD
S3150802B6D0DBB2002B00F0FA809C4B93F86832002B01
S3150802B6E062D19A4BD3F850329AB2984BA3F86C228D
S3150802B6F0964B0F22C3F8502210233B703B785AB25E
S3150802B700924BB3F86C321B0A9BB25BB203F00F037F
S3150802B7105BB213435BB2DBB23B708C4BB3F86C3251
S3150802B720DBB27B703B4602333E221946864854F00A
S3150802B730C8FA0346002B33D04FF47A71844839F09D
S3150802B74087FF0346002B0AD1FFF7DEFC3A46814BF8
S3150802B7508149FFF7FBFE7E4839F0BCFF02E07F48CD
S3150802B76029F00CFB794BB3F86C323E3B9AB2774B15
S3150802B770A3F86C22754BB3F86A3201339AB2734B4B
S3150802B780A3F86A22714B012283F868226F4BFF22C3
S3150802B79083F86E226D4B4FF4FA62C3F870222FE1DA
S3150802B7A06F4829F0EBFA2BE1684B93F86E32002BBF
S3150802B7B005D0664B93F86E32012B40F02181634B1C
S3150802B7C0B3F86C323E2B02D940237B6404E05F4B0C
S3150802B7D0B3F86C3201337B6420233B703B785AB250
S3150802B7E05A4BB3F86A325BB203F00F035BB21343E8
S3150802B7F05BB2DBB23B707B6C5A1E3B460133194681
S3150802B800514854F05EFA0346002B5BD07B6C9BB220
S3150802B8101846FFF7DBFC03464C4AC2F850324FF48F
S3150802B8207A714B4839F014FF0346002B0AD1FFF709
S3150802B8306BFC3A46474B4849FFF788FE444839F0BD
S3150802B84049FF02E0454829F099FA404BB3F86C22C1
S3150802B8507B6C9BB2D31A9BB201339AB23B4BA3F8C9
S3150802B8606C223A4BB3F86A3201339AB2374BA3F8D1
S3150802B8706A22364BB3F86C32002B40F0C180242280
S3150802B8800021354863F0C6F9304B002283F8682256
S3150802B8902E4B0022A3F86A222C4BFF2283F86E2233
S3150802B8A01BF072F8034618461CF03EFA0346002BB4
S3150802B8B000F0A680254BB3F86C321946294829F0C0
S3150802B8C05DFA9DE0284829F059FA99E0274854F08C
S3150802B8D0A1F9034683F00103DBB2002B00F0908046
S3150802B8E03B4601221946214854F0EBF90346002B40
S3150802B8F000F083803B781B09DBB2032B38D13B4629
S3150802B900013302221946194854F0DBF90346002B83
S3150802B91076D00E4B0322DA604FF47A710C4839F06E
S3150802B92097FE0346002B0AD1FFF7EEFB3A46094B70
S3150802B9300649FFF70BFE064839F0CCFE60E00748D9
S3150802B94029F01CFA5CE000BF20300120EC2D012012
S3150802B950A41B0120A040012030300120144F090801
S3150802B960344F0908484F0908584F0908102E012074
S3150802B9703B781B09DBB2002B42D13B46013301223D
S3150802B9801946214854F09DF90346002B37D03B78D7
S3150802B9901B029BB203F47063A7F842307B781A46FF
S3150802B9A0B7F842301343A7F84230B7F842203B466D
S3150802B9B002331946144854F084F90346002B1FD063
S3150802B9C0B7F8423002339BB21846FFF7FFFB03462D
S3150802B9D00E4AD3604FF47A710D4839F039FE0346A0
S3150802B9E0002B0DD1FFF790FB3A460A4B0749FFF7A2
S3150802B9F0ADFD074839F06EFE02E000BF00E000BF69
S3150802BA004837BD4680BD00BF102E0120EC2D01200F
S3150802BA10A41B0120A040012080B59AB000AF3B4686
S3150802BA2068220021184663F0F5F80E4854F0F2F839
S3150802BA30034683F00103DBB2002B0ED004E03B463B
S3150802BA406821184600F010F83B4668221946054850
S3150802BA5054F037F90346002BF1D100BF6837BD46CB
S3150802BA6080BD00BFDC25012080B582B000AF7860BA
S3150802BA700B467B80786800F00FFC00BF0837BD468E
S3150802BA8080BD000080B500AF1D4B93F86832002BCD
S3150802BA9034D01B4B93F86E32FF2B2FD1184BD3F8A9
S3150802BAA07032002B07D0164BD3F87032013B144A7A
S3150802BAB0C2F8703222E024220021124863F0AAF862
S3150802BAC04FF400621049114854F000F80C4B00225A
S3150802BAD083F868220A4B0022A3F86A22084BFF223F
S3150802BAE083F86E221AF050FF034618461CF01CF91A
S3150802BAF00346002B02D0064829F040F900BF80BD54
S3150802BB00EC2D012030300120603001202030012048
S3150802BB106C4F090880B582B000AF78600B467B800F
S3150802BB20786800F0DFFA00BF0837BD4680BD00001E
S3150802BB3080B582B000AF78600B467B807B881A4658
S3150802BB407968064854F082F80346002B02D1044865
S3150802BB5029F014F900BF0837BD4680BDCC1D012067
S3150802BB60804F090880B59AB000AF3B46682200218B
S3150802BB70184663F04FF80E4854F04CF8034683F023
S3150802BB800103DBB2002B0ED004E03B4668211846BF
S3150802BB90FFF7C0FF3B4668221946054854F091F85C
S3150802BBA00346002BF1D100BF6837BD4680BD00BFF2
S3150802BBB0CC1D012080B582B000AF78600B4A7B6845
S3150802BBC01360FFF75BFB24220021094863F022F881
S3150802BBD024220021074863F01DF824220021064882
S3150802BBE063F018F800BF0837BD4680BDC81D01209E
S3150802BBF0EC2D0120303001207038012080B485B048
S3150802BC0000AF78607B681B681B6CBB600023FB6017
S3150802BC10BB68DBB2002B05D0BB68DBB2FB60FB68F6
S3150802BC20DBB2FB60FB6818461437BD465DF8047B39
S3150802BC30704780B485B000AF78607B681B681B6C60
S3150802BC40BB600023FB60BB6803F4FE43002B07D0EE
S3150802BC50BB6803F4FE43FB60FB681B0ADBB2FB60AE
S3150802BC60FB6818461437BD465DF8047B704700002A
S3150802BC7080B485B000AF78607B681B685B6CBB607C
S3150802BC800023FB60BB6803F00703002B3BD0BB68AD
S3150802BC9003F00703013B052B2CD801A252F823F027
S3150802BCA0B9BC0208C3BC0208CDBC0208D7BC02084C
S3150802BCB0E1BC0208EBBC0208FB6843F00103FB6027
S3150802BCC019E0FB6843F00203FB6014E0FB6843F0EB
S3150802BCD00303FB600FE0FB6843F00403FB600AE022
S3150802BCE0FB6843F00503FB6005E0FB6843F00603C7
S3150802BCF0FB6000E000BF7B681B685A6C7B681B68A8
S3150802BD0022F007025A64FB68DBB218461437BD46AE
S3150802BD105DF8047B704700BF80B582B000AF7860DB
S3150802BD207B68013B052B27D801A252F823F000BFF6
S3150802BD3049BD020851BD020859BD020861BD020883
S3150802BD4069BD020871BD02080D481BF073FD13E0B8
S3150802BD500C481BF06FFD0FE00B481BF06BFD0BE068
S3150802BD600A481BF067FD07E009481BF063FD03E07C
S3150802BD7008481BF05FFD00BF00BF0837BD4680BDFF
S3150802BD80C44F0908D44F0908E44F090800500908A6
S3150802BD90185009083050090880B483B000AF03462A
S3150802BDA0FB71054AFB791370012318460C37BD4609
S3150802BDB05DF8047B704700BF2C09002080B400AFF1
S3150802BDC0034B1B781846BD465DF8047B704700BFD7
S3150802BDD02C09002080B500AFFFF7F0FF0346002BC1
S3150802BDE002D04FF4807301E04FF48073184680BD89
S3150802BDF080B500AFFFF7E2FF0346002B02D04FF4EF
S3150802BE00806301E04FF48063184680BD80B500AFB9
S3150802BE10FFF7D4FF0346002B02D04FF4805301E00C
S3150802BE204FF48053184680BD80B500AFFFF7C6FFB2
S3150802BE300346002B02D04FF4817301E04FF481735D
S3150802BE40184680BDB0B5A4B006AFF860B96013460F
S3150802BE50FB800023A7F87630FB683B65FFF7AEFF49
S3150802BE600346002B03D04FF080437B6501E0002395
S3150802BE707B650023BB65FB8802339BB21846FFF736
S3150802BE80A5F90346FB6500233B664FF480137B66E0
S3150802BE904FF40013BB660023FB6600233B670023AF
S3150802BEA03B743B7C5AB2FB881B0A9BB25BB203F01B
S3150802BEB00F035BB213435BB2DBB23B74FB88DBB2A4
S3150802BEC07B740223A7F8763010E0B7F87630023B87
S3150802BED0BA681A44B7F87630127878333B4403F8CE
S3150802BEE0682CB7F876300133A7F87630B7F876209B
S3150802BEF0FB8801339A42E8DD0023A7F876300DE085
S3150802BF00B7F8763078333B4413F8683C1846FFF79F
S3150802BF1001FBB7F876300133A7F87630B7F8762002
S3150802BF20FB8801339A42EBDD6D4607F160040FCCBC
S3150802BF300FC523682B6007F150030FCBFFF7D4F91F
S3150802BF4000BF7837BD46B0BD80B58EB000AFF86089
S3150802BF50B9601346FB80002387F83730FB683B61DC
S3150802BF60FFF72CFF0346002B03D04FF080437B617B
S3150802BF7001E000237B610023BB61FB88FB61002390
S3150802BF803B624FF480137B624FF40013BB620023BB
S3150802BF90FB6200233B63FA8807F110031146184631
S3150802BFA0FFF7BAF9034687F8373097F83730002B88
S3150802BFB006D0FA8897F83730B9681846FFF75AFA5A
S3150802BFC000BF3837BD4680BDB0B5A2B006AF7860AF
S3150802BFD0084611461A460346FB700B46BB701346C3
S3150802BFE07B70002387F86F307B68BB64FFF7E6FE39
S3150802BFF00346002B03D04FF08043FB6401E0002385
S3150802C000FB6400233B6503237B650023BB654FF472
S3150802C0108013FB654FF400133B6600237B660023FF
S3150802C020BB6630233B723B7A5AB297F9033003F068
S3150802C0300F035BB213435BB2DBB23B72BB787B7214
S3150802C0407B78BB72002387F86F300DE097F86F3064
S3150802C05070333B4413F8683C1846FFF75BFA97F8C7
S3150802C0606F30013387F86F3097F86F30022BEDD9AE
S3150802C0706D4607F158040FCC0FC523682B6007F1EC
S3150802C08048030FCBFFF730F900BF7037BD46B0BD86
S3150802C09080B582B000AF786000230022002178685C
S3150802C0A0FFF792FF00BF0837BD4680BD80B584B052
S3150802C0B000AFF860B9601346FB80FB883E2B06D8B2
S3150802C0C0FB881A46B968F868FFF7BCFE05E0FB88E4
S3150802C0D01A46B968F868FFF737FF00BF1037BD463A
S3150802C0E080BD000080B588B000AF7860FF23FB767C
S3150802C0F000237B610023FB6100237B827B68FB6054
S3150802C100FB6893F828301B09FB76FB681B687B6182
S3150802C110FFF76EFE02467B69934202D1FFF784FE61
S3150802C120F861FB7E032B00F2A78001A252F823F0E6
S3150802C13041C1020883C10208CDC102081BC2020816
S3150802C140FB6893F8283003F00F039AB24C4B1A8017
S3150802C1504B4B1B881B029AB2494B1A80FB6893F811
S3150802C16029301A46464B1B8813439AB2444B1A8007
S3150802C170FB682A33424A12881146184610F040FADA
S3150802C1807AE0FB6893F8283003F00F039AB23C4B27
S3150802C1901A803B4B1B881B029AB2394B1A80FB68E2
S3150802C1A093F829301A46364B1B8813439AB2344BF6
S3150802C1B01A80344B01221A70FB682A333E2118462C
S3150802C1C010F01EFAF869FFF763FF55E02D4B1B784E
S3150802C1D01A46FB6893F8283003F00F039A4248D1AF
S3150802C1E0FB68DB681846FEF79BFF0346013B7B822A
S3150802C1F0FB6829337A8A1146184610F001FA214B50
S3150802C2001B780133DAB21F4B1A701E4B1B780F2BA1
S3150802C2102FD91C4B00221A702BE01B4BD3F8443241
S3150802C220FA699A420FD1FB6893F8283003F00F0394
S3150802C230DAB2154B83F86E22FB6893F82920124B63
S3150802C24083F86F2217E0104BD3F8843AFA699A42B8
S3150802C25011D1FB6893F8283003F00F03DAB20A4BC0
S3150802C26083F8AE2AFB6893F82920074B83F8AF2A8E
S3150802C27001E000BF00E000BF00BF2037BD4680BD19
S3150802C280BC400120BE400120EC2D012080B500AF44
S3150802C29047F0A6FE00BF80BD80B485B000AF7860C7
S3150802C2A07B68FB60FB681B68B3F5806F05D1FB688A
S3150802C2B093F82830002B00D100BF00BF1437BD46C3
S3150802C2C05DF8047B7047000080B500AF4FF48072BA
S3150802C2D00349044853F0FAFB0123184680BD00BF00
S3150802C2E0D0400120C040012080B500AF054853F078
S3150802C2F091FC0346002B01D0012300E000231846D7
S3150802C30080BD00BFC040012080B584B000AF786010
S3150802C3100B46FB700023FB604FF47A710F4839F025
S3150802C32097F90346002B0AD1FB781A4679680C4816
S3150802C33053F0FBFDF860094839F0CCF902E00948E8
S3150802C34028F01CFDFB68002B02D1074828F016FDD1
S3150802C350012318461037BD4680BD00BFC41A012006
S3150802C360C0400120405009086850090880B584B0C9
S3150802C37000AF78600023FB734FF47A710B4839F0EB
S3150802C38067F90346002B09D17968094853F0DEFD9F
S3150802C3900346FB73054839F09DF902E0054828F083
S3150802C3A0EDFCFB7B18461037BD4680BDC41A01203A
S3150802C3B0C0400120A050090880B500AF4FF40072B2
S3150802C3C00349044853F082FB0123184680BD00BF87
S3150802C3D0E0410120D041012080B582B000AF0023A0
S3150802C3E0FB71074853F016FC0346FB71FB79002BD9
S3150802C3F001D0012300E0002318460837BD4680BD58
S3150802C400D041012080B584B000AF78600B46FB703E
S3150802C4100023FB604FF47A710F4839F019F9034685
S3150802C420002B0AD1FB781A4679680C4853F07DFD31
S3150802C430F860094839F04EF902E0094828F09EFCEE
S3150802C440FB68002B02D1074828F098FC01231846FE
S3150802C4501037BD4680BD00BFC41A0120D041012055
S3150802C460C8500908F050090880B584B000AF786052
S3150802C4700023FB734FF47A710B4839F0E9F8034647
S3150802C480002B09D17968094853F060FD0346FB730E
S3150802C490054839F01FF902E0054828F06FFCFB7BD6
S3150802C4A018461037BD4680BDC41A0120D041012066
S3150802C4B02051090880B584B000AF78600B46FB703E
S3150802C4C00023FB81012178684BF0BFFE034683F007
S3150802C4D00103DBB2002B1DD007F00CFFFB781A46CE
S3150802C4E0022108F03DF80346002B0ED007F002FFA2
S3150802C4F0FB781A46042108F0C9F80346002B09D12D
S3150802C5005E4828F03BFC0023B3E05D4828F036FC81
S3150802C5100023AEE0FB78184600F0DEF80346002B4F
S3150802C52004D1584828F02AFC0023A2E0FB781846D2
S3150802C53000F054F90346002B04D1534828F01EFC98
S3150802C540002396E0FB78184600F0C6F80346002B4F
S3150802C55004D14E4828F012FC00238AE00023FB810E
S3150802C56009E0642038F034F9FB78184628F0E6FD2D
S3150802C570FB890133FB81FB89062BF2D90020FDF7E3
S3150802C580BDF91AF001FA034618461BF01CFE0346CB
S3150802C590002B45D1012178684BF057FE034683F0FC
S3150802C5A00103DBB2002B63D007F0A4FEFB781A4620
S3150802C5B0012107F0D5FF0346002B0ED007F09AFE9D
S3150802C5C0FB781A46032108F061F80346002B09D1C5
S3150802C5D02F4828F0D3FB00234BE02E4828F0CEFB49
S3150802C5E0002346E007F086FEFB781A46022107F08A
S3150802C5F0B7FF0346002B0ED007F07CFEFB781A46DF
S3150802C600042108F043F80346002B31D11B4828F0D1
S3150802C610B5FB00232DE01A4828F0B0FB002328E0DA
S3150802C620012178684BF011FE034683F00103DBB261
S3150802C630002B1DD007F05EFEFB781A46052107F08F
S3150802C6408FFF0346002B0ED007F054FEFB781A46DE
S3150802C650082108F01BF80346002B09D10E4828F0DA
S3150802C6608DFB002305E00D4828F088FB002300E037
S3150802C670012318461037BD4680BD00BF7051090810
S3150802C68094510908BC510908E451090818520908C5
S3150802C69040520908645209088C520908B45209081A
S3150802C6A080B584B000AF0346FB710023FB6009E046
S3150802C6B0FB680133FB60012038F08AF8FB791846DB
S3150802C6C028F03CFDFB6840F6B7329342F0D900BF2A
S3150802C6D000BF1037BD4680BD80B584B000AF0346A3
S3150802C6E0FB710023FB810023BB81364828F046FBF9
S3150802C6F00023BB810023FB810DF076F8034618461A
S3150802C7000DF08CF90346022B53D10DF01DFD3BE0CB
S3150802C710012038F05DF8FB79184628F00FFDBB8931
S3150802C7200133BB81BB8942F20F7293420DD90DF0D8
S3150802C73021FD254828F022FB5DF0B2F901230222E9
S3150802C7401D2119F0D9FC002337E01AF01DF903461A
S3150802C75018461BF057FD0346012B06D10DF00AFDBC
S3150802C7601A481BF067F8002327E00DF03DF8034648
S3150802C77018460DF053F90346012B03D1FB89013301
S3150802C780FB8101E00023FB810DF02EF803461846D3
S3150802C7900DF044F90346022BBAD0FB89092BB7D907
S3150802C7A00B4828F0EBFA0DF0E5FC0A4828F0E6FA01
S3150802C7B002E0094828F0E2FA012318461037BD4676
S3150802C7C080BD00BFE05209081C5309085C530908DA
S3150802C7D080530908B4530908F053090880B584B090
S3150802C7E000AF0346FB710023FB810023BB81384857
S3150802C7F028F0C4FA0023BB810023FB81354B4FF096
S3150802C80000021A600CF0F0FF034618460DF006F90E
S3150802C8100346012B54D10DF097FC3BE0012037F07B
S3150802C820D7FFFB79184628F089FCBB890133BB81FF
S3150802C830BB8942F20F7293420DD90DF09BFC264832
S3150802C84028F09CFA5DF02CF9012301221D2119F02A
S3150802C85053FC002338E01AF097F8034618461BF0F3
S3150802C860D1FC0346012B06D10DF084FC1B481AF0B5
S3150802C870E1FF002328E00CF0B7FF034618460DF047
S3150802C880CDF80346022B03D1FB890133FB8101E074
S3150802C8900023FB810CF0A8FF034618460DF0BEF8EC
S3150802C8A00346022BBAD1FB89B3F57A7FB6D30C4875
S3150802C8B028F064FA0DF05EFC0A4828F05FFA02E0F6
S3150802C8C0094828F05BFA012318461037BD4680BD91
S3150802C8D024540908E043012060540908A0540908B1
S3150802C8E0C0540908F45409083055090880B582B0BD
S3150802C8F000AF0346FB7165481AF09CFF1AF044F82C
S3150802C900034618461BF05FFC0346002B56D107F078
S3150802C910F1FCFB791A46012107F022FE0346002B99
S3150802C92014D007F0E7FCFB791A46032107F0AEFE9E
S3150802C9300346002B16D11AF027F80346002118469B
S3150802C9401AF040FC52481AF075FF0BE01AF01CF870
S3150802C9500346002118461AF035FC4D481AF06AFFBC
S3150802C96000238EE007F0C6FCFB791A46022107F07F
S3150802C970F7FD0346002B15D007F0BCFCFB791A46D7
S3150802C980042107F083FE0346002B6FD119F0FCFF42
S3150802C9900346002118461AF015FC3E481AF04AFFCB
S3150802C9A000236EE019F0F0FF0346002118461AF03C
S3150802C9B009FC38481AF03EFF002362E007F09AFCA9
S3150802C9C0FB791A46022107F0CBFD0346002B15D048
S3150802C9D007F090FCFB791A46042107F057FE034636
S3150802C9E0002B17D119F0D0FF0346002118461AF07A
S3150802C9F0E9FB28481AF01EFF002342E019F0C4FF9B
S3150802CA000346002118461AF0DDFB22481AF012FFE7
S3150802CA10002336E007F06EFCFB791A46032107F07D
S3150802CA209FFD0346002B15D007F064FCFB791A46D6
S3150802CA30052107F02BFE0346002B17D119F0A4FF98
S3150802CA400346002118461AF0BDFB13481AF0F2FEF7
S3150802CA50002316E019F098FF0346002118461AF03B
S3150802CA60B1FB0D481AF0E6FE00230AE019F08CFF26
S3150802CA700346002118461AF0A5FB08481AF0DAFE02
S3150802CA80012318460837BD4680BD00BF645509080C
S3150802CA907855090890550908A8550908C45509087A
S3150802CAA080B582B000AF0346FB7119F06DFF0346ED
S3150802CAB018461BF01DFC10481AF0BCFEFB791846F6
S3150802CAC0FFF78CFE10210D481AF0B4FEFB791946C1
S3150802CAD0102000F097FD19F057FF034618461BF081
S3150802CAE077FC07481AF0A6FEFB791846FFF7F4FD0D
S3150802CAF000BF0837BD4680BDD8550908F055090854
S3150802CB000856090880B586B000AF0346FB710B4686
S3150802CB10BB7113467B710023FB750023BB7500238B
S3150802CB20BB820023FB7419F02FFF03460121184626
S3150802CB301CF0D8F819F028FF034618461BF043FBE9
S3150802CB400346012B40F0A08017F014FE034601218C
S3150802CB50184617F03DFE0346002B77D117F00AFE5A
S3150802CB6003460221184617F033FE0346002B6DD101
S3150802CB7017F000FE03460321184617F029FE03465E
S3150802CB80002B63D117F0F6FD03460421184617F069
S3150802CB901FFE0346002B59D117F0ECFD034605216B
S3150802CBA0184617F015FE0346002B4FD117F0E2FD83
S3150802CBB003460B21184617F00BFE0346002B45D1F8
S3150802CBC017F0D8FD03460C21184617F001FE034656
S3150802CBD0002B3BD117F0CEFD03461521184617F058
S3150802CBE0F7FD0346002B31D117F0C4FD0346162183
S3150802CBF0184617F0EDFD0346002B27D117F0BAFDAC
S3150802CC0003461721184617F0E3FD0346002B1DD1EC
S3150802CC1017F0B0FD03461821184617F0D9FD03464A
S3150802CC20002B13D117F0A6FD03461921184617F053
S3150802CC30CFFD0346002B09D117F09CFD03461A21A6
S3150802CC40184617F0C5FD0346002B1DD0CB481AF02F
S3150802CC50F1FD19F099FE034618461BF095FB0346AB
S3150802CC60002B03D07B791846FFF71AFF19F08CFEC2
S3150802CC70034618461BF050FB19F086FE0346184673
S3150802CC801BF0A6FB0123F6E319F07EFE03461846BF
S3150802CC901AF0CCFB0346002B01D00123FB7519F0D1
S3150802CCA073FE034618461BF013FB0346002B31D0CE
S3150802CCB019F06AFE034618461BF066FB0346002B6C
S3150802CCC028D07B791846FFF711FE0346002B21D19F
S3150802CCD0AB481AF0AFFD19F057FE034618461BF08B
S3150802CCE053FB0346002B03D07B791846FFF7D8FE81
S3150802CCF019F04AFE034618461BF00EFB19F044FECD
S3150802CD00034618461BF064FB9E499F481AF092FD9B
S3150802CD100023B0E319F038FE034618461BF034FB2D
S3150802CD200346002B69D007F0E5FA7B791A460221F9
S3150802CD3007F016FC0346002B32D007F0DBFA7B79A4
S3150802CD401A46042107F0A2FC0346002B51D119F01A
S3150802CD501BFE0346002118461AF034FA8B481AF0CD
S3150802CD6069FD19F011FE034618461BF00DFB034632
S3150802CD70002B03D07B791846FFF792FE19F004FEC2
S3150802CD80034618461BF0C8FA19F0FEFD0346184674
S3150802CD901BF01EFB7B497E481AF04CFD00236AE312
S3150802CDA019F0F2FD0346002118461AF00BFA7948E3
S3150802CDB01AF040FD19F0E8FD034618461BF0E4FA9E
S3150802CDC00346002B03D07B791846FFF769FE19F054
S3150802CDD0DBFD034618461BF09FFA19F0D5FD0346FC
S3150802CDE018461BF0F5FA67496B481AF023FD00232B
S3150802CDF041E37B791846FFF753FE19F0C5FD034652
S3150802CE0018461BF065FA0346002B00F0338307F039
S3150802CE1071FA7B791A46012107F0A2FB0346002B19
S3150802CE201ED007F067FA7B791A46032107F02EFC13
S3150802CE300346002B29D159481AF0FCFC19F0A4FD27
S3150802CE40034618461BF068FA19F09EFD0346184673
S3150802CE501BF0BEFA4B4952481AF0ECFC00230AE3CF
S3150802CE6050481AF0E7FC19F08FFD034618461BF0E6
S3150802CE7053FA19F089FD034618461BF0A9FA4149E7
S3150802CE8049481AF0D7FC0023F5E2FB79002B02D0B9
S3150802CE9046481AF0CFFC17F06DFC034600211846E7
S3150802CEA017F096FC0346002B32D117F063FC0346B3
S3150802CEB00021184617F08CFC0346002B28D117F0E0
S3150802CEC059FC03460121184617F082FC0346002B3B
S3150802CED01ED117F04FFC03460221184617F078FCBC
S3150802CEE00346002B14D117F045FC034603211846C6
S3150802CEF017F06EFC0346002B0AD117F03BFC0346DB
S3150802CF006521184617F064FC0346002B00F0AA8038
S3150802CF1027481AF08FFC19F037FD034618461BF00E
S3150802CF2052F90346002B5ED107F0E4F97B791A46DB
S3150802CF30022107F015FB0346002B3FD007F0DAF96A
S3150802CF407B791A46042107F0A1FB0346002B40F021
S3150802CF50908218481AF06EFC19F016FD0346184618
S3150802CF601BF0DAF919F010FD034618461BF030FAE1
S3150802CF70044911481AF05EFC00237CE2245609088B
S3150802CF8048560908685609088C5609089456090825
S3150802CF90B4560908BC560908DC560908E4560908B5
S3150802CFA00057090808570908245709082C57090879
S3150802CFB04C5709087857090898570908BF481AF0BC
S3150802CFC039FC19F0E1FC034618461BF0A5F919F0DD
S3150802CFD0DBFC034618461BF0FBF9B949B9481AF0B7
S3150802CFE029FC002347E207F085F97B791A460321D3
S3150802CFF007F0B6FA0346002B1FD007F07BF97B79B8
S3150802D0001A46052107F042FB0346002B40F03182FF
S3150802D010AD481AF00FFC19F0B7FC034618461BF088
S3150802D0207BF919F0B1FC034618461BF0D1F9A4495D
S3150802D030A6481AF0FFFB00231DE2A5481AF0FAFBE0
S3150802D04019F0A2FC034618461BF066F919F09CFC77
S3150802D050034618461BF0BCF999499E481AF0EAFBA2
S3150802D060002308E219F090FC0346012118461AF03B
S3150802D070A8F90023BB750023BB8210E0BB8A0133E3
S3150802D080BB82BB8AB3F5167F02D30123BB750FE0B9
S3150802D0907B79184628F052F8642037F099FB19F084
S3150802D0A073FC034618461AF05BF90346002BE5D1D2
S3150802D0B0BB7D012B1BD188481AF0BCFB5CF0F0FC47
S3150802D0C00123FA22F92119F017F819F05DFC034633
S3150802D0D018461BF021F919F057FC034618461BF0AF
S3150802D0E077F977497D481AF0A5FB0023C3E119F0C1
S3150802D0F04BFC0346012118461AF0A7F90023BB7513
S3150802D1000023BB8210E0BB8A0133BB82BB8AB3F51C
S3150802D110167F02D30123BB750FE07B79184628F0E8
S3150802D1200DF8642037F054FB19F02EFC0346184616
S3150802D1301AF05AF90346002BE5D1BB7D012B1BD108
S3150802D14067481AF077FB5CF0ABFC0123FA22F92157
S3150802D15018F0D2FF19F018FC034618461BF0DCF843
S3150802D16019F012FC034618461BF032F954495D4879
S3150802D1701AF060FB00237EE132215B481AF05AFB63
S3150802D1801BF06EFF034618461CF0C6F807F10803A3
S3150802D19008220021184661F03DFD07F108033221F5
S3150802D1A018461CF0F8FEBB79022B0FD14F481AF02D
S3150802D1B041FB07F108030C2118461CF022FF07F170
S3150802D1C00803022118461CF037FF15E0BB79032B2A
S3150802D1D00FD147481AF02EFB07F10803102118460B
S3150802D1E01CF00FFF07F10803032118461CF024FF61
S3150802D1F002E040481AF01EFB07F10803194601200F
S3150802D2001CF02AFF7B79184627F098FF1BF028FFA7
S3150802D210034618461CF05AF80346012B0DD1364828
S3150802D2201AF008FB00BF1BF01BFF034618461CF04A
S3150802D2304DF80346002B72D068E0FB7C0133FB7481
S3150802D2401BF00EFF034618461CF040F80346022B55
S3150802D2502FD11BF005FF034618461CF037F8034684
S3150802D260194626481AF0E6FA0023FB74BB79022B04
S3150802D2700BD123481AF0DEFA0C2102201CF0D8FA48
S3150802D2800C2102201CF08AFA11E0BB79032B0BD180
S3150802D2901C481AF0CFFA0C2103201CF0C9FA0C21FB
S3150802D2A003201CF07BFA02E017481AF0C3FA00239F
S3150802D2B0E1E0012037F08CFAA4E700BFA05709087D
S3150802D2C068560908C0570908C8570908E8570908D7
S3150802D2D0F0570908145809081C5809084458090837
S3150802D2E0505809087858090884580908A05809089E
S3150802D2F0C0580908E0580908085909082C590908A4
S3150802D3005059090870590908905909081BF0A8FECE
S3150802D310034618461BF0DAFF0346022B53D1584838
S3150802D3201AF088FA19F030FB0346002118461AF05B
S3150802D33048F8FB7D002B06D119F026FB034600218F
S3150802D34018461AF082F806F0D5FF7B791A460321A9
S3150802D35007F006F90346002B1ED006F0CBFF7B79B1
S3150802D3601A46052107F092F90346002B29D14548AA
S3150802D3701AF060FA19F008FB034618461AF0CCFFB1
S3150802D38019F002FB034618461BF022F83E493F48AD
S3150802D3901AF050FA00236EE03D481AF04BFA19F0DB
S3150802D3A0F3FA034618461AF0B7FF19F0EDFA0346E0
S3150802D3B018461BF00DF8344936481AF03BFA002392
S3150802D3C059E0002357E019F0DFFA03460021184610
S3150802D3D019F0F7FF7B791846FFF762F9FB7D002BF8
S3150802D3E006D119F0D1FA0346002118461AF02DF88B
S3150802D3F029481AF01FFA06F07DFF7B791A4603219F
S3150802D40007F0AEF80346002B1ED006F073FF7B79B1
S3150802D4101A46052107F03AF90346002B2AD11F4876
S3150802D4201AF008FA19F0B0FA034618461AF074FF09
S3150802D43019F0AAFA034618461AF0CAFF12491848FA
S3150802D4401AF0F8F9002316E016481AF0F3F919F05B
S3150802D4509BFA034618461AF05FFF19F095FA034637
S3150802D46018461AF0B5FF08490F481AF0E3F90023DF
S3150802D47001E000BF012318461837BD4680BD00BF2C
S3150802D480B4590908D859090868560908F8590908FB
S3150802D490045A0908285A0908345A0908505A090820
S3150802D4A0705A09087C5A0908A05A090890B587B023
S3150802D4B002AF0446084611461A462346FB7103463E
S3150802D4C0BB710B467B7113463B7100233B810023DC
S3150802D4D0FB813B799BB21A46920013445B003B815F
S3150802D4E0F979BA7978793B7900930346434827F064
S3150802D4F045FC97F820301846FFF770F900237B732E
S3150802D50000233B730023FB720023BB72FB79002BBB
S3150802D51001D00CF045FCBB79002B01D00CF0B8FC0D
S3150802D5207B79002B01D00CF023FD3B89002B01D01F
S3150802D5300DF0E2F97B7B002B08D03B7B002B05D054
S3150802D540FB7A002B02D0BB7A002B44D1FB799BB223
S3150802D550FA899A4203D301237B730CF03FFCBB7909
S3150802D5609BB2FA899A4203D301233B730CF0ACFCB3
S3150802D5707B799BB2FA899A4203D30123FB720CF098
S3150802D58015FDFA893B899A4203D30123BB720DF032
S3150802D590BFF919F0F9F9034618461AF033FE03469D
S3150802D5A0012B0CD10CF01AFC0CF08EFC0CF0FEFCD4
S3150802D5B00DF0AEF912481AF03DF900231AE0FB897C
S3150802D5C00133FB81642037F003F997F820301846B7
S3150802D5D027F0B4FDAEE700BF97F820301846FFF7EC
S3150802D5E07BF80CF0FBFB0CF06FFC0CF0DFFC0DF08B
S3150802D5F08FF9012318461437BD4690BD105B0908FA
S3150802D600605B090890B585B000AF03460A46FB7110
S3150802D6101346BB710023FB810023BB81FB799BB2B6
S3150802D6201A46920013445B00BB81BB89FA791946F4
S3150802D6304E4827F0A3FB19F0A7F9034618461AF035
S3150802D640E1FD0346012B06D149481AF0F3F80DF01D
S3150802D6505FF9002385E019F097F9034618461BF08F
S3150802D6602DFA0346012B0BD10DF05EF9BB89414A0F
S3150802D670A2FB0323DB089BB219463F481AF0DAF8E5
S3150802D68019F082F9034618461BF03AFA0346012BAB
S3150802D6900BD10DF031F9BB89364AA2FB0323DB080D
S3150802D6A09BB2194635481AF0C5F819F06DF90346C2
S3150802D6B018461BF025FA0346012B1CD019F064F90B
S3150802D6C0034618461BF0FAF90346012B13D019F044
S3150802D6D05BF9034618461BF013FA03461C4619F073
S3150802D6E053F9034618461BF0E9F903461A4621463A
S3150802D6F023481AF09FF80023FB811BE0BB791846E2
S3150802D70027F01CFD642037F063F819F03DF903464B
S3150802D71018461AF077FD0346012B08D114481AF069
S3150802D72089F80DF0F5F80DF00BF9002319E0FB89DD
S3150802D7300133FB81FA89BB899A42DFD30DF0E8F8F7
S3150802D7400DF0FEF819F020F90346002118461BF0E1
S3150802D750C4F919F019F90346002118461BF0DFF936
S3150802D760012318461437BD4690BD00BF805B0908E1
S3150802D770A85B0908CDCCCCCCC85B0908E85B0908CC
S3150802D780085C0908000000002DE9F047ADF50A7D9E
S3150802D79006AF04460846114607F50473A3F20923A1
S3150802D7A022461A7007F50473A3F20A2302461A7070
S3150802D7B007F50473A3F20B230A461A700023C7F867
S3150802D7C00C320023C7F808324FF00003C7F8E431D9
S3150802D7D04FF00003C7F804324FF00003C7F80032CF
S3150802D7E0002387F8FF31002387F8FE310023C7F8A4
S3150802D7F0F831012387F8F731002387F8F631002339
S3150802D800A7F8F4314FF00003C7F8F0310023C7F840
S3150802D810EC31002387F8EB31002387F8EA3107F564
S3150802D8200473A3F20A231B78002B02D1012300F00A
S3150802D8302FBE0020FCF77CF887ED790AAC4BD3EDB6
S3150802D840007AF5EE407AF1EE10FA03D1A84AD7F833
S3150802D850E431136007F50473A3F209231C78D7F899
S3150802D860E401F2F79FFF02460B462146A14819F04A
S3150802D870E1FF07F50473A3F20A231B78022B03D8E8
S3150802D8800023C7F80C3251E007F50473A3F20A2302
S3150802D8901B78022B0AD907F50473A3F20A231B780D
S3150802D8A0042B03D80023C7F80C323FE007F50473AC
S3150802D8B0A3F20A231B78042B0AD907F50473A3F2E9
S3150802D8C00A231B78062B03D80023C7F80C322DE04F
S3150802D8D007F50473A3F20A231B78062B0AD907F560
S3150802D8E00473A3F20A231B78082B03D80023C7F86C
S3150802D8F00C321BE007F50473A3F20A231B78082BE4
S3150802D9000AD907F50473A3F20A231B780A2B03D84C
S3150802D9100023C7F80C3209E007F50473A3F20A23B9
S3150802D9201B780A2B02D90023C7F80C3207F50473B1
S3150802D930A3F209231B78D7F80C2219466E4819F068
S3150802D94079FFD7F80C32002B71D00023C7F80832BA
S3150802D95045E064200CF004FA07F50473A3F20923E0
S3150802D9601B78652B02D10CF01BFA28E007F5047325
S3150802D970A3F209231B78662B02D10CF089FA1EE062
S3150802D98007F50473A3F209231B78672B0ED118F047
S3150802D990FBFF034618461BF0F7F80346012B02D194
S3150802D9A00CF056FB0BE00CF0E3FA08E007F50473FB
S3150802D9B0A3F209231B78682B01D10CF049FB6420DA
S3150802D9C036F006FF07F50473A3F20B231B781846F5
S3150802D9D027F0B4FBD7F808320133C7F80832D7F86C
S3150802D9E00822D7F80C329A42B3D30CF0CBF90CF0D2
S3150802D9F0F5F90CF069FA0CF0D9FA0CF043FB00239E
S3150802DA00C7F808320FE0642036F0E2FE07F5047321
S3150802DA10A3F20B231B78184627F090FBD7F8083297
S3150802DA200133C7F80832D7F80832052BEBD900209C
S3150802DA30FBF77EFF87ED810AD7F80432C7F8003272
S3150802DA40D7F80432C7F8F03107F50473A3F20923AD
S3150802DA501C7897ED817AD7ED797A77EE677A17EEA1
S3150802DA60900AF2F79FFE02460B462146234819F012
S3150802DA70E1FE07F50473A3F209231E7807F504737A
S3150802DA80A3F20A2393F80080D7F8E401F2F78AFE94
S3150802DA9004460D460020FBF7D5FF386018F074FFE0
S3150802DAA00346184619F095F903461846F4F71AFB81
S3150802DAB0034603933B680293CDE900454246314645
S3150802DAC00F4819F0B7FE97F8FE31322B00F0FA82AA
S3150802DAD0322B00F30783022B00F08082022B00F31D
S3150802DAE00183002B0ED0012B00F00482FAE200BF5C
S3150802DAF0E04301203C5C09085C5C09087C5C090877
S3150802DB009C5C09080020FBF713FF87ED810A07F5DD
S3150802DB100473A3F209231C78D7F80402F2F742FE2B
S3150802DB2002460B462146DE4819F084FED7F8000263
S3150802DB30F2F738FE04460D46D7F80402F2F732FE2B
S3150802DB404FF00002D74BF2F7CFFC02460B462046AF
S3150802DB502946F3F705F90346002B1ED097F8FF313D
S3150802DB60013387F8FF31D7F80002F2F71BFE0446A5
S3150802DB700D46D7F80402F2F715FE02460B46CDE922
S3150802DB80002322462B46C84819F054FE5BF088FF4C
S3150802DB900223FE221A2118F0AFFAD7F80432C7F880
S3150802DBA0003297F8FF31042B22D90CF0EBF80CF06F
S3150802DBB015F90CF089F90CF0F9F90CF063FA05215C
S3150802DBC0BA4819F037FE012387F8F631002387F899
S3150802DBD0F73118F0D9FE0346032118461AF033FE28
S3150802DBE05BF05EFF0123FF221A2118F085FA79E21B
S3150802DBF097ED817AD7ED797A37EE677A07F5047366
S3150802DC00A3F20A231B78043B07EE903AF8EEE77A6A
S3150802DC10B4EEE77AF1EE10FA1CD507F50473A3F20F
S3150802DC200A231B78042B15D90023A7F8F43197ED9C
S3150802DC30817AD7ED797A77EE677A17EE900AF2F754
S3150802DC40B1FD02460B469A4827F098F8012387F851
S3150802DC50FE317EE097ED817AD7ED797A77EE677AAB
S3150802DC6017EE900AF2F79EFD8BA3D3E90023F2F78B
S3150802DC703BFC02460B4614461D4607F50473A3F2FF
S3150802DC800A231B781846F2F77BFD02460B46204606
S3150802DC902946F3F751F80346002B15D00023A7F8B7
S3150802DCA0F43197ED817AD7ED797A77EE677A17EEBE
S3150802DCB0900AF2F777FD02460B467E4827F05EF891
S3150802DCC0022387F8FE3144E097ED817AD7ED797A17
S3150802DCD077EE677A17EE900AF2F764FD02460B466C
S3150802DCE0754827F04BF897ED817AD7ED797A77EE72
S3150802DCF0677A17EE900AF2F755FD02460B466F4809
S3150802DD0027F03CF815F038FC044618F03DFE0346A9
S3150802DD1018461AF017FF0346194607F50473A3F2C5
S3150802DD2009231B789AB297ED817AD7ED797A77EE3D
S3150802DD30677AB2EE047A67EE877AFCEEE77A17EE2E
S3150802DD40903A9BB2204615F0C5FC012387F8F631B6
S3150802DD50C8E197F8FE31012B47D197F8EA31012B32
S3150802DD6008D0012387F8EA310023C7F8EC310023EB
S3150802DD7087F8EB3197ED817AD7ED7C7A77EE677A79
S3150802DD80B6EE007AF4EEC77AF1EE10FA22D597F8D3
S3150802DD90EB31013387F8EB3197F8EB31052B40F27B
S3150802DDA09E810CF01BF80CF08FF80CF0FFF80CF0C3
S3150802DDB069F9434819F03EFD002387F8F73118F050
S3150802DDC0E3FD0346032118461AF03DFD012387F8B1
S3150802DDD0F63187E1D7F80432C7F8F0310023C7F8DD
S3150802DDE0EC31002387F8EB3179E197F8FE31022B03
S3150802DDF075D197F8EA31022B08D0022387F8EA315F
S3150802DE000023C7F8EC31002387F8EB31D7F8EC3159
S3150802DE100133C7F8EC3197ED817AD7ED7C7A77EE44
S3150802DE20677AB6EE007AF4EEC77AF1EE10FA4BD5B7
S3150802DE30D7F8EC31042B40F252810523C7F8EC31AE
S3150802DE400023A7F8F431012387F8FE3197F8EB315E
S3150802DE50013387F8EB3197F8EB31032B40F23F8118
S3150802DE600BF090FF0BF0BAFF0CF02EF80CF09EF8B0
S3150802DE700CF008F9134819F0DDFC002387F8F7318E
S3150802DE80012387F8F63118F07FFD03460321184669
S3150802DE901AF0D9FC26E100BF9A9999999999B93F3E
S3150802DEA0BC5C09080000E03FCC5C0908F85C09087C
S3150802DEB01C5D09083C5D09085C5D09087C5D09086A
S3150802DEC0C05D0908E45D0908D7F80432C7F8F031DD
S3150802DED00023C7F8EC31002387F8EB31FFE0D7F8C7
S3150802DEE00432C7F8F0310023C7F8EC31002387F86B
S3150802DEF0EB31F4E0B7F8F431002B51D107F504738E
S3150802DF00A3F209231B78652B08D1A04819F092FCC5
S3150802DF1064200BF025FF0BF043FF59E007F5047365
S3150802DF20A3F209231B78662B08D1994819F082FCBB
S3150802DF3064200BF015FF0BF0ABFF49E007F50473FD
S3150802DF40A3F209231B78672B1AD118F01DFD034685
S3150802DF5018461AF019FE0346012B08D18D4819F006
S3150802DF6069FC64200BF0FCFE0CF072F830E08A487B
S3150802DF7019F060FC64200BF0F3FE0BF0F9FF27E0C2
S3150802DF8007F50473A3F209231B78682B20D183486B
S3150802DF9019F050FC64200BF0E3FE0CF059F817E078
S3150802DFA0B7F8F431042B13D97D4819F043FC0BF06A
S3150802DFB0E9FE0BF013FF0BF087FF0BF0F7FF0CF0EF
S3150802DFC061F80023A7F8F431322387F8FE3189E095
S3150802DFD0B7F8F4310133A7F8F43183E0B7F8F4312E
S3150802DFE0002B51D107F50473A3F209231B78652B7D
S3150802DFF008D16C4819F01EFC64200BF0B1FE0BF038
S3150802E000CFFE59E007F50473A3F209231B78662BA2
S3150802E01008D1654819F00EFC64200BF0A1FE0BF03E
S3150802E02037FF49E007F50473A3F209231B78672B28
S3150802E0301AD118F0A9FC034618461AF0A5FD03469C
S3150802E040012B08D1594819F0F5FB64200BF088FE1C
S3150802E0500BF0FEFF30E0564819F0ECFB64200BF09B
S3150802E0607FFE0BF085FF27E007F50473A3F2092369
S3150802E0701B78682B20D14F4819F0DCFB64200BF083
S3150802E0806FFE0BF0E5FF17E0B7F8F431002B13D05B
S3150802E090494819F0CFFB0BF075FE0BF09FFE0BF00B
S3150802E0A013FF0BF083FF0BF0EDFF0023A7F8F43103
S3150802E0B0322387F8FE3115E0B7F8F4310133A7F8B1
S3150802E0C0F4310FE0B7F8F4310133A7F8F431B7F8B1
S3150802E0D0F431052B05D9002387F8FE3102E000BF8B
S3150802E0E000E000BF97F8F631002B6BD1D7F8F8316C
S3150802E0F00133C7F8F831D7F8F831B3F5E17F17D30A
S3150802E1000BF040FE0BF06AFE0BF0DEFE0BF04EFF44
S3150802E1100BF0B8FF294819F08DFB18F035FC0346B9
S3150802E120032118461AF08FFB002387F8F7314AE0D5
S3150802E13018F02AFC034618461AF064F80346012B1F
S3150802E14017D10BF01FFE0BF049FE0BF0BDFE0BF0CC
S3150802E1502DFF0BF097FF1A4819F06CFB002387F87E
S3150802E160F73118F011FC0346032118461AF06BFB27
S3150802E17029E007F50473A3F20B231B78184626F049
S3150802E180DDFF642036F024FB9DE400BF085E090823
S3150802E190185E0908285E0908405E0908585E0908DB
S3150802E1A0685E0908985E0908DC5E0908205F0908A6
S3150802E1B06C5F0908B85F0908FC5F0908446009082A
S3150802E1C07060090800BF0BF0DDFD0BF007FE0BF0CF
S3150802E1D07BFE0BF0EBFE0BF055FF07F50473A3F27B
S3150802E1E009231E7807F50473A3F20A2393F800A0FD
S3150802E1F097ED817AD7ED797A77EE677A17EE900AF4
S3150802E200F2F7D0FA04460D46D7F80402F2F7CAFA2C
S3150802E210804689460020FBF715FC386018F0B4FBE7
S3150802E2200346184618F0D5FD03461846F3F75AFF73
S3150802E230034605933B680493CDE90289CDE9004577
S3150802E24052463146954819F0F5FA07F50473A3F2D2
S3150802E2500A231B78023307EE903AB8EEE77AD7ED2F
S3150802E260816AD7ED797A76EEE77AB4EEE77AF1EE55
S3150802E27010FA67D807F50473A3F20A231B789C1CC5
S3150802E28097ED817AD7ED797A77EE677A17EE900A63
S3150802E290F2F788FA02460B462146814819F0CAFA6D
S3150802E2A007F50473A3F209231B78652B07D15BF0E4
S3150802E2B0F7FB012365221A2117F01EFF42E007F534
S3150802E2C00473A3F209231B78662B07D15BF0E8FBDC
S3150802E2D0012366221A2117F00FFF33E007F50473AC
S3150802E2E0A3F209231B78672B1ED118F04DFB0346B0
S3150802E2F018461AF049FC0346012B0AD1694819F057
S3150802E30099FA5BF0CDFB022367221A2117F0F4FE75
S3150802E31018E0654819F08EFA5BF0C2FB0223672201
S3150802E3201A2117F0E9FE0DE007F50473A3F2092393
S3150802E3301B78682B06D15BF0B3FB012368221A21EE
S3150802E34017F0DAFE07F5EE7308220021184660F088
S3150802E35061FC07F50473A3F209231B789AB207F541
S3150802E360EE73114618464AF02FF918F00DFB0346CC
S3150802E370184619F0ABFE03461A4607F5EE73114620
S3150802E38018464AF030F997ED817AD7ED797AB4EEE4
S3150802E390E77AF1EE10FA15DD97ED817AD7ED797AFB
S3150802E3A077EE677AB2EE047A67EE877AFCEEE77A58
S3150802E3B017EE903A9AB207F5EE73114618464AF0E6
S3150802E3C0E8F805E007F5EE73002118464AF0E1F889
S3150802E3D007F10C0207F5EE73114618464FF038FF9F
S3150802E3E007F10C0318464EF018FE044607F10C0313
S3150802E3F018464EF02EFE0346194620460EF0DAF867
S3150802E40007F5EC7302220021184660F003FC274B3D
S3150802E410D3ED007A97ED817AB4EEE77AF1EE10FA47
S3150802E42016DD224BD3ED007A97ED817A77EE677A7D
S3150802E4309FED1F7A67EE877AFCEEE77A17EE903A37
S3150802E4409AB207F5EC73114618464AF0F5F905E053
S3150802E45007F5EC73002118464AF0EEF907F10C02AB
S3150802E46007F5EC731146184650F03DF907F10C030F
S3150802E47018464EF0D2FD044607F10C0318464EF034
S3150802E480E8FD0346194620460EF094F897F8F73148
S3150802E490184607F50477BD46BDE8F0879060090877
S3150802E4A0B4600908E860090810610908E043012018
S3150802E4B000007A4490B587B000AF04460846114674
S3150802E4C01A462346FB8003467B710B463B7113466D
S3150802E4D0FB7000237B6107F10C0308220021184612
S3150802E4E060F098FBFA8807F10C03114618461BF0F0
S3150802E4F052FD3B79022B0CD107F10C030C2118466D
S3150802E5001BF07FFD07F10C03022118461BF094FD50
S3150802E5100EE03B79032B0BD107F10C0310211846A9
S3150802E5201BF06FFD07F10C03032118461BF084FD4F
S3150802E5301AF096FD034618461AF0EEFE07F10C038A
S3150802E540194601201BF088FDF9883A797B794848F3
S3150802E55019F070F91AF084FD034618461AF0B6FE49
S3150802E5600346012B07D1434819F064F900BF7B79AA
S3150802E570002B74D158E07B6901337B617B694FF6C6
S3150802E580E752934208D81AF06BFD034618461AF06A
S3150802E5909DFE0346022B3FD13C791AF061FD0346E4
S3150802E5A018461AF093FE03461A462146324819F0CF
S3150802E5B041F900237B613B79022B11D13B790C216E
S3150802E5C018461BF035F93B790C2118461BF0E6F87C
S3150802E5D018F0DAF90346032118461AF0A8F919E0E1
S3150802E5E03B79032B11D13B79102118461BF020F9F0
S3150802E5F03B79102118461BF0D1F818F0C5F90346E5
S3150802E600032118461AF007FA04E03B7919461B4813
S3150802E61019F010F9002326E0012036F0D9F8FB7824
S3150802E620184626F08BFD95E73B79022B07D118F0A1
S3150802E630ABF90346022118461AF04AF90FE03B796C
S3150802E640032B07D118F0A0F90346022118461AF03F
S3150802E650B3F904E03B791946094819F0EBF8094879
S3150802E66019F0E8F8012318461C37BD4690BD00BFCD
S3150802E670346109086061090880610908AC61090802
S3150802E680D0610908F461090890B591B002AF044651
S3150802E690084611461A462346FB710346BB800B46BB
S3150802E6A07B801346BB71002387F837304FF4167305
S3150802E6B0FB8300233B630023FB624FF00003BB612D
S3150802E6C00023BB624FF000037B6200233B620023F8
S3150802E6D07B61FB79012B2AD9FB79032B27D8FB7996
S3150802E6E0184600F05DFF87ED060A00BFB869F2F723
S3150802E6F059F802460B46B9880091C94819F09AF8A2
S3150802E700FB8B1946C74826F039FB07F10C0308228A
S3150802E7100021184660F07EFAFA8B07F10C031146BF
S3150802E72018461BF038FCFB79022B0CD104E0BE48D4
S3150802E73019F080F8002366E207F10C030C2118464B
S3150802E7401BF05FFC08E0FB79032B05D107F10C03EC
S3150802E750102118461BF055FCFA7907F10C031146ED
S3150802E76018461BF069FC1AF07BFC034618461AF099
S3150802E770D3FD07F10C03194601201BF06DFC1AF0B4
S3150802E7806FFC044607F10C0318461BF02EFC0346E1
S3150802E790194620461AF0CEFD02463B6B93420FD02D
S3150802E7A01AF05EFC044607F10C0318461BF01DFC22
S3150802E7B00346194620461AF0BDFD38630023FB625C
S3150802E7C0FB6A42F20F72934267D95BF069F9012339
S3150802E7D06522092117F090FCFB791A467969934854
S3150802E7E019F028F8FB79022B26D1FB790C21184659
S3150802E7F01BF01EF8FB790C2118461AF0CFFF18F009
S3150802E800C3F80346032118461AF091F81AF028FCB1
S3150802E81003460C2118461AF04FFF04461AF020FC4C
S3150802E82003460C2118461AF085FD03461A46214668
S3150802E8307F4818F0FFFF2EE0FB79032B26D1FB79E0
S3150802E840102118461AF0F4FFFB79102118461AF01F
S3150802E850A5FF18F099F80346032118461AF0DBF8C3
S3150802E8601AF0FEFB0346102118461AF025FF044645
S3150802E8701AF0F6FB0346102118461AF05BFD03460A
S3150802E8801A4621466A4818F0D5FF04E0FB7919466C
S3150802E890684818F0CFFF0023B5E1FB79184697EDD3
S3150802E8A0060A00F0AFFEF0EE407AB3EE0E7AF4EE08
S3150802E8B0C77AF1EE10FA06DB97F83730002B02D149
S3150802E8C0012387F83730FB79184697ED060A00F0D8
S3150802E8D099FEB0EE407ABB8807EE903AF8EEE77AF0
S3150802E8E0B4EEE77AF1EE10FAC0F2B480FB79022BA5
S3150802E8F005D1FB790C2118461AF09AFF07E0FB7935
S3150802E900032B04D1FB79102118461AF091FF1AF04D
S3150802E910A7FB034618461AF0D9FC0346012B2CD14D
S3150802E920FB791946444818F085FF00BFFB7918465B
S3150802E93097ED060A00F066FE10EE103A1846F1F751
S3150802E94031FF02460B46F97900913C4818F072FFEE
S3150802E9503B4826F013FA00BF3A4826F00FFA3A481F
S3150802E96018F068FF12F04EFF0346184613F001F935
S3150802E9700346642B40F0468134E13B6A01333B622D
S3150802E9803B6A42F22732934208D81AF069FB0346D9
S3150802E99018461AF09BFC0346022B3DD100233B6224
S3150802E9A01AF05EFB034618461AF090FC034619460F
S3150802E9B0264818F03FFFFB79022B11D1FB790C216F
S3150802E9C018461AF035FFFB790C2118461AF0E6FEAE
S3150802E9D017F0DAFF03460321184619F0A8FF19E0D3
S3150802E9E0FB79032B11D1FB79102118461AF020FF67
S3150802E9F0FB79102118461AF0D1FE17F0C5FF034617
S3150802EA00032118461AF007F804E0FB79194610485C
S3150802EA1018F010FF0023F6E0012035F0D9FE76E75C
S3150802EA203C6209085C6209081062090884620908DE
S3150802EA30B4620908C4620908E86209084063090859
S3150802EA405C630908286409085C6409080463090800
S3150802EA5028630908FB79184697ED060A00F0D2FDE5
S3150802EA60B0EE407AD7ED097AF0EE086A77EEA67A22
S3150802EA70B4EEE77AF1EE10FA09DDFB79184697ED5E
S3150802EA80060A00F0BFFD87ED090A0023BB62BB6ACE
S3150802EA900133BB62BB6A4EF65F22934209D817F06E
S3150802EAA073FF0346184619F0ADFB0346012B40F0E7
S3150802EAB08D80574818F0BEFE17F066FF03461846C3
S3150802EAC019F0A0FB0346012B03D1524818F0B2FEF7
S3150802EAD07AE0FB79184600F063FD10EE103A184604
S3150802EAE0F1F760FE02460B464B4818F0A3FE97F86C
S3150802EAF0483041F270721E21022004F0B3F903462F
S3150802EB00002B0BD1454818F095FE5AF0C9FF012390
S3150802EB100322082117F0F0FA002374E097F8483028
S3150802EB20184626F00BFB4FF47A7035F051FE97F82B
S3150802EB304830184626F002FBFB79184600F030FDED
S3150802EB4010EE103A1846F1F72DFE02460B463448E7
S3150802EB5018F070FE97F8483041F270721E210120B3
S3150802EB6004F080F90346002B0BD12C4818F062FEFC
S3150802EB705AF096FF01230322082117F0BDFA002353
S3150802EB8041E097F84830184626F0D8FA4FF47A70DA
S3150802EB9035F01EFE97F84830184626F0CFFAFB796C
S3150802EBA0184600F0FDFC10EE103A1846F1F7FAFD89
S3150802EBB002460B461B4818F03DFE5AF071FF012328
S3150802EBC00322082117F098FA00231CE0FB6A013396
S3150802EBD0FB6297F84830184626F0B0FA012035F05D
S3150802EBE0F7FDCCE517F0D0FE0346184619F0EBFA06
S3150802EBF00346002B06D012F005FE034601211846ED
S3150802EC0012F0C4FF012318463C37BD4690BD00BF2B
S3150802EC107C630908AC630908D0630908E463090838
S3150802EC20006409081464090890B52DED028B87B0B3
S3150802EC3002AF0446084611461A462346FB80034697
S3150802EC407B710B463B711346FB704FF00003BB60AA
S3150802EC500023FB810023BB8117F096FE3B791A46F7
S3150802EC606E2118F081FDBC4818F0E4FDBB4B00226A
S3150802EC701A80BB4B00221A8015F07CFD034601213F
S3150802EC80184615F0A5FD0346002B04D0B54818F022
S3150802EC90D1FD0023EDE205F02DFB97F848301A4620
S3150802ECA0012105F05DFC0346002B1BD005F022FB73
S3150802ECB097F848301A46032105F0E8FC0346002B6C
S3150802ECC009D1A94818F0B6FD97F848301846FDF755
S3150802ECD00DFE0023CDE2A54818F0ACFDFB88772B84
S3150802ECE07BD104E0A24818F0A5FD0023C1E217F083
S3150802ECF04BFE0346184619F066FA0346012B6CD1F9
S3150802ED0097F84030002B5ED17B79022B08D104F0AC
S3150802ED1091FF034601220C21184605F07BF810E004
S3150802ED207B79032B08D104F085FF034601221021C3
S3150802ED30184605F06FF804E07B7919468D4818F0F5
S3150802ED4079FD0023BB8113E0642035F041FD97F875
S3150802ED504830184626F0F2F917F016FE034618460A
S3150802ED6019F050FA0346012B0ED0BB890133BB8139
S3150802ED7017F00AFE0346184618F078FC03461A46A8
S3150802ED80BB899342E0D300E000BF7B79022B08D10E
S3150802ED9004F050FF034600220C21184605F03AF803
S3150802EDA09FE07B79032B08D104F044FF0346002237
S3150802EDB01021184605F02EF893E07B7919466E481D
S3150802EDC018F038FD8DE097F8403098B297F8483039
S3150802EDD07A790121FFF76EFB83E07B79022B08D152
S3150802EDE004F028FF034601220C21184605F012F802
S3150802EDF010E07B79032B08D104F01CFF034601229D
S3150802EE001021184605F006F804E07B7919465B4896
S3150802EE1018F010FD17F0B8FD0346184619F0D3F995
S3150802EE200346002B22D10023BB8113E0642035F070
S3150802EE30CFFC97F84830184626F080F917F0A4FD5B
S3150802EE400346184619F0DEF90346012B29D0BB8979
S3150802EE500133BB8117F098FD0346184618F006FCE5
S3150802EE6003461A46BB899342E0D31DE00023BB81C1
S3150802EE7013E0642035F0ACFC97F84830184626F0C3
S3150802EE805DF917F081FD0346184619F0BBF90346EA
S3150802EE90012B08D0BB890133BB81BB89132BE8D967
S3150802EEA002E000BF00E000BF7B79022B08D104F024
S3150802EEB0C1FE034600220C21184604F0ABFF10E0FF
S3150802EEC07B79032B08D104F0B5FE034600221021F4
S3150802EED0184604F09FFF04E07B791946264818F085
S3150802EEE0A9FCFB88772B2BD117F04EFD0346184653
S3150802EEF019F069F90346012B22D10023BB8113E0DD
S3150802EF00642035F065FC97F84830184626F016F95D
S3150802EF1017F03AFD0346184619F074F90346012B11
S3150802EF200CD0BB890133BB81B98997F844201346B3
S3150802EF309B0013445B009942E2DB3AE000BF38E0EB
S3150802EF4017F022FD0346184619F03DF90346002B31
S3150802EF502FD00023BB8127E070640908E44301200F
S3150802EF60E643012080640908A8640908C4640908FC
S3150802EF70DC64090800650908246509084865090862
S3150802EF80642035F025FC97F84830184626F0D6F85E
S3150802EF9017F0FAFC0346184619F034F90346012B12
S3150802EFA006D0BB890133BB81BB89132BE8D900E0A4
S3150802EFB000BF17F0E9FC0346184619F023F9034681
S3150802EFC0012B04D1AE4818F035FC002351E117F0A5
S3150802EFD0DBFC3B791A46712118F0C6FB3B8D002BE8
S3150802EFE01BD097F848307A79388D0021FFF762FAF4
S3150802EFF00346002B40F0BE80A24818F01BFC97F887
S3150802F00048301846FDF772FC5AF04AFD01230122E0
S3150802F010082117F071F800232BE1BB8D002B00F0B5
S3150802F020A9807B79184600F0BBFA87ED020A97F8A1
S3150802F0303C40FA88B98D787997F848300093234688
S3150802F040FFF722FB0346002B09D18F4818F0F2FB83
S3150802F05097F848301846FDF749FC002309E10023D2
S3150802F060BB810AE0642035F0B3FB97F848301846AE
S3150802F07026F064F8BB890133BB81BB890E2BF1D913
S3150802F0807B79184697ED020A00F0BCFAB0EE407A90
S3150802F090BB8D0A3B07EE903AF8EEE77AB4EEE77ACA
S3150802F0A0F1EE10FA52D8BB8D142B4FD9BB8D07EE51
S3150802F0B0903AB8EEE78A7B79184697ED020A00F08D
S3150802F0C0A1FAF0EE407A78EE677AFCEEE77A17EE66
S3150802F0D0903AFB81FC897B79184697ED020A00F083
S3150802F0E091FA10EE103A1846F1F75CFB02460B4607
S3150802F0F0B98D00912146654818F09CFB97F83C406B
S3150802F100FA88F989787997F8483000932346FFF701
S3150802F110BBFA0346002B09D15B4818F08BFB97F81C
S3150802F12048301846FDF7E2FB0023A2E07B79184631
S3150802F13097ED020A00F066FA10EE103A1846F1F751
S3150802F14031FB02460B46524818F074FBFC897B7960
S3150802F150184697ED020A00F055FA10EE103A1846CC
S3150802F160F1F720FB02460B46B98D00912146494824
S3150802F17018F060FB17F008FC0346184619F023F846
S3150802F1800346012B28D105F0B5F897F848301A46F8
S3150802F190072105F0E5F90346002B18D005F0AAF871
S3150802F1A097F848301A460B2105F070FA0346002BE9
S3150802F1B009D1394818F03EFB97F848301846FDF74A
S3150802F1C095FB002355E0354818F034FB04E0344833
S3150802F1D018F030FB00234CE097F83C30002B23D183
S3150802F1E00023BB8113E0642035F0F2FA97F8483021
S3150802F1F0184625F0A3FF17F0C7FB0346184619F071
S3150802F20001F80346012B0ED0BB890133BB8117F0E7
S3150802F210BBFB0346184618F04CFA03461A46BB8946
S3150802F2209342E0D300E000BF17F0AEFB0346184650
S3150802F23018F0E8FF0346012B04D1114818F0FAFA30
S3150802F240002316E0FB88772B08D017F09DFB0246B1
S3150802F250144B1B881946104619F0BFF9124818F0C4
S3150802F260E9FA17F091FB3B791A46722118F07CFAF3
S3150802F270012318461437BD46BDEC028B90BD00BF6C
S3150802F2806C6509088C650908AC650908CC65090826
S3150802F290F0650908106609083C66090858660908EF
S3150802F2A070660908E64301209466090880B584B0A9
S3150802F2B000AF0346FB800B467B7113463B71002366
S3150802F2C0FB81A74818F0B6FA17F05EFB0346184604
S3150802F2D018F079FF0346002B2FD117F055FB03468A
S3150802F2E0184618F0F5FF0346002B08D117F04CFB19
S3150802F2F00346184619F080F80346002B5FD004F03F
S3150802F300F9FF3B791A46022105F02AF90346002B32
S3150802F3100ED004F0EFFF3B791A46042105F0B6F940
S3150802F3200346002B4BD18F4818F084FA002313E1C9
S3150802F3308D4818F07FFA00230EE117F025FB0346E5
S3150802F340184618F0C5FF0346002B1AD117F01CFB06
S3150802F3500346184619F050F80346002B11D104F05B
S3150802F360C9FF0346184604F0DBFF0346032B08D001
S3150802F37004F0C0FF0346184604F0D2FF03460B2BDF
S3150802F3801DD104F0B7FF3B791A46032105F0E8F8C8
S3150802F3900346002B0ED004F0ADFF3B791A46052131
S3150802F3A005F074F90346002B09D1704818F042FAA1
S3150802F3B00023D1E06E4818F03DFA0023CCE017F09E
S3150802F3C0E3FA0346184618F0FEFE0346002B25D13B
S3150802F3D004F090FF3B791A46012105F0C1F803466D
S3150802F3E0002B12D004F086FF3B791A46032105F05A
S3150802F3F04DF90346002B37D15E4818F01BFA3B79C4
S3150802F4001846FDF773FA0023A6E05B4818F012FACD
S3150802F4103B791846FDF76AFA00239DE004F06AFF75
S3150802F4203B791A46042105F09BF80346002B12D0B5
S3150802F43004F060FF3B791A46072105F027F90346CF
S3150802F440002B11D14D4818F0F5F93B791846FDF70E
S3150802F4504DFA002380E04A4818F0ECF93B79184641
S3150802F460FDF744FA002377E03B797A79F888012197
S3150802F470FFF720F80346002B08D1424818F0DAF9BC
S3150802F4803B791846FDF732FA002365E00023FB8133
S3150802F49016E0642035F09CF93B79184625F04EFEB5
S3150802F4A017F072FA0346184618F0ACFE0346012B0B
S3150802F4B003D1354818F0BEF905E0FB890133FB8113
S3150802F4C0FB89092BE5D917F05FFA0346184618F0A7
S3150802F4D07AFE0346002B1DD104F00CFF3B791A462F
S3150802F4E0032105F03DF80346002B0ED004F002FF77
S3150802F4F03B791A46052105F0C9F80346002B27D1A0
S3150802F500224818F097F9002326E0214818F092F9C4
S3150802F510002321E004F0EEFE3B791A46052105F0A8
S3150802F5201FF80346002B0ED004F0E4FE3B791A4678
S3150802F530092105F0ABF80346002B09D1154818F046
S3150802F54079F9002308E0144818F074F9002303E057
S3150802F550124818F06FF9012318461037BD4680BDC8
S3150802F560A4660908B8660908E4660908146709085A
S3150802F5704C67090888670908B0670908DC6709083B
S3150802F580146809085068090888680908A8680908F3
S3150802F590D4680908046909083C69090878690908E8
S3150802F5A080B582B000AF0346FB71FB79012B08D107
S3150802F5B017F0EAF90346184618F018FAF0EE407AF8
S3150802F5C019E0FB79022B08D117F0DEF90346184633
S3150802F5D018F032FAF0EE407A0DE0FB79032B08D1E7
S3150802F5E017F0D2F90346184618F04CFAF0EE407AAC
S3150802F5F001E0DFED037AB0EE670A0837BD4680BD43
S3150802F6000000000080B582B000AF87ED010A03460C
S3150802F610FB70FB78012B0CD117F0B6F90346184696
S3150802F62018F0E4F9B0EE407AD7ED017A77EE677A08
S3150802F63021E0FB78022B0CD117F0A6F903461846EF
S3150802F64018F0FAF9B0EE407AD7ED017A77EE677AD2
S3150802F65011E0FB78032B0CD117F096F903461846EE
S3150802F66018F010FAB0EE407AD7ED017A77EE677A9B
S3150802F67001E0DFED037AB0EE670A0837BD4680BDC2
S3150802F68000000000B0B584B000AF04460846114633
S3150802F6901A462346FB710346BB710B467B7113461A
S3150802F6A03B710023FB6003220021A8485FF0B2FAEF
S3150802F6B0FB791946A54852F0E9FA7B791946A34817
S3150802F6C052F0FFFABB79012B04D101219F4852F06F
S3150802F6D0C2FADDE0BB79022B04D102219B4852F023
S3150802F6E0BAFAD5E0BB79032B04D10321974852F025
S3150802F6F0B2FACDE0BB79042B04D10421934852F027
S3150802F700AAFAC5E0BB79C82B40F0BB8001218F4815
S3150802F71052F0A1FAFB79012B07D18D4825F02EFB71
S3150802F72006218A4852F0B2FAB2E0FB79022B07D1D7
S3150802F730884825F023FB0721844852F0A7FAA7E058
S3150802F740FB79032B07D1844825F018FB08217F484B
S3150802F75052F09CFA9CE0FB79042B07D17F4825F0EE
S3150802F7600DFB0121794852F091FA91E0FB79052BBC
S3150802F77007D17B4825F002FB0221744852F086FA2B
S3150802F78086E0FB79062B07D1764825F0F7FA03219E
S3150802F7906E4852F07BFA7BE0FB79072B07D1724859
S3150802F7A025F0ECFA0421694852F070FA70E0FB7908
S3150802F7B0082B07D16D4825F0E1FA0521634852F076
S3150802F7C065FA65E0FB79092B07D1694825F0D6FA6F
S3150802F7D00E215E4852F05AFA5AE0FB790A2B07D1F3
S3150802F7E0644825F0CBFA0F21584852F04FFA4FE0F9
S3150802F7F0FB790B2B07D1604825F0C0FA1021534834
S3150802F80052F044FA44E0FB790C2B07D15B4825F009
S3150802F810B5FA09214D4852F039FA39E0FB790D2B30
S3150802F82007D1574825F0AAFA0A21484852F02EFA73
S3150802F8302EE0FB790E2B07D1524825F09FFA0B21B1
S3150802F840424852F023FA23E0FB790F2B07D14E48A0
S3150802F85025F094FA0C213D4852F018FA18E0FB7983
S3150802F860102B07D1494825F089FA0D21374852F05D
S3150802F8700DFA0DE0FB791946454825F07FFA002373
S3150802F8805FE0BB791946434825F078FA002358E029
S3150802F89041492E4852F098FF51F044FC04463E482E
S3150802F8A052F0EBFC05463C4852F0F3FC03461A4676
S3150802F8B02946204644F070FE0023FB60FB680133AC
S3150802F8C0FB60FB68C72B08D817F05EF80346184694
S3150802F8D018F098FC0346012B10D117F055F8034689
S3150802F8E0184618F08FFC0346012B02D12B4817F055
S3150802F8F0A1FF2B4825F042FA002322E040F0D4FC6F
S3150802F9000346184640F023FE0346012B11D140F068
S3150802F910CBFC0346184640F047FE0346012B08D1A6
S3150802F920204825F02BFA00BF1F4825F027FA0123A5
S3150802F93007E03B79184625F001FC642034F048FFBD
S3150802F940BCE718461037BD46B0BD00BF2C4401209F
S3150802F9508C690908AC690908CC690908EC690908BF
S3150802F9600C6A09082C6A09084C6A09086C6A0908AB
S3150802F9708C6A0908AC6A0908CC6A0908EC6A09089B
S3150802F9800C6B09082C6B09084C6B09086C6B090887
S3150802F9908C6B0908D06B0908E8430120046C090836
S3150802F9A0286C0908686C0908B86C090880B584B01F
S3150802F9B000AF0346FB710B46BB7113467B710023EE
S3150802F9C0FB60FB680133FB60FB68B3F5E17F15D288
S3150802F9D040F06AFC0346184640F0E2FC0346184625
S3150802F9E051F051FF0346002B08D116F0CDFF03460E
S3150802F9F0184618F007FC0346012B22D116F0C4FF5D
S3150802FA000346184618F0FEFB0346012B03D1C748E6
S3150802FA1017F010FF12E0C64825F0B0F940F044FC92
S3150802FA200346184640F0BCFC0346184651F02BFF25
S3150802FA300346002B02D0BF4825F0A0F9002300F0A8
S3150802FA40BBBFBB79012B40F09781FB79012B13D100
S3150802FA5040F02AFC0346184640F0A2FC0346184624
S3150802FA6051F0F4FE03460B2B40F09D87B24825F071
S3150802FA7085F9012300F0A0BFFB79022B13D140F0D0
S3150802FA8013FC0346184640F08BFC0346184651F011
S3150802FA90DDFE03460C2B40F08687A84825F06EF952
S3150802FAA0012300F089BFFB79032B13D140F0FCFB3D
S3150802FAB00346184640F074FC0346184651F0C6FE43
S3150802FAC003460D2B40F06F879D4825F057F9012311
S3150802FAD000F072BFFB79042B13D140F0E5FB034615
S3150802FAE0184640F05DFC0346184651F0AFFE034641
S3150802FAF00E2B40F05887934825F040F9012300F071
S3150802FB005BBFFB79052B13D140F0CEFB03461846A3
S3150802FB1040F046FC0346184651F098FE03460F2B62
S3150802FB2040F04187884825F029F9012300F044BFAF
S3150802FB30FB79062B13D140F0B7FB0346184640F073
S3150802FB402FFC0346184651F081FE0346102B40F05F
S3150802FB502A877E4825F012F9012300F02DBFFB798A
S3150802FB60072B13D140F0A0FB0346184640F018FCB9
S3150802FB700346184651F06AFE0346112B40F01387D6
S3150802FB80734825F0FBF8012300F016BFFB79082B12
S3150802FB9013D140F089FB0346184640F001FC0346A0
S3150802FBA0184651F053FE0346122B40F0FC8669486C
S3150802FBB025F0E4F8012300F0FFBEFB79092B13D1E7
S3150802FBC040F072FB0346184640F0EAFB0346184625
S3150802FBD051F03CFE0346132B40F0E5865E4825F0BD
S3150802FBE0CDF8012300F0E8BEFB790A2B13D140F0C9
S3150802FBF05BFB0346184640F0D3FB0346184651F012
S3150802FC0025FE0346142B40F0CE86544825F0B6F856
S3150802FC10012300F0D1BEFB790B2B13D140F044FB34
S3150802FC200346184640F0BCFB0346184651F00EFE42
S3150802FC300346152B40F0B786494825F09FF801235D
S3150802FC4000F0BABEFB790C2B13D140F02DFB03460C
S3150802FC50184640F0A5FB0346184651F0F7FD034641
S3150802FC60162B40F0A0863F4825F088F8012300F0BD
S3150802FC70A3BEFB790D2B13D140F016FB034618469B
S3150802FC8040F08EFB0346184651F0E0FD0346172B5B
S3150802FC9040F08986344825F071F8012300F08CBEBD
S3150802FCA0FB790E2B13D140F0FFFA0346184640F0B3
S3150802FCB077FB0346184651F0C9FD0346182B40F058
S3150802FCC072862A4825F05AF8012300F075BEFB7998
S3150802FCD00F2B13D140F0E8FA0346184640F060FBB2
S3150802FCE00346184651F0B2FD0346192B40F05B86CF
S3150802FCF01F4825F043F8012300F05EBEFB79102B5E
S3150802FD0040F0518640F0D0FA0346184640F048FBC8
S3150802FD100346184651F09AFD03461A2B40F04386CD
S3150802FD20144825F02BF8012300F046BEDC6C0908BE
S3150802FD30046D0908406D09087C6D0908C46D090837
S3150802FD400C6E0908546E09089C6E0908E46E0908C7
S3150802FD502C6F0908746F0908BC6F09080470090832
S3150802FD604C70090894700908DC700908247109089E
S3150802FD706C710908B4710908BB79012B40F07181CD
S3150802FD80FB79012B13D140F08FFA0346184640F04F
S3150802FD9007FB0346184651F059FD03461B2B40F054
S3150802FDA00286C94824F0EAFF012300F005BEFB7962
S3150802FDB0022B13D140F078FA0346184640F0F0FABF
S3150802FDC00346184651F042FD03461C2B40F0EB85CC
S3150802FDD0BE4824F0D3FF012300F0EEBDFB79032BC6
S3150802FDE013D140F061FA0346184640F0D9FA0346A1
S3150802FDF0184651F02BFD03461D2B40F0D485B44816
S3150802FE0024F0BCFF012300F0D7BDFB79042B13D1E4
S3150802FE1040F04AFA0346184640F0C2FA0346184624
S3150802FE2051F014FD03461E2B40F0BD85A94824F067
S3150802FE30A5FF012300F0C0BDFB79052B13D140F0C5
S3150802FE4033FA0346184640F0ABFA0346184651F011
S3150802FE50FDFC03461F2B40F0A6859F4824F08EFF23
S3150802FE60012300F0A9BDFB79062B13D140F01CFA39
S3150802FE700346184640F094FA0346184651F0E6FC43
S3150802FE800346202B40F08F85944824F077FF012300
S3150802FE9000F092BDFB79072B13D140F005FA034611
S3150802FEA0184640F07DFA0346184651F0CFFC034641
S3150802FEB0212B40F078858A4824F060FF012300F060
S3150802FEC07BBDFB79082B13D140F0EEF903461846A1
S3150802FED040F066FA0346184651F0B8FC0346222B50
S3150802FEE040F061857F4824F049FF012300F064BD94
S3150802FEF0FB79092B13D140F0D7F90346184640F08F
S3150802FF004FFA0346184651F0A1FC0346232B40F04C
S3150802FF104A85754824F032FF012300F04DBDFB796E
S3150802FF200A2B13D140F0C0F90346184640F038FAB6
S3150802FF300346184651F08AFC0346242B40F03385C3
S3150802FF406A4824F01BFF012300F036BDFB790B2B10
S3150802FF5013D140F0A9F90346184640F021FA0346A0
S3150802FF60184651F073FC0346252B40F01C85604861
S3150802FF7024F004FF012300F01FBDFB790C2B13D1DB
S3150802FF8040F092F90346184640F00AFA0346184624
S3150802FF9051F05CFC0346262B40F00585554824F0B3
S3150802FFA0EDFE012300F008BDFB790D2B13D140F0BD
S3150802FFB07BF90346184640F0F3F90346184651F012
S3150802FFC045FC0346272B40F0EE844B4824F0D6FE28
S3150802FFD0012300F0F1BCFB790E2B13D140F064F932
S3150802FFE00346184640F0DCF90346184651F02EFC43
S3150802FFF00346282B40F0D784404824F0BFFE01234D
S3150803000000F0DABCFB790F2B13D140F04DF9034608
S31508030010184640F0C5F90346184651F017FC03463F
S31508030020292B40F0C084364824F0A8FE012300F0AB
S31508030030C3BCFB79102B40F0B68440F035F9034670
S31508030040184640F0ADF90346184651F0FFFB034640
S315080300502A2B40F0A8842B4824F090FE012300F0B5
S31508030060ABBCBB79012B40F08B81FB79012B13D1F8
S3150803007040F01AF90346184640F092F90346184623
S3150803008051F0E4FB03462B2B40F08D841E4824F0E5
S3150803009075FE012300F090BCFB79022B38D140F0A2
S315080300A003F90346184640F07BF90346184651F010
S315080300B0CDFB03462C2B40F07684144824F05EFED1
S315080300C0012300F079BC00BFFC71090844720908D2
S315080300D08C720908D47209081C7309086473090821
S315080300E0AC730908F47309083C740908847409088D
S315080300F0CC740908147509085C750908A4750908F8
S31508030100EC750908347609087C760908C476090863
S31508030110FB79032B13D140F0C7F80346184640F082
S315080301203FF90346184651F091FB03462D2B40F041
S315080301303A84C14824F022FE012300F03DBCFB7932
S31508030140042B13D140F0B0F80346184640F028F9BB
S315080301500346184651F07AFB03462E2B40F02384B8
S31508030160B64824F00BFE012300F026BCFB79052BC9
S3150803017013D140F099F80346184640F011F903469F
S31508030180184651F063FB03462F2B40F00C84AC480A
S3150803019024F0F4FD012300F00FBCFB79062B12D1E2
S315080301A040F082F80346184640F0FAF80346184624
S315080301B051F04CFB0346302B40F0F583A14824F05D
S315080301C0DDFD0123F8E3FB79072B12D140F06CF828
S315080301D00346184640F0E4F80346184651F036FB42
S315080301E00346312B40F0DF83974824F0C7FD0123EC
S315080301F0E2E3FB79082B12D140F056F8034618467A
S3150803020040F0CEF80346184651F020FB0346322B3E
S3150803021040F0C9838D4824F0B1FD0123CCE3FB7973
S31508030220092B12D140F040F80346184640F0B8F8B7
S315080302300346184651F00AFB0346332B40F0B383B3
S31508030240834824F09BFD0123B6E3FB790A2B12D1DD
S3150803025040F02AF80346184640F0A2F80346184623
S3150803026051F0F4FA0346342B40F09D83794824F081
S3150803027085FD0123A0E3FB790B2B12D140F014F87B
S315080302800346184640F08CF80346184651F0DEFA42
S315080302900346352B40F087836F4824F06FFD01230F
S315080302A08AE3FB790C2B12D13FF0FEFF034618466F
S315080302B040F076F80346184651F0C8FA0346362B3B
S315080302C040F07183654824F059FD012374E3FB79F3
S315080302D00D2B12D13FF0E8FF0346184640F060F8AD
S315080302E00346184651F0B2FA0346372B40F05B83B0
S315080302F05B4824F043FD01235EE3FB790E2B12D101
S315080303003FF0D2FF0346184640F04AF8034618461C
S3150803031051F09CFA0346382B40F04583514824F0A4
S315080303202DFD012348E3FB790F2B12D13FF0BCFFC8
S315080303300346184640F034F80346184651F086FA41
S315080303400346392B40F02F83474824F017FD012332
S3150803035032E3FB79102B40F026833FF0A5FF0346D3
S31508030360184640F01DF80346184651F06FFA03463F
S315080303703A2B40F018833D4824F000FD01231BE384
S31508030380BB79012B40F08581FB79012B12D13FF014
S315080303908BFF0346184640F003F80346184651F008
S315080303A055FA03463B2B40F0FE82314824F0E6FC1F
S315080303B0012301E3FB79022B12D13FF075FF0346B4
S315080303C018463FF0EDFF0346184651F03FFA034639
S315080303D03C2B40F0E882274824F0D0FC0123EBE2CB
S315080303E0FB79032B12D13FF05FFF034618463FF014
S315080303F0D7FF0346184651F029FA03463D2B40F02A
S31508030400D2821D4824F0BAFC0123D5E2FB79042BDA
S3150803041036D13FF049FF034618463FF0C1FF03466E
S31508030420184651F013FA03463E2B40F0BC82134894
S3150803043024F0A4FC0123BFE20C77090854770908C2
S315080304409C770908E47709082C7809087478090859
S31508030450BC780908047909084C79090894790908C4
S31508030460DC790908247A09086C7A0908B47A090830
S31508030470FC7A0908447B09088C7B0908D47B09089C
S31508030480FB79052B12D13FF00FFF034618463FF0C1
S3150803049087FF0346184651F0D9F903463F2B40F028
S315080304A08282C04824F06AFC012385E2FB79062B85
S315080304B012D13FF0F9FE034618463FF071FF034693
S315080304C0184651F0C3F90346402B40F06C82B648F0
S315080304D024F054FC01236FE2FB79072B12D13FF07A
S315080304E0E3FE034618463FF05BFF0346184651F002
S315080304F0ADF90346412B40F05682AC4824F03EFC46
S31508030500012359E2FB79082B12D13FF0CDFE0346AE
S3150803051018463FF045FF0346184651F097F9034638
S31508030520422B40F04082A24824F028FC012343E2F0
S31508030530FB79092B12D13FF0B7FE034618463FF065
S315080305402FFF0346184651F081F90346432B40F023
S315080305502A82984824F012FC01232DE2FB790A2B00
S3150803056012D13FF0A1FE034618463FF019FF034692
S31508030570184651F06BF90346442B40F014828E4813
S3150803058024F0FCFB012317E2FB790B2B12D13FF076
S315080305908BFE034618463FF003FF0346184651F001
S315080305A055F90346452B40F0FE81844824F0E6FBC3
S315080305B0012301E2FB790C2B12D13FF075FE0346AA
S315080305C018463FF0EDFE0346184651F03FF9034639
S315080305D0462B40F0E8817A4824F0D0FB0123EBE16F
S315080305E0FB790D2B12D13FF05FFE034618463FF009
S315080305F0D7FE0346184651F029F90346472B40F020
S31508030600D281704824F0BAFB0123D5E1FB790E2B7E
S3150803061012D13FF049FE034618463FF0C1FE034692
S31508030620184651F013F90346482B40F0BC81664837
S3150803063024F0A4FB0123BFE1FB790F2B12D13FF072
S3150803064033FE034618463FF0ABFE0346184651F001
S31508030650FDF80346492B40F0A6815C4824F08EFB3F
S315080306600123A9E1FB79102B40F09D813FF01CFE85
S31508030670034618463FF094FE0346184651F0E6F83B
S3150803068003464A2B40F08F81514824F077FB012318
S3150803069092E1BB79C82B40F07F81FB79012B12D1FC
S315080306A03FF002FE034618463FF07AFE0346184615
S315080306B051F0CCF80346102B40F07581454824F0D9
S315080306C05DFB012378E1FB79022B12D13FF0ECFDA8
S315080306D0034618463FF064FE0346184651F0B6F83B
S315080306E00346112B40F05F813B4824F047FB012367
S315080306F062E1FB79032B12D13FF0D6FD0346184678
S315080307003FF04EFE0346184651F0A0F80346122B57
S3150803071040F04981314824F031FB01234CE1FB7950
S31508030720042B12D13FF0C0FD034618463FF038FEAE
S315080307300346184651F08AF803460B2B40F03381DB
S31508030740274824F01BFB012336E1FB79052B12D13D
S315080307503FF0AAFD034618463FF022FE0346184615
S3150803076051F074F803460C2B40F01D811D4824F004
S3150803077005FB012320E1FB79062B37D13FF094FDD6
S31508030780034618463FF00CFE0346184651F05EF83A
S3150803079003460D2B40F00781134824F0EFFA012393
S315080307A00AE100BF1C7C0908647C0908AC7C0908BB
S315080307B0F47C09083C7D0908847D0908CC7D090871
S315080307C0147E09085C7E0908A47E0908EC7E0908DC
S315080307D0347F09087C7F0908C47F09080C80090847
S315080307E0548009089C800908E4800908FB79072BCB
S315080307F012D13FF059FD034618463FF0D1FD034693
S31508030800184651F023F803460E2B40F0CC806C486B
S3150803081024F0B4FA0123CFE0FB79082B12D13FF079
S3150803082043FD034618463FF0BBFD0346184651F001
S315080308300DF803460F2B40F0B680624824F09EFA63
S315080308400123B9E0FB79092B12D13FF02DFD0346AD
S3150803085018463FF0A5FD0346184650F0F7FF034632
S31508030860182B40F0A080584824F088FA0123A3E007
S31508030870FB790A2B12D13FF017FD034618463FF0C2
S315080308808FFD0346184650F0E1FF0346192B40F047
S315080308908A804E4824F072FA01238DE0FB790B2BEC
S315080308A011D13FF001FD034618463FF079FD034693
S315080308B0184650F0CBFF03461A2B74D1444824F04C
S315080308C05DFA012378E0FB790C2B11D13FF0ECFCA0
S315080308D0034618463FF064FD0346184650F0B6FF34
S315080308E00346132B5FD13B4824F048FA012363E000
S315080308F0FB790D2B11D13FF0D7FC034618463FF081
S315080309004FFD0346184650F0A1FF0346142B4AD160
S31508030910314824F033FA01234EE0FB790E2B11D12B
S315080309203FF0C2FC034618463FF03AFD0346184615
S3150803093050F08CFF0346152B35D1284824F01EFAB0
S31508030940012339E0FB790F2B11D13FF0ADFC0346A8
S3150803095018463FF025FD0346184650F077FF034631
S31508030960162B20D11E4824F009FA012324E0FB792B
S31508030970102B18D13FF098FC034618463FF010FD9C
S315080309800346184650F062FF0346172B0BD115484A
S3150803099024F0F4F901230FE0BB791946124816F03F
S315080309A049FF002308E07B79184624F0C7FB642037
S315080309B033F00EFFFFF705B818461037BD4680BD5E
S315080309C02C81090874810908BC810908048209086D
S315080309D0508209089C820908E882090834830908B1
